:1000000000400020D57B0000157C0000177C00001C
:1000100000000000000000000000000000000000E0
:10002000000000000000000000000000197C00003B
:1000300000000000000000001B7C00001D7C000090
:100040001F7C000059590000817F00001F7C0000C8
:100050001F7C0000000000001F7C00001F7C0000CF
:1000600021380000558300001F7C00001F7C000029
:100070001F7C00001F7C00001F7C00001F7C000014
:100080001F7C0000058000001F7C00001F7C00001A
:100090001F7C00001F7C00001F7C00001F7C0000F4
:1000A0001F7C00001F7C000000000000000000001A
:1000B0000000000000000000000000000000000040
:1000C00010B5064C2378002B07D1054B002B02D02E
:1000D000044800E000BF0123237010BD700200201F
:1000E000000000000CF00000044B10B5002B03D002
:1000F0000349044800E000BF10BDC04600000000F6
:10010000740200200CF00000164B002B00D1144BA1
:100110009D46402292029A1A924600218B460F4633
:100120001348144A121A0BF049FF0F4B002B00D052
:1001300098470E4B002B00D0984700200021040068
:100140000D000D48002802D00C4800E000BF0BF065
:10015000F5FE2000290007F065FF0BF0C9FEC04640
:100160000000080000400020000000000000000027
:1001700070020020D42F00200000000000000000CA
:1001800002000120104011D1042A0ED91368180969
:1001900080B2002809D001388000031D11180979A8
:1001A000002902D001309842F8D170470020FCE7C6
:1001B0000378002B03D05AB2002A01DB01307047CC
:1001C0003F229343C03B59424B41C01803789343AD
:1001D000802BF4D10130F9E710B500240378002B0F
:1001E00001D1200010BDFFF7E3FF0134F6E770B541
:1001F000002204000D00411C092003F039FE0028F4
:1002000006D001236200134343600023A34200DBB6
:1002100070BD9A00A958821891600133F6E770B555
:10022000012803DC1C2001F0E9F970BD01230D68F1
:1002300011201D42F7D04868184206D1042804D97D
:100240000F2302681340042B01D00E20EBE703F0CC
:100250006DFC6D100400002D03DDFFF7BDFFA8420B
:1002600006DA1220DFE72000FFF7A2FF0400013DBD
:10027000012DF8D120787F2809DDDF280BDCF82359
:100280003F22DB00800118406378134018430123AC
:1002900040001843C9E7EF280BDCFC226378120109
:1002A0009B0113403F220007000C0343A07810403D
:1002B000ECE7F72812DCFC22637892021B03134060
:1002C000E0228004520310403F221843E378134099
:1002D000FC220343A07812018001E8E7012040429C
:1002E000D5E7F8B54D680F00EB0706D4042D04D907
:1002F0000F232E683340092B03D00B2001F07EF929
:10030000F8BD6B683609B6B25C10731EA3420FD8F5
:100310000321200009F00EFD6421642803DC0100A4
:10032000032800DA03212800891903F0D3FD050012
:100330002B6800201B099BB2013B9C42E0D23A682B
:10034000A31C9B005A510123013464001C436C60C0
:10035000D6E7F0B585B0012803DC1C2001F04EF98A
:1003600012E001274B683A000093022806D08B6800
:100370003B4203D05F10002F00DC17000125009BDB
:100380002B4203D00120404205B0F0BD009B042B5E
:10039000F8D91B680C680F261900314004292DD1AB
:1003A0002C4205D1042C03D923681E40042E01D011
:1003B0000E20D3E70098FFF7E3FEB842E2DB009897
:1003C00003F0B4FB0600200003F0B0FB037801004B
:1003D000002BD7D0781E30180CF0A6F9041ED1D00F
:1003E0003378002B01D0A64202D36800012521E01A
:1003F0003000FFF7DDFE01350600F1E709293ED1A7
:10040000009B5B685B1001939F42BBDC2C422ED1AA
:10041000042C2CD923683340042B28D1200003F06E
:1004200085FB039602907E1C009AB300D05884424C
:1004300002D178002843A7E728420ED104280CD91E
:100440000368039A1340042B07D103F06FFB0100EC
:1004500002980CF033F90028EBD0019B37009E4244
:10046000E1DD8FE71F00019B9F4200DD8AE77B1CD7
:1004700000999A008A58A242F4D17800B6E703297D
:1004800000D07FE71A0992B25B0F92000B40D31A9B
:1004900001939F4200DD75E72C4229D1042C27D916
:1004A00022681640032E19D1100980B2520F800025
:1004B0003240251D801A019B2E181B1A0193009BA8
:1004C000781E0433019A904200DD5BE72A00191878
:1004D000B2420FD316D10130400087E7042E07D176
:1004E000200003F023FB05002000FFF749FEE2E7B0
:1004F0000F2033E70C78A4461478A44502D10131CB
:100500000132E5E70130DDE7F0B50C0085B00128E8
:1005100004DC1C2001F072F805B0F0BD012708686A
:10052000384206D1042804D90F2102680A40042A5F
:1005300001D00E20EEE762681740FAD1042AF8D9FC
:1005400013680B40042BF4D103F0F0FA0500606847
:1005500003F0ECFA02900CF0BBF8039003002800C3
:10056000002B19D1FFF738FE0190019B0122591C85
:10057000092003F07DFC334E306000280ED10020AE
:10058000CAE7039B0299C0180CF0CEF80196019BB4
:100590005E1C0028F5D1E8E70197F8E70122019BEE
:1005A0005B0013434360039B002B18D12800FFF727
:1005B000FFFD019B0400BB4201DC3068ACE7611B1E
:1005C000280003F0D3FC0028D9D0BB1C32689B0064
:1005D00098502000FFF7ECFD01372500E9E7019B6B
:1005E000012B02D12368836096E7681C02990CF006
:1005F0009BF801240700019B002F13D0A342DCDBF2
:10060000791B280003F0B2FC0028B8D0326801340E
:10061000A3009850039B0299FD1828000CF084F861
:100620000700E8E7A342C8DB28000CF051F80100FE
:10063000280003F09BFC0028A1D001343368A400FB
:10064000E050BAE7E40F002010B503F053FA43007E
:100650000120184310BD0000C30711D404280FD98E
:100660000F2302681340032B0AD119400133591A92
:10067000C0234907DB051940024B1A4011430160B2
:100680007047C046FFFFFF9FF7B507000E001C2014
:10069000012F06DD4C68012322001A40009203D18D
:1006A0000D2000F0ABFF53E0022F02D08A681A42FF
:1006B000F6D0012335681D4200D0A9E0042D00D8F2
:1006C000A6E01C41002C00DC1C000F20296808401B
:1006D000092828D16B685B100093022F05D0B368FE
:1006E000009A5B109A4200DD0093009B01221D1BC3
:1006F0000135EB43DB171D40691C092003F0B8FBF3
:10070000071E09D001236D001D4303003268083322
:1007100045600099A14201DA3800FEBD0134A10014
:10072000515802C3F5E7042845D1280003F0FEF92B
:10073000FFF752FD0190022F04D0B3685B1098427E
:1007400000DD0193019BA34204DA002003F002FCC8
:100750000700E1E7280003F0E9F90700009BA34246
:1007600021DB2800009703F0E1F905003800FFF7CE
:100770001FFD019B01340700A342F7DA009BC41A56
:10078000200003F0E7FB071EC6D003F0CFF901906D
:10079000306803F0CBF92200009B591B41180198E7
:1007A0000BF0F0FBB8E73800FFF702FD009B0700F5
:1007B00001330093D2E703282AD10B099BB2490FDA
:1007C0009B000140591A022F04D0B2685210914286
:1007D00000DD1100A14205DA00220320110003F020
:1007E00047FBB5E703200E1B331DD9170140C9187D
:1007F0008910002203F03CFB071E00D18CE7013674
:1008000031000334FFF728FF381D29193200C7E7EC
:10081000212046E7F7B5002804DC1C2000F0EEFE9E
:10082000040014E00D6801272E003E4011D03D4128
:10083000FF2D01D91320F1E700223900032003F036
:1008400017FB041E03D00021FFF706FF25712000CF
:10085000FEBD042DEED90F232A681340042B1BD1B3
:100860002800FFF78DFCC31C07000320D9170140A7
:10087000C9188910320003F0FBFA041EE7D03900D2
:10088000FFF7EAFE280003F051F9231D01003A00AA
:1008900018000BF077FBDAE7092B1FD103206B68F8
:1008A00032005B1001930333D9170140C918891036
:1008B00003F0DEFA041ECAD00199FFF7CDFE019BBA
:1008C0009E42C4DAB300EB189B683B4204D05B1035
:1008D000FF2BAFD8A21913710136F0E7032BA9D172
:1008E0002C00B4E710B57F2902DC0170013010BD87
:1008F0001A4B99420CDC40238A115B42134303706C
:100900003F230B4080214942194341700230EEE7FA
:10091000134B994210DC20230A135B4213433F24FC
:10092000802203708B1152422340214013430A431B
:10093000437082700330DAE70A4B9942D7DCF02328
:100940000370603B4370113B8A11FF3B1A43827076
:100950003F2211401943C1700430C8E7FF0700006F
:10096000FFFF0000FF0F0100F0B50D0085B000286B
:1009700003DC1C2000F042FE0DE0096801220800A3
:1009800010400AD002AC11412000FFF7ABFF011B61
:10099000200003F0EBFA04001AE004293FD90F23EA
:1009A0000C682340092B3AD14B685B100193032359
:1009B0009C46019B9A420EDD03F0CCFA041E07D040
:1009C0002E68012503F0B2F82F00019B9D421DDD2A
:1009D000200005B0F0BD01329300CC580123234024
:1009E00001D10D20C6E764107F2C0DDD0D4E0223D2
:1009F000B44209DD0C4E6346B44205DD00270B4EC0
:100A0000E30FA6427B419B00C018D2E70135AB0043
:100A1000F1583942E5D04910FFF764FFD5E72120AE
:100A2000A8E7C046FF070000FFFF0000FF0F01001E
:100A300070B5002805DC1C2000F0E0FD0500280052
:100A400070BD0C68E30701D40D20F5E76410E343A3
:100A5000DB171C40E11C89100022032003F008FA78
:100A6000051EECD02100FFF7F7FDE8E710B5040004
:100A70000120084010D104290DD90F230A68134022
:100A8000042B08D1080003F051F8010020000BF0FE
:100A900015FE4342584110BD0020FCE7F7B50F009A
:100AA000012803DC1C2000F0A9FDFEBD01264D68D5
:100AB0002E4006D1042D04D90F222B681A40092A92
:100AC00001D00B20EFE76A681B099BB25410A342C8
:100AD00000D85C1E39681E48FFF7C8FF012301904B
:100AE000002813D139681B48FFF7C0FF002811D038
:100AF000002C0DD00123621C013C9C4092005351FC
:100B000023436B6004E00136B200AB50B442FADA22
:100B10000020CAE73B680D20DA07C4D55B10002B24
:100B200011DD9C420FDB9B00A200291DEB188918E8
:100B30000433994209D10123013C9C40AA181C436B
:100B400053606C60E4E71220ADE758681860EFE787
:100B50005FD6000063D60000002310B50C000B70B8
:100B6000C30705D50D49421020000BF06BFD08E0CE
:100B70000B49002802D0042804D10A4920000BF0B8
:100B800081FD10BD0428FCD90F2302681340042BFB
:100B9000F7D102F0CBFF04490200E5E704E10000D1
:100BA00068D600006ED6000073D60000F0B593B092
:100BB000060002911C20012E1DDD029B01251B68F1
:100BC0001C002C4000D0ADE0042B00D8E6E01A68F1
:100BD0000F231A40092A4AD10394039A02999200DA
:100BE0008A5817002F4005D1042A03D910681840ED
:100BF000092806D0222000F001FD0190019813B0D1
:100C0000F0BD52685210A418039A01320392964222
:100C1000E3D1611C012203F02BF90190002802D1DD
:100C200000230193EAE7019B6400190025435D60FE
:100C30000831029ABB00D05802684368120992B288
:100C40005B109A4200D8531E0022934209DCDA431B
:100C5000D21713409B00C918039B01379F42E8DB62
:100C6000CCE794000519AD6801320D51EDE727007E
:100C7000032A59D10193029ABB00D3582B42B9D110
:100C8000042BB7D9186801990140032939D1020909
:100C900092B2430F92000B40D31A1C190137BE4287
:100CA000E9D10320E31CD9170140C918891000229B
:100CB00003F0DEF801900028B2D000252100FFF7F4
:100CC000CBFC019B1E1D029AAB00D45801231C4291
:100CD0001FD1042C1DD90F2123681940032918D1D5
:100CE000180980B25B0F80000B40C01A00238342BA
:100CF00013DBC343DB17184001353618BD42E2DB76
:100D00007CE7042900D075E71800FFF739FA2418AA
:100D1000C4E72000FFF734FAE8E7E2181279F2544A
:100D20000133E4E700273C000F25029ABB00D358AB
:100D30000122134234D1042B32D918680100294012
:100D4000042935D11800FFF71BFA24180137BE42D9
:100D5000EBD1200003F0FEF80190002800D15FE7FE
:100D6000029FB600BB19041D029301233D681D427A
:100D700029D1042D27D90F262B681E40042E37D1E8
:100D80002800FFF7FDF90600280002F0CFFE010061
:100D9000200032000BF0F6F8A41922E02700C3E788
:100DA000180005A9FFF7D8FE05A80BF091FCCCE7C9
:100DB000032900D01EE7020992B2430F92000B40B4
:100DC000D31A1C19C2E705A92800FFF7C5FE05A81C
:100DD0000BF07EFC05A90500020020000BF0D2F804
:100DE0006419029B0437BB42BFD10023237005E77F
:100DF000032EF6D11A0992B25B0F92001E40961B89
:100E0000291DC5E7F0B50D0097B0002806DC1C20B1
:100E100000F0F4FB0700380017B0F0BD0C680121AA
:100E200023000B40009306D1042C04D922680F3311
:100E30001A40092A01D00B20EAE762685210039297
:100E4000002A03DC009803F085F8E3E7504A01929A
:100E500001280BD06868084208D1042806D9026826
:100E60001340042B02D102F061FE019001980BF0B7
:100E70002FFC06000F27039B0834013B05935E43BC
:100E8000039B02909B00E3180493012320681842FF
:100E900073D1042871D901680B003B409C46042B98
:100EA00003D1FFF76DF9861909E0032B6CD1624677
:100EB0000B099BB2490F9B0011405A1A9619049BCB
:100EC0000434A342E1D1300003F044F8071EA2D05D
:100ED0002B680793029B002B03D0686802F026FE64
:100EE0000190380002F022FE0400009B079A9B004C
:100EF000D3189E68300002F019FE0123334005002C
:100F00000693002B01D1042E04D809A93000FFF765
:100F100023FE09AD28000BF0DBFB069B0490002BA1
:100F20000ED1042E0CD90F2133681940032907D1A3
:100F30001A0992B25B0F92000B40D31A351D04932D
:100F40002000049A29000BF01DF8049BE418029B72
:100F5000002B0AD0059B009A934206DD2000029ADE
:100F600001990BF00FF8029BE418009B01330093EA
:100F7000009A039B9342B8D14DE709A9FFF7ECFD16
:100F800009A80BF0A5FB8EE702F0D0FDF9E7C046FB
:100F900023DB000010B50024A04207DD0B680134FC
:100FA0001C4003D05C10E343DB171C40611C012292
:100FB000092002F05DFF002803D0012364001C43D8
:100FC000446010BD0A6870B510000125284034D176
:100FD000042A32D90F24136849681C40092C17D100
:100FE00054681B099BB22C41A34200D85C1E84426A
:100FF00005DC02200133984206DB00200FE085006B
:101000005519A9600130F2E7840011510130F2E76F
:10101000032C12D1294203D1132000F0EFFA70BD46
:101020004910FF29F8D81B099BB204329B00D31842
:101030009342E2D911700132FAE70B2000F0DEFA98
:10104000DBE70000F8B5012700254E680C003740AB
:10105000AF420ED13D00042E0BD90F2233681A4047
:10106000092A10D172681B099BB25510AB4200D8F7
:101070005D1E2168CB0716D54C10002C01DDA54262
:101080001CDA122030E0042A04D13000FFF778F88F
:101090000500EEE7032AECD11D09ADB25B0FAD00F0
:1010A0001340ED1AE5E72748FFF7E0FC002813D0CE
:1010B0000BF064FA290008F023FF4C1C002F3ED1EE
:1010C000042E3CD90F2332681340092B10D1013470
:1010D000A400A4592000F8BD21681B48FFF7C6FCF6
:1010E0002C000028EAD1113000F088FA0400F1E762
:1010F000042B1CD1300002F019FD0500012C0EDC80
:10110000FFF756F8461B300002F024FF041EE1D022
:1011100002F00CFD320029000AF034FFDAE72B78E8
:10112000013C002BADD02800FFF742F8E5E7032B88
:1011300005D13419E37801245B001C43CAE70B2076
:10114000D2E7C04658D6000063D60000F7B54D6818
:101150000F002A0001210A402FD1042D2DD90F2480
:101160002B68BE681C40092C14D169681B099BB20E
:101170004C100192A34200D85C1E39682A48FFF740
:1011800075FC00282DD00F232A681340092B1DD190
:10119000012317E0032C10D10E4203D1132000F0DD
:1011A0002DFAFEBD72100192FF2AF7D81A0992B2E9
:1011B0005B0F92001C40141BDFE70B20EFE70133AD
:1011C0009A00AE509C42FADA0020EAE7032BFBD1EA
:1011D0002B0001335A1BA242F6DC6A461279DA7000
:1011E000F7E73968CB0706D54910002901DD8C42A5
:1011F00009DA1220D3E70D48FFF738FC2100002858
:1012000001D11130CBE70F232A681340092B03D1FA
:10121000013189004E51D7E7032BD5D16B461B799D
:101220006D18EB70D0E7C0465FD6000063D60000B3
:1012300070B501240868204207D1042805D90F257C
:1012400001680D40092D02D14468200070BD032DB6
:1012500008D10A0992B24B0F92002B40D31A5B00BF
:101260001C43F2E7042DF0D102F060FCFEF7B4FF5E
:1012700040000443E9E7000010B5034A0D2103488C
:1012800004F03EFC10BDC046F0D50000E8D50000DB
:1012900000207047042070470120704710B50020DF
:1012A00002F058FE10BD002070470020704700205B
:1012B00070470020704700207047002070470020D2
:1012C000704700207047000010B5034A0C21034806
:1012D00004F016FC10BDC046F8D6000058D7000038
:1012E00070470378002B03D05AB2002A01DB01308B
:1012F00070473F229343C03B59424B41C01803788B
:101300009343802BF4D10130F9E70000F8B50127B1
:10131000060014000800394227D104293FD90F23C1
:101320000A681A40042A3AD13C4213D1042C11D93C
:1013300022681340042B0DD102F0F8FB05002000B9
:1013400002F0F4FB010028000BF0B8F900282EDBB6
:101350001FD127E0E30722D502F0E8FB0A22002193
:101360000BF07EFA0500601010E0174015D1042A3A
:1013700015D90F2312681340042B10D120004D10F3
:1013800002F0D4FB0A2239000BF06AFA85420EDB28
:1013900008DD002E09DC00200CE04D10E3E70F22F1
:1013A000054B1A700136022EF5D8042002E0042005
:1013B00076173040F8BDC046B0020020F8B50600F0
:1013C0000024294BE500ED182B79032B06D00134BE
:1013D000FF2CF6D1013CFF3C2000F8BD30000BF0A3
:1013E00077F9E3B202003100180004F0C5FB0028D1
:1013F000F2D12A6851688842E9D08300D3189B68EB
:101400000130F02BF7D101238000083012181A4266
:10141000DDD1042ADBD90F21136819400429D6D164
:101420001B0998B201230130800010181842CED158
:101430000428CCD90F2203681340042BC7D102F033
:1014400075FB03270500092128000BF029F9002866
:10145000BDD0013F451C002FF5D1310028000BF015
:1014600063F98542B8D0B2E7A825002010B5012461
:10147000044002D04410200010BD042810D90F23CE
:1014800002681340042B07D102F050FB21000A220E
:101490000BF0E6F90400EEE7032B01D10430F5E789
:1014A0000D22014B1A70E6E7B0020020012210B5B0
:1014B000024018D1042802D903681A0992B2012304
:1014C0000B4012D1042902D90B681B099BB20024DE
:1014D000934206D104309B000431C318984206D3CE
:1014E0000124200010BD0022E9E70023EFE7047883
:1014F0000A78002C01D1002AF2D001300131944247
:10150000ECD00024EDE70000F7B50700009101934F
:101510003049314B002A02D002220A70013A0026DB
:101520001A601B68CE54BE4200DBF7BD009AB300C0
:10153000D058294B274D1C68C8239B0065191C1BDC
:101540000123184206D0254A4310210028000BF041
:1015500047F809E0224A002802D004281BD1214A7A
:10156000210028000BF03CF81A4C20000BF0B0F8DA
:10157000194A019B1060002B0BD07B1EB34208DD83
:10158000194B984205D8431C136020222254002294
:10159000E2540136C7E7042819D90F2301680B402C
:1015A000042B04D102F0C2FA104A0300CDE7092B44
:1015B00003D143680E4A5B10C7E7032B08D10A0921
:1015C00092B2490F92000B40D31A0A4ABDE7012399
:1015D000094ABAE7B1020020D405002004E1000066
:1015E00068D600006ED600001F0300002FE7000041
:1015F000C8D90000D7D90000E2D90000014B18700B
:1016000000207047B002002070B501F0E5FF094CE2
:101610000100251D1F2228000BF072F828000BF096
:1016200057F804230430800800011843206020008C
:1016300070BDC0468C020020C368F0B59D00836871
:1016400089B05D190300183306930369069A9F0059
:10165000069B0290DF19436901939B00D318039303
:10166000D14B1B78002B26D17F222B68CF491C122F
:1016700013409B005B58043501929F46029B5878AB
:1016800004F096FE0023029A137027E0C64B1B78E5
:10169000002B10D12B68019A1C121340C34A9B00E7
:1016A0009B580435E9E7069B3A1DD11ABE4BD82951
:1016B00028DD1A221A70029BBB4C9B68217801938B
:1016C000EA1A029B92109B7812021A43029B5878E6
:1016D00004F076FE0023029A23701370029B069A90
:1016E0009B680193ED1A029BAD10DD60069BFE1A0C
:1016F000029BB6101E61039B9B1A029A9B105361BA
:1017000009B0F0BD39001B7817000C60002BD2D156
:101710002B68019A1C121340A44A9B009B58043565
:10172000ABE7069B3A1DD11A9F4BD82902DD1A223E
:101730001A70C0E738001B7817002A68291D02605C
:10174000002B01D00D00B6E76B68019A1C12134004
:10175000964A9B009B5808358FE7069B3A1DD11A85
:10176000914BD82902DD1A221A70A4E73900A4008F
:101770001B782C1917000C60002B9CD12B68019A48
:101780001C121340894A9B009B58043575E7069B41
:101790003A1DD11A844BD82902DD1A221A708AE721
:1017A00039001700824AA400A2581B780A60002B57
:1017B00000D080E72B68019A1C1213407B4A9B00E3
:1017C0009B58043559E7043F794B3A68A400E2502E
:1017D000754B1B78002B00D06DE72B68019A1C120B
:1017E0001340724A9B009B58043546E7704BA40097
:1017F000E058FFF73BFE6C4B06001B78002B09D12D
:10180000043F3868FFF732FE0123861976001E4335
:10181000674BE650644B1B78002B00D04BE72B68DE
:10182000019A1C121340614A9B009B58043524E71F
:10183000069B391DCA1A5C4BD82A02DD1A221A707F
:1018400039E70698039C0122A04202D222000C3AFA
:10185000126838001B780F000260002B00D02AE7C6
:101860002B68019A1C121340504A9B009B58043568
:1018700003E7069A3B1D991A4B4AD82902DD1A2321
:10188000137018E706990398814219D202000C3AA6
:101890001068484A4010A418241A039AA400A258B9
:1018A0003A601F00404B1B78002B00D003E72B68E9
:1018B000019A1C1213403D4A9B009B580435DCE6FC
:1018C000182111700022EBE7069B039A934219D26C
:1018D00013000C3B1868374B043FE418130040100A
:1018E000241A3A68A400E2502F4B1B78002B00D03A
:1018F000E1E62B68019A1C1213402C4A9B009B586E
:101900000435BAE61822284B1A70EDE7069B039AB5
:10191000934228D2274B043FE61814000C3C23685E
:101920005B10F31A9B009858FFF7A0FD04903868ED
:10193000FFF79CFD2468049B6410341B1E180123D0
:1019400076001E43039BA400E650174B1B78002B28
:1019500000D0B0E62B68019A1C121340134A9B007A
:101960009B58043589E618220F4B1A70EDE7069B49
:101970003A1DD11A0C4BD82902DD1A221A709AE6A8
:1019800039001700039AA400A2581B780A60002BA4
:1019900000D090E62B68019A1C121340034A9B006A
:1019A0009B58043569E6C046B0020020C8D7000045
:1019B000A02D0020FDFFFF3F043F039B3A68A400D9
:1019C000E250D64B1B78002B00D074E62B68019AAE
:1019D0001C121340D24A9B009B5804354DE6039BD2
:1019E000A4001C192368043F38685E10FFF73EFD11
:1019F0000123361876001E43C84B26601B78002B47
:101A000000D058E62B68019A1C121340C44A9B0070
:101A10009B58043531E6069BA4003F1BBF4CBB42DC
:101A20000CD82378002B00D045E62B68019A1C12B5
:101A30001340BB4A9B009B5804351EE6B94802F090
:101A400065F82378002B00D035E62B68019A1C122C
:101A50001340B34A9B009B5804350EE6A300ED18D3
:101A6000002C00DA3AE6AD4B1B78002B00D022E6C2
:101A70002B68019A1C121340A94A9B009B580435FD
:101A8000FBE5043F3B68042B04D1A300ED18002CB8
:101A900000DA23E6A14B1B78002B00D00BE62B6865
:101AA000019A1C1213409E4A9B009B580435E4E5A2
:101AB000043F3B68042B04D0A300ED18002C00DA8F
:101AC0000CE6964B1B78002B00D0F4E52B68019AAE
:101AD0001C121340924A9B009B580435CDE501230C
:101AE0003E1F306818420AD018410138002809DB2F
:101AF00001234000A40018432D193060EEE5FFF7E4
:101B0000B5FCF2E7854B1B78002B01D03700D2E5FE
:101B10002B68019A1C121340814A9B009B58370086
:101B20000435AAE5FF20610040000140FE38FF387F
:101B30000143396002993B008968241204916D1AAF
:101B40000299AD1089782D020D43854005437D60D3
:101B500006991700039A521A9210824002439A6023
:101B6000029B029A9C70E4B26F4BE400E3589360CE
:101B70006A4A1278002A03D008331D0003979AE5B9
:101B80001D00019A9B680C351C121340644A9B008F
:101B90009B58039771E53B1F1C68039A069B934271
:101BA00032D10A20E30711D4042C18D90F2322685C
:101BB0001340042B16D1200001F0B8FF0AF088FD75
:101BC000C8239B00984200D918000630643004F006
:101BD00007F800280FD1043D069B03937EE50720FC
:101BE000042CF3D02000431E9841FA234042FF33D7
:101BF00018400730EAE7029B2100587804F0F2FB16
:101C00000023029A1370E7E7039B039A0C3B1B68BF
:101C100002995B109B00D31A0C3B1C601F1D130024
:101C2000083B1B685A108A70D2B23F49D2005B0051
:101C300055589B0A029A9B009560ED18039B069AE3
:101C4000043B1B685B109B00D3180393334B1B783A
:101C5000002B00D02FE52B68019A1C121340304A4C
:101C60009B009B58043508E53B1F1868FFF7FEFBF7
:101C7000A40006003F1B1E2827DC00280DDC274B94
:101C80001B78002B00D016E52B68019A1C1213401C
:101C9000234A9B009B580435EFE401F083FC033E8C
:101CA000361801F07FFC214B801B9842F9D81B4B62
:101CB0001B78002B00D0FEE42B68019A1C12134005
:101CC000174A9B009B580435D7E40123029A1370EE
:101CD00001F068FC029B0A3886195E60FEE43B1F37
:101CE0001868FFF7C3FBA40006003F1B00280DDCAB
:101CF0000A4B1B78002B00D0DDE42B68019A1C12E4
:101D00001340074A9B009B580435B6E4084B9842A1
:101D100010DD1D22014B1A70CDE4C046B002002038
:101D2000C8D70000F4D90000A82500203F420F00CA
:101D300080EE36000123029A137001F033FCFA237F
:101D40009B005E430A3E3018029B5860C6E4A30025
:101D5000FF1A002320001A003900FFF7D5FBD74EE9
:101D6000D74C3168200002F001F9D64B3168186079
:101D7000200004F0F7F93168200004F03AFBD24B60
:101D80001B78002B00D096E42B68019A1C1213409C
:101D9000CE4A9B009B5804356FE4CB4BA4001B78C4
:101DA0003F1B002B00D086E42B68019A1C121340C5
:101DB000C64A9B009B5804355FE4029803F074FF09
:101DC000C14B1B78002B00D075E42B68019A1C12C4
:101DD0001340BE4A9B009B5804354EE43B1F1B68D2
:101DE000002B58D13B0001260C3B186806402FD031
:101DF00046103A0001217300083A0B431360002E8D
:101E000000DC95E0012173000B433A1F13603B0097
:101E1000083B1B680B419B1B04933B000C3B186861
:101E200008423BD0049BA4005B188B400B43039AF1
:101E3000A350A54B1B78002B00D03CE42B68019AE3
:101E40001C121340A14A9B009B580435FFF715FC58
:101E500004281BD90F2302681340092B02D14368C1
:101E60005E10C6E7042B08D101F060FE0378002B5A
:101E7000BFD0FFF736FA0136F8E7032B06D1160973
:101E8000B6B2520FB6001340F61AB2E719228E4BC3
:101E90001A70FFF710FC5B105E1EB0E7042842D9F1
:101EA0000F2302681340092B05D1049BA4000233C1
:101EB0009B001B58BBE7042B2BD1039BA4001B19D1
:101EC000079301F033FE0600049C0134012C10DC62
:101ED0003000FFF706FA831B1800049302F03AF86B
:101EE000041E0ED001F022FE049A31000AF04AF8D6
:101EF00007E03178013C002906D112220C00724B18
:101F00001A70079B1C6094E73000FFF7EAF906009F
:101F1000DCE7032B07D10122049BA400C3181B7923
:101F20005B00134383E71922674B1A70FFF7C3FB6B
:101F300004357EE7A300069AFB189B1AD82B08DD10
:101F40001A22614B1A70FFF7B6FB01221C003A609F
:101F50000437631E002CF8DC5B4B1B78002B01D090
:101F6000FFF7A9FB2B68019A1C121340574A9B00EC
:101F70009B580435FFF781FB069A3B1D9B1A524E76
:101F8000D82B03DD1A233370FFF795FB069B039ACA
:101F9000A40093422AD23B1F1868FFF767FA011E7C
:101FA00021DD039B0C3B1A68521082421BDB900719
:101FB000801A474B4018C018039B8000C2583B1B37
:101FC0001A60414B3F1B1B780437002B01D0FFF7F1
:101FD00072FB2B68019A1C1213403C4A9B009B58D1
:101FE0000435FFF74AFB20233370EAE71823FBE7A9
:101FF000344BA4001A683B1B1F001A60324B043795
:102000001B78002B01D0FFF756FB2B68019A1C129E
:1020100013402E4A9B009B580435FFF72EFB3A1FB6
:102020001368042B02D13A00A4002D19264B1B780B
:10203000002B02D01700FFF73EFB2B6801991C1202
:102040000B4022499B005B5817000435FFF715FB36
:10205000043F3B68042B04D00023A4003B602D19EF
:102060000437194B1B78002B01D0FFF724FB2B689A
:10207000019A1C121340154A9B009B580435FFF728
:10208000FCFAA3009C46F81A002C23DC1C22002634
:102090000D4B1A706346FF1A0B4B06601B78043712
:1020A000002B01D0FFF707FB2B68019A1C1213408D
:1020B000064A9B009B580435FFF7DFFAD405002041
:1020C000B102002008000020B0020020C8D70000A4
:1020D000FCFFFF3F002103685B1001268A00825845
:1020E000164003D10D22D54B1A70D3E752109342FC
:1020F00000DD130001318C42EFDC5E0001231E4342
:10210000C8E7A3009C46F81A002C17DC1C22002606
:10211000CA4B1A706346FF1AC84B06601B78043717
:10212000002B01D0FFF7C7FA2B68019A1C1213404D
:10213000C34A9B009B580435FFF79FFA00210368B0
:102140005B1001268A008258164003D10D22BB4B3A
:102150001A70DFE75210934200DA130001318C420B
:10216000EFDC5E0001231E43D4E73B000122083B65
:102170001968A40011421DD03B1F1B68134219D0DF
:10218000114113410022994200DA04323B1B1A60CC
:10219000AA4B3F1B1B780437002B01D0FFF78BFAAB
:1021A0002B68019A1C121340A54A9B009B580435CA
:1021B000FFF763FA02203B1F1A684042FFF7A6F8B8
:1021C0003E1B3060E4E73B000120083B1968A40097
:1021D00001421ED03B1F1A6802421AD00141501022
:1021E000CB0FD217884253413A1B9B001360934B8D
:1021F0003F1B1B780437002B01D0FFF75CFA2B68DC
:10220000019A1C1213408E4A9B009B580435FFF71D
:1022100034FA01203B1F1A684042FFF777F83E1B53
:102220003060E4E73B00083B18683B1F1968A600D4
:10223000BE1B0423814202D0042802D8002333604D
:1022400016E001231842F9D10F2302681A40042A2C
:10225000F4D1033A1142F1D10429EFD90A681340AD
:10226000042BEBD1FFF722F9431E98418000306028
:10227000724BA4001B783F1B0437002B01D0FFF7E3
:102280001AFA2B68019A1C1213406D4A9B009B5846
:102290000435FFF7F2F93B00083B18683B1F19684B
:1022A000A600BE1B0023814202D0042802D80423CA
:1022B000336016E001231842F9D10F2302681A4057
:1022C000042AF4D1033A1142F1D10429EFD90A6862
:1022D0001340042BEBD1FFF7E9F84342584180004B
:1022E0003060564BA4001B783F1B0437002B01D0F5
:1022F000FFF7E1F92B68019A1C121340504A9B002A
:102300009B580435FFF7B9F93B000122083B1968D7
:10231000A40011421ED03B1F1B6813421AD05B1051
:102320004A10D80FC9179A4241413B1B89001960D6
:10233000424B3F1B1B780437002B01D0FFF7BBF942
:102340002B68019A1C1213403D4A9B009B58043590
:10235000FFF793F93B1F1A680120FEF7D7FF3E1BDA
:102360003060E5E73B000122083B1968A4001142F8
:102370001DD03B1F1B68134219D01141134100228D
:10238000994200DD04323B1B1A602C4B3F1B1B782B
:102390000437002B01D0FFF78EF92B68019A1C122D
:1023A0001340274A9B009B580435FFF766F93B1FF3
:1023B0001A680220FEF7AAFF3E1B3060E5E73B1FCC
:1023C0001B68A400043B5A1E93413A1B17009B0054
:1023D00013601A4B04371B78002B01D0FFF76BF901
:1023E0002B68019A1C121340154A9B009B58043518
:1023F000FFF743F93B00083B1868FFF737F83B1F2E
:1024000006001868FFF732F80121A4003B1B1F00EB
:10241000321852000A431A60084B04371B78002B0D
:1024200001D0FFF748F92B68019A1C121340044AA7
:102430009B009B580435FFF720F9C046B0020020EE
:10244000C8D700003B00083B1868FFF70FF83B1F98
:1024500006001868FFF70AF80121A4003B1B1F00C3
:10246000321A52000A431A60E44B04371B78002BDF
:1024700001D0FFF720F92B68019A1C121340E04AA3
:102480009B009B580435FFF7F8F83B00083B1868A1
:10249000FEF7ECFF3B1F06001868FEF7E7FF02009F
:1024A0000121A4003B1B1F00724352000A431A6023
:1024B000D24B04371B78002B01D0FFF7FCF82B68B8
:1024C000019A1C121340CE4A9B009B580435FFF71B
:1024D000D4F83B1F1868FEF7C9FF061E17D11F234B
:1024E000C64A1370A4003B1B1F001E60C34B043779
:1024F0001B78002B01D0FFF7DEF82B68019A1C1225
:102500001340BF4A9B009B580435FFF7B6F83B00C9
:10251000083B1868FEF7AAFF310007F00BFC012307
:1025200046001E43DEE73B1F1868FEF79FFF061EAE
:1025300017D11F23B14A1370A4003B1B1F001E605C
:10254000AE4B04371B78002B01D0FFF7B4F82B6893
:10255000019A1C121340AA4A9B009B580435FFF7AE
:102560008CF83B00083B1868FEF780FF310007F04D
:10257000C7FC01234E001E43DEE73B1F1868FEF731
:1025800075FFC11743184B400121A4003A1B1700E7
:102590005B000B431360994B04371B78002B01D071
:1025A000FFF789F82B68019A1C121340944A9B008C
:1025B0009B580435FFF761F8A300FE1A3068012C20
:1025C00025D1FEF753FF01230790049309F0D6FFAE
:1025D0000799002900DC012107F092FC049BA4006C
:1025E000C918012349001943844B3F1B1B783160F4
:1025F0000437002B01D0FFF75EF82B68019A1C12FC
:1026000013407F4A9B009B580435FFF736F8FEF7CE
:102610002DFF04907068FEF729FF049B0130C31A58
:102620000793D3E7A300FE1A31002000049301F0C2
:1026300023FE049B3060FF1A704B04371B78002B7D
:1026400001D0FFF738F82B68019A1C1213406C4A2E
:102650009B009B580435FFF710F83B00083B1868B7
:10266000FEF704FF3B1F06001868FEF7FFFE02009E
:102670000121A4003B1B1F00324052000A431A6094
:102680005E4B04371B78002B01D0FFF714F82B6842
:10269000019A1C1213405A4A9B009B580435FEF7BE
:1026A000ECFF3B00083B1868FEF7E0FE06003B1F0E
:1026B0001868FEF7DBFE32000121A4003B1B1F005F
:1026C000024352000A431A604C4B04371B78002B1C
:1026D00001D0FEF7F0FF2B68019A1C121340484A04
:1026E0009B009B580435FEF7C8FF3B00083B186869
:1026F000FEF7BCFE06003B1F1868FEF7B7FE32006F
:102700000121A4003B1B1F00424052000A431A60F3
:102710003A4B04371B78002B01D0FEF7CCFF2B6817
:10272000019A1C121340364A9B009B580435FEF751
:10273000A4FF3B1F1868FEF799FEC3430121A400C4
:102740003A1B17005B000B4313602C4B04371B78BC
:10275000002B01D0FEF7AFFF2B68019A1C1213402B
:10276000274A9B009B580435FEF787FF3B00083B38
:102770001868FEF77BFE06003B1F1868FEF776FE22
:10278000320082400121A4003B1B1F0052000A437B
:102790001A601A4B04371B78002B01D0FEF78BFF11
:1027A0002B68019A1C121340154A9B009B58043554
:1027B000FEF763FF3B00083B1868FEF757FE060074
:1027C0003B1F1868FEF752FE320002410121A400AF
:1027D0003B1B1F0052000A431A60084B04371B784A
:1027E000002B01D0FEF767FF2B68019A1C121340E3
:1027F000034A9B009B580435FEF73FFFB0020020C0
:10280000C8D700003B000C3B1868FEF72FFE3B00CA
:10281000083B06001868FEF729FEF1170200C317EF
:10282000300007F0BFFB3B1F049005911868FEF7CE
:102830001DFE02000498059907F068FB0123A4001F
:102840003E1B370040001843E54B30601B780437CF
:10285000002B01D0FEF72FFF2B68019A1C121340AA
:10286000E04A9B009B580435FEF707FFA300FE1AC1
:10287000310020000493FEF78DFB049B3060FF1AAB
:10288000D74B04371B78002B01D0FEF714FF2B68C1
:10289000019A1C121340D34A9B009B580435FEF743
:1028A000ECFEA300FF1A39002000FEF78BFBCC4B97
:1028B0001B78002B01D0FEF7FEFE2B68019A1C123C
:1028C0001340C84A9B009B580435FEF7D6FEA30070
:1028D000FE1A310020000493FEF7B4FB049B306025
:1028E000FF1ABF4B04371B78002B01D0FEF7E3FE25
:1028F0002B68019A1C121340BA4A9B009B5804355E
:10290000FEF7BBFEA300FF1A39002000FEF71EFCF5
:10291000B34B1B78002B01D0FEF7CDFE2B68019A3C
:102920001C121340AF4A9B009B580435FEF7A5FECE
:10293000A300FE1A310020000493FEF779FC049BEB
:102940003060FF1AA64B04371B78002B01D0FEF72E
:10295000B2FE2B68019A1C121340A24A9B009B589E
:102960000435FEF78AFE3B1F186801F0DFF83A00D5
:102970000121083A12680300A4000A4229D1042A5E
:102980000CD910680F221040013808280FD807F022
:102990003DF9052026220E0E0E0E24009249180045
:1029A00009F08CFE434258413B1B800018608C4B61
:1029B0003F1B1B780437002B01D0FEF77CFE2B68F1
:1029C000019A1C121340874A9B009B580435FEF75E
:1029D00054FE8649E3E78649E1E78649DFE7864911
:1029E000DDE7069B3E1DF31A7D4CD82B03DD1A2331
:1029F0002370FEF760FE00F0DFFD01223B00400087
:102A00001043186023783700002B01D0FEF753FEE7
:102A10002B68019A1C121340724A9B009B58043584
:102A2000FEF72BFE069B3E1DF31A6D4CD82B03DDE3
:102A30001A232370FEF73FFE00F0B4FD6F4A4000FA
:102A4000104001223B001043186023783700002B10
:102A500001D0FEF730FE2B68019A1C121340614A28
:102A60009B009B580435FEF708FE069A3B1D9B1AF7
:102A70005B4CD82B03DD1A232370FEF71CFE00F0FD
:102A80009BFD5F4B1A68831A904201D25D4A9B18E6
:102A900001213A005B000B43136023780437002BBD
:102AA00001D0FEF708FE2B68019A1C1213404D4A14
:102AB0009B009B580435FEF7E0FD00F07DFD504B78
:102AC000A4001860464B3F1B1B78002B01D0FEF77B
:102AD000F2FD2B68019A1C121340424A9B009B583E
:102AE0000435FEF7CAFD00F075FDA300002810D1E3
:102AF000FF1A3B4B1B78002B01D0FEF7DCFD2B6847
:102B0000019A1C121340374A9B009B580435FEF76C
:102B1000B4FD3E00FF1A012320001A003900FEF721
:102B2000F3FC394C2068643003F05AF8002803D1D4
:102B3000043D3700FEF7D2FD029B21685A783348E6
:102B400003F069FC0123029A137000F02BFD304B57
:102B500022681B68063253431818FFF7F5F800F097
:102B600039FDA300002810D1FF1A1D4B1B78002B44
:102B700001D0FEF7A0FD2B68019A1C121340194AE0
:102B80009B009B580435FEF778FD3E00FF1A20009D
:102B9000012300223900FEF7B7FC1B4C206864308B
:102BA00003F01EF80028C3D0184803F0C5F9C9E7A0
:102BB000A4003E1BFEF728FD3700094B30601B7850
:102BC0000437002B01D0FEF776FD2B68019A1C120A
:102BD0001340044A9B009B580435FEF74EFDC04647
:102BE000B0020020C8D7000004DA00000CDA0000B0
:102BF00013DA00001ADA00001FDA0000FEFFFF7F80
:102C0000DC05002037894100D4050020B1020020F6
:102C100004000020FB4BA4001B783F1B002B01D0BD
:102C2000FEF749FD2B68019A1C121340F64A9B00DF
:102C30009B580435FEF721FDA4003E1B300000F038
:102C4000F6FC3700EF4B30601B780437002B01D0C7
:102C5000FEF731FD2B68019A1C121340EA4A9B00D3
:102C60009B580435FEF709FDA4003E1B300000F020
:102C7000E0FC3700E34B30601B780437002B01D0B9
:102C8000FEF719FD2B68019A1C121340DE4A9B00C7
:102C90009B580435FEF7F1FCA300FE1A310020001A
:102CA000049300F0C9FC049B3060FF1AD54B043735
:102CB0001B78002B01D0FEF7FEFC2B68019A1C123A
:102CC0001340D14A9B009B580435FEF7D6FCA40064
:102CD0003F1B380000F0E2FCCA4B1B78002B01D0F0
:102CE000FEF7E9FC2B68019A1C121340C64A9B00B0
:102CF0009B580435FEF7C1FCA300FE1A31002000EA
:102D0000049300F0F3FC049B3060FF1ABD4B0437C2
:102D10001B78002B01D0FEF7CEFC2B68019A1C1209
:102D20001340B94A9B009B580435FEF7A6FCA4004B
:102D30003F1B380000F01CFDB24B1B78002B01D06C
:102D4000FEF7B9FC2B68019A1C121340AE4A9B0097
:102D50009B580435FEF791FC0121200000F0F0FCA7
:102D6000A84B1B78002B01D0FEF7A5FC2B68019A1D
:102D70001C121340A44A9B009B580435FEF77DFCAF
:102D80000021200000F0DCFC9E4B1B78002B01D0C2
:102D9000FEF791FC2B68019A1C1213409A4A9B0083
:102DA0009B580435FEF769FCA4003E1B300000F080
:102DB00001FD3700934B30601B780437002B01D0A6
:102DC000FEF779FC2B68019A1C1213408E4A9B0077
:102DD0009B580435FEF751FCA4003E1B300000F068
:102DE000FDFC3700874B30601B780437002B01D087
:102DF000FEF761FC2B68019A1C121340824A9B006B
:102E00009B580435FEF739FCA4003F1B380000F046
:102E1000BFFC7C4B1B78002B01D0FEF74CFC2B68D1
:102E2000019A1C121340784A9B009B580435FEF708
:102E300024FCA4003F1B380003F0F8FE714B1B7804
:102E4000002B01D0FEF737FC2B68019A1C121340AF
:102E50006D4A9B009B580435FEF70FFCA4003E1BF7
:102E6000300003F09DFF3700664B30601B7804375D
:102E7000002B01D0FEF71FFC2B68019A1C12134097
:102E8000614A9B009B580435FEF7F7FBA4003F1BEB
:102E9000380003F065FE5B4B1B78002B01D0FEF77A
:102EA0000AFC2B68019A1C121340574A9B009B583E
:102EB0000435FEF7E2FBA4003E1B300003F06AFE7F
:102EC0003700504B30601B780437002B01D0FEF7E1
:102ED000F2FB2B68019A1C1213404B4A9B009B5833
:102EE0000435FEF7CAFBA300FF1A3900200001F0E9
:102EF00025FD444B1B78002B01D0FEF7DCFB2B6833
:102F0000019A1C121340404A9B009B580435FEF75F
:102F1000B4FBA300FF1A3900200001F023FB394B5A
:102F20001B78002B01D0FEF7C6FB2B68019A1C1200
:102F30001340354A9B009B580435FEF79EFBA300C7
:102F4000FF1A3900200001F031FC2E4B1B78002BBA
:102F500001D0FEF7B0FB2B68019A1C1213402A4ADD
:102F60009B009B580435FEF788FBA300FF1A39002D
:102F7000200001F043FC234B1B78002B01D0FEF70F
:102F80009AFB2B68019A1C1213401F4A9B009B5806
:102F90000435FEF772FBA300FE1A310020000493F3
:102FA00003F0E8FF049B3060FF1A164B04371B78D0
:102FB000002B01D0FEF77FFB2B68019A1C121340F7
:102FC000114A9B009B580435FEF757FBA300FE1ADD
:102FD00031002000049303F0D5FF049B3060FF1AFA
:102FE000084B04371B78002B01D0FEF764FB2B68DD
:102FF000019A1C121340044A9B009B580435FEF7AB
:103000003CFBC046B0020020C8D70000A300FE1A57
:1030100031002000049303F0BDFF049B3060FF1AD1
:10302000984B04371B78002B01D0FEF744FB2B682C
:10303000019A1C121340944A9B009B580435FEF7DA
:103040001CFBA300FE1A31002000049303F058FC7F
:10305000049B3060FF1A8B4B04371B78002B01D088
:10306000FEF729FB2B68019A1C121340864A9B002D
:103070009B580435FEF701FBA300FF1A390020001E
:1030800001F0A8FA7F4B1B78002B01D0FEF713FB51
:103090002B68019A1C1213407B4A9B009B580435F5
:1030A000FEF7EBFAA300FF1A3900200001F0CEFB77
:1030B000744B1B78002B01D0FEF7FDFA2B68019AA8
:1030C0001C121340704A9B009B580435FEF7D5FA3A
:1030D000A300FE1A31002000049301F033FB049B8F
:1030E0003060FF1A674B04371B78002B01D0FEF7C6
:1030F000E2FA2B68019A1C121340634A9B009B580A
:103100000435FEF7BAFAA300FF1A3900200001F0D7
:10311000E1FA5C4B1B78002B01D0FEF7CCFA2B6850
:10312000019A1C121340584A9B009B580435FEF725
:10313000A4FA002C55DD3B1F1E68012C0CD1264241
:1031400007D1042E05D90F23326830001340042B19
:1031500011D00120404212E0022CFAD13B00083B82
:10316000186801231842F4D10428F2D902680E33FA
:103170001340042BEDD100F0D9FCFEF71FF9A3009A
:10318000FF1A00282DDB0022022C11D1012333402D
:10319000934222D1042E20D931680F320A40092AE5
:1031A0001BD172685210D2B29100994210D17F188F
:1031B0000002104304003A00069B0C32D31AD82BAD
:1031C00001DCFEF7AFFC1A222E4B1A70FEF773FAE1
:1031D000F418A468FC500433E7E73E60012204378A
:1031E000E6E700233B60274B3A1D1B78002B02D0FB
:1031F0001700FEF760FA2B6801991C120B40224958
:103200009B005B5817000435FEF737FA069B029ABD
:10321000FB1A9B101361A300FF1A3900200002F073
:10322000C9FE184B1B78002B01D0FEF744FA2B681F
:10323000019A1C121340144A9B009B580435FEF758
:103240001CFA069B029AFB1A9B101361A300FE1A3C
:1032500031002000049302F0ADFE049B3060FF1AA1
:10326000084B04371B78002B01D0FEF724FA2B689B
:10327000019A1C121340044A9B009B580435FEF728
:10328000FCF9C046B0020020C8D700000023F7B503
:103290005A1E0192002B07DA01F066FB02F0A2FF32
:1032A00003F018F91923019300263000194B19680F
:1032B000B14212DD184B1A6801328A420FDAF0244B
:1032C0001A601D68154F6C43E35D002B1FD0E41995
:1032D000022B06D12000FEF7AFF9019BD8E70022B0
:1032E000EDE7012B0DD1002801D100F05BF9F022B0
:1032F0006A43BB185B680A49C31A8B4201D8022390
:10330000BB54F0235D43054BEB5C022BE2D001364E
:10331000CCE7C046D805002000000020481C002053
:103320003F420F0080220B4B52001A600121A8225D
:10333000A920094BD20019649A58C00005321A50CE
:1033400006481A50C122C020920000039850044B36
:103350001970704700E100E0008000404C0500005B
:103360000306002004207047F8B550C9012322004D
:103370001A40101E2DD03340181E2AD06410002091
:103380001C2C26D81D4B761035009E4200DD1D00FA
:103390001B4F3B5D012B05D00121200005F026F8D5
:1033A00001233B55174B1B78002B01D1FFF7BAFFC8
:1033B0000023154A9E420DDCFF2514491448D65CB3
:1033C000B44202D15E007052D5540133042BF6D1C1
:1033D0000420F8BDD15C8C4203D10C4A5B009D52A5
:1033E000F6E70133042BF5D10023D15CFF2901D18D
:1033F000D454F2E70133042BF7D1E9E78813000036
:10340000E4050020030600201C0000200E00002020
:10341000DC05000070B530C9012322001A40101EDF
:103420001BD02B40181E18D064101C2C00D900246F
:10343000154E335D012B05D00121200004F0D6FF8D
:103440000123335569100800104A1038104B904280
:1034500004D9012252421A60042070BD1C600D483C
:1034600006F068FC0C4B040018800C4B1B78002BFA
:1034700001D1FFF757FF0122094B9A64A922D2001C
:10348000995864189C50E7E7E405002090860100F5
:103490001800002020A107000C00002003060020D7
:1034A00000800040F8B501260D683400B04200DD10
:1034B0004C682B003340181E0BD023003340181EDD
:1034C00007D06D10002D05DCA12300201E4ADB0073
:1034D000D650F8BD641000201C2CFAD81B4F3B5D61
:1034E000012B04D00121200004F080FF3E5529006B
:1034F000174806F01FFC0A21053006F01BFC154B8F
:10350000A400E258144B12021343A2221349D20022
:103510008B50134C0C4B9C50124C195101241249E6
:103520005C50124B196900219950114A904200DDFC
:103530001000A8228021D2009850012289005A5000
:1035400004201A60C5E7C04600F00140E4050020F1
:1035500000B4C404C8EA0000030003000060004097
:1035600040A10040140500000405000000A0004038
:10357000FFFF0000030010B50120002B02DC1B3010
:10358000FEF73CF810BD0420704710B5002803DC9E
:103590001C20FEF733F810BD0B680020DB07FAD4BF
:1035A0000D30F6E70122034B1A64A822D200985886
:1035B0007047C046008000400122054B10B51A64D8
:1035C000A822FA21D2009858890006F029FB10BDE4
:1035D00000800040012070470048704784DA0000F6
:1035E0001D20704770B5054E0400335C0D008B4202
:1035F00002D004F0FBFE355570BDC046E405002046
:1036000070B50024084D635D012B09D10021200015
:1036100004F00AFF0021200004F0E8FE00236355B7
:1036200001341D2CEED170BDE405002070470D2043
:1036300070473B2070470000F8B501240B68060076
:103640000D00234204D10D20FDF7D8FF2000F8BD66
:103650005B102000052BFAD80E4A9B009C580E4F99
:103660003B5D002B05D00021200004F0BFFE0023AD
:103670003B55012E06DD6B68042B03D1022120008F
:1036800004F0B4FE200004F05FFD0124400020435C
:10369000DDE7C0466CDA0000E4050020F8B501263D
:1036A0000568354202D04468344203D10D20FDF74D
:1036B000A5FFF8BD6D101C2DFBD80A4F7B5D012BBB
:1036C00004D03100280004F091FE7E5506496410B4
:1036D0008C4202DCE143C9172140280004F0BAFD06
:1036E000E7E7C046E4050020FF03000070B50124B1
:1036F0000D68254204D10D20FDF780FF200070BD2C
:103700006D101C2D17D80024012804DD4C68043CE2
:1037100063425C416400094E735DA34204D0210002
:10372000280004F063FE7455280004F093FE0300A3
:103730000420012BE3D00020E1E7C046E40500208F
:1037400070B504000D001C280ED8084E335C012B08
:1037500004D0012104F04AFE012333552900200042
:103760004D1EA94104F060FE70BDC046E405002076
:10377000036810B5DA0703D40D20FDF73FFF10BD35
:103780004168581004394A425141FFF7D9FFF6E722
:1037900037B569460A00064B30CB30C203680220B9
:1037A000042B02D101F002F837BD01F027F8FBE746
:1037B0002CDA000010B5084C6379002B05D00021ED
:1037C000052004F013FE00236371052004F042FE7F
:1037D00043425841800010BDE405002010B5084C5C
:1037E000E37A002B05D000210B2004F0FFFD00231D
:1037F000E3720B2004F02EFE43425841800010BDBE
:10380000E4050020A02200230349D2008B50034985
:1038100010328B507047C04600F0014000600040FD
:10382000F7B52F4D2F4EEB6C002B14D0A92400239D
:10383000E4003759EB642C4B186800280BDB2B4B4A
:1038400019784A425141C9B2197004F0EDFD284B74
:103850001B88DF1937512B6D002B38D00021254BE9
:10386000254FF45829653A780193244D8A4206D0B1
:103870002B68032B03D8224AD05C04F0D5FD2B68BB
:10388000204A0133134004D50422013B5242134322
:1038900001331B4900228C462B60042B18D0604654
:1038A000C05C591CFF2802D10B000122F5E7002A59
:1038B00000D02B60012104F0B7FD01233B702B6881
:1038C000114A5B009B5A0C34E418019BF450F7BD7D
:1038D00001235B422B6000233B700C4BF4E7C04696
:1038E000FC800040008000401800002002060020FC
:1038F0000C0000204C05000001060020E00500201F
:103900001C000020030000800E0000205C46000028
:10391000084B094AFF201A805A809A80DA800023D7
:10392000064A07491370074A087048708870C870C3
:10393000136070470E000020DC0500000106002027
:103940001C000020E00500200122024B52421A60B8
:103950007047C0461800002010B5034A07210348ED
:1039600002F0CEF810BDC04634DA000036E20000A6
:10397000E12170B54902194804F05CF900240122E4
:103980000320174B17491A615C50043158508018B6
:10399000083158501A60063004F0D0FBFF21124A5B
:1039A000A15401341D2CFBD1012200200F4B01003A
:1039B0001A6004230E4A0F4D1468002CFCD02C68AA
:1039C0000002013B20431160002BF5D101220A4B7C
:1039D0001A6004F0EBFA01F013F970BDD01B00205F
:1039E0000080004004050000E405002000D00040F5
:1039F00000D1004008D5004004D00040F8B50B4E7F
:103A0000070030000D0004F05DF90400A84200DD5D
:103A10002C003D00EB1B9C4205DD300004F05CF9FE
:103A200028700135F6E72000F8BDC046D01B002005
:103A300010B50100014804F005F910BDD01B0020AD
:103A400010B5054C200004F00BF9E12120004902DB
:103A500004F0F0F810BDC046D01B0020C3070CD402
:103A6000064B1B68834208D8054B1B68984204D854
:103A7000031F1B68002B00D0180070470C060020A5
:103A8000080600200023012210B50A4899000133DE
:103A90004250642BFAD1084C084B00211A602000D8
:103AA000074A08F08BFA074B074A6360074B1A6016
:103AB00010BDC046A02D00201006002008000020E8
:103AC000D40900003027000014060020040600205E
:103AD00010B5044B044A1A60044B054A1A60FFF7FC
:103AE000D1FF10BD0C0600201006002008060020A3
:103AF000E40F0020044B1B681868000980B20238EC
:103B0000C343DB17184070470406002000B59BB084
:103B10000200054901A808F095FD01A802F028FA65
:103B200002F0D8FCFCE7C04613DB00000B4BC207D9
:103B300004D4042804D80A4B00D00A4B180070475C
:103B40000F2203681A40031D042AF7D0064B092AE6
:103B5000F4D0064B032AF1D0054BEFE7EDDA000075
:103B60006ED6000068D60000F7DA000007DB000020
:103B7000FEDA00000020064A0649131F1860136889
:103B80001B099BB202339B00D2188A42F5D37047BF
:103B900014060020E40F0020F7B50F240126314B56
:103BA000314A1968314B324D186813681F0027409D
:103BB000072F26D813681B099BB202339B00D2182B
:103BC000AA42F2D300242B4EA500AD192868FFF7B6
:103BD00045FF01342860642CF6D1274C2068FFF79C
:103BE0003DFF2060254C2068002802D0FFF736FFFB
:103BF00020600025224B1B680093009B9D4214DB34
:103C0000F7BD1B099BB29B00D3189A42D2D01F6804
:103C1000374208D1B94206D2B84204D3043F3F68C4
:103C2000002F00D01F60043BEFE7F0236B43154AE1
:103C30009B181A78002A01D10135DEE71F693C2361
:103C400000266B43DB199B0001930136BB1BF3D4A9
:103C5000019BB4001C1B0B4B1C19A069FFF7FEFE57
:103C6000A061F2E70C0600201406002008060020E0
:103C7000E40F0020A02D002008000020E40F002009
:103C8000D8050020481C0020F7B50124204246D169
:103C9000234B1B689C46984241D3224B1B680193DF
:103CA00098423CD8031F1B68002B38D102000368E0
:103CB00000941B099BB2002B0FD10099131F1960B0
:103CC00090422CD015682B1F1B68990069180C684E
:103CD000013B14600A602A00EDE79D005519296830
:103CE000009C214219D18C4517D8019C8C4214D3D9
:103CF0000E1F3468002C10D10F680F343C40072C85
:103D000008D92F60151F2B600B680A601B099BB236
:103D10000A00D0E700993160CDE7013BCBE7F7BD62
:103D20000C060020080600200D4970B50A000D4D54
:103D30001368141F1B0926689BB2981C002E0BD019
:103D400000238A4200D00B0023608300C918800042
:103D50001218AA42ECD370BD1B011360F7E7C046EE
:103D600014060020E40F0020F8B5124C27000F22A3
:103D70003B681D09ADB213420DD06E1CB600A742C0
:103D800004D032003900200008F005F90022A31900
:103D90000436A4191A600235AD00074B7F199F4203
:103DA000E5D31B1B9B10013B1B012360034B1C60D5
:103DB000F8BDC04614060020E40F002004060020D1
:103DC000F0B59BB0FFF7EEFB00240700214AA300EB
:103DD000D0580134FFF758FF642CF7D11E4B1868F8
:103DE000FFF752FF1D4B1868002801D0FFF74CFF6A
:103DF00000261B4B1B689E4217DBFFF795FFFFF762
:103E0000CBFEFFF7B1FFFFF7CDFB164BC21B1B68C4
:103E100015491B6801A81B099BB2023B08F012FC64
:103E200001A802F0A5F81BB0F0BDF02575430F4BBB
:103E3000ED182B78002B01D10136DAE72B695C1ED7
:103E4000002CF9DBA300EB189869FFF71DFF013C7C
:103E5000F6E7C046A02D002008000020E40F002057
:103E6000D805002004060020CDDA0000481C002000
:103E7000F7B5174D4F1C2B6806001B680C001B097B
:103E80009BB201929F420BDBFFF79AFF2B681B68E6
:103E90001B099BB29F4203DB0A20FDF7AFFBFEBD6F
:103EA0002868A71CBA00DB1B81181B010B60296066
:103EB0000021031F19600F231E4003002401264325
:103EC00040C3083A9A189A42E9D9019902C3FAE71D
:103ED00004060020F7B503000122134004000D0082
:103EE0000193002B2BD1174B1B68834227D8164B0D
:103EF0001B68834223D90F23144F38600068184091
:103F0000FFF7B6FF019B3C68061E3B6017D0236895
:103F100004301B099BB29D4200DD1D00AA00211D3B
:103F2000251F08F02FF8FFF725FE2E60FFF734FE5F
:103F300000232B602268064B1340236034002000CE
:103F4000FEBDC0460C06002008060020E40F00203D
:103F5000F0FF0F000323043010B5C11719400918F2
:103F6000891000220420FFF783FF10BD70B5050003
:103F700008000C00FFF7EEFF0023002804D170BDFD
:103F8000E95CC21811710133A342F9DBE343DB178B
:103F90001C40002304192371F1E7F0B50C009BB01D
:103FA000022804DC1C20FDF729FB1BB0F0BD012317
:103FB0000868184206D1042804D90F260168314048
:103FC000042901D00E20EEE761680D001D40F9D1F3
:103FD0000429F7D90A683240042AF3D1A2681A42A8
:103FE00001D10D20DFE7FFF7A1FD06006068FFF7B4
:103FF0009DFDA768010001AC7F103000257003F023
:1040000043FA39006423220003F0A3FA200008F0E9
:104010005FFB01002000FFF7A9FFC6E710B51C4CAD
:10402000A544041E02D1FFF795FF0BE003F044F90D
:104030000138062828D805F0E9FD090911182904D6
:10404000240000208023DB009D4410BD200003F0ED
:10405000AFF9011B2000FFF789FFF3E7200003F011
:1040600055F9430001201843ECE780226946D2004D
:10407000200003F062F9684608F02AFB0100684658
:10408000E9E704210348E6E70020CCE70420D9E76C
:1040900000FCFFFF5CDB000070B50C00022803DCB5
:1040A0001C20FDF7ABFA70BD01230868184206D149
:1040B000042804D90F2501682940042901D00E20C5
:1040C000EFE761681942FAD10429F8D90A682A4051
:1040D000042AF4D1A2681A4201D10D20E1E7FFF7CA
:1040E00025FD05006068FFF721FDA468010064104C
:1040F000280003F0C9F9210003F006FAFFF78EFF4C
:10410000D1E770B50D00012803DC1C20FDF776FA1D
:1041100070BD01240868204206D1042804D90F216B
:1041200002680A40042A01D00E20EFE76A682242A2
:10413000FAD1042AF8D913680B40042BF4D1FFF705
:10414000F5FC06006868FFF7F1FC0100300003F0A1
:104150009BF903F01DFA40002043D9E7F8B50700AA
:104160000C001C20012F0BDD01250868284206D118
:10417000042804D90F2102680A40042A03D00E2023
:10418000FDF73CFAF8BD62682A42F8D1042AF6D954
:1041900013680B40042BF2D1FFF7C8FC06006068DF
:1041A000FFF7C4FC0100022F14D0A4682C4211D0E8
:1041B0006410300003F068F9050003F07DF8012871
:1041C00011D1002C02DD0135012C06D12800FFF7AA
:1041D00025FFD7E701246442EBE7280003F0F5F858
:1041E000013C0500F0E70228F0D1002CEEDD01359E
:1041F000012CEBD000222800110003F018F903F085
:10420000E4F8013C0500F3E710B501240868044018
:1042100016D04410200006F021F8154905F0ECFEF8
:1042200007F0D2FD04F024FA0022124B06F086FFBC
:1042300004F0C6F907F058FD43000120184310BDF3
:10424000042810D90F2302681340042B07D1FFF76D
:104250006DFC21000A2208F003FB0400DAE7032BBF
:1042600001D10430F5E70D20FDF7C8F9D2E7C046CB
:10427000D30237390000D040086870B5012405002A
:10428000254006D1042804D90F2302681340042BCB
:1042900003D00E20FDF7B2F970BDFFF747FC03789D
:1042A0002900233B5A4253411022C01808F0D8FA83
:1042B00080239B05C218044B9A4201D91420E9E7D8
:1042C00040002043E8E7C046FFFFFF3F10B5034A28
:1042D0000621034801F014FC10BDC0462CDB000091
:1042E00024DB00000020704710B51E20FDF786F982
:1042F00010BD10B51E20FDF781F910BD10B51E20B0
:10430000FDF77CF910BD10B51E20FDF777F910BD43
:1043100010B51E20FDF772F910BD10B51E20FDF777
:104320006DF910BD10B51E20FDF768F910BD10B570
:104330001E20FDF763F910BD10B51E20FDF75EF9D4
:1043400010BD10B51E20FDF759F910BD10B51E2087
:10435000FDF754F910BD10B51E20FDF74FF910BD43
:1043600010B51E20FDF74AF910BD10B51E20FDF74F
:1043700045F910BD10B51E20FDF740F910BD10B570
:104380001E20FDF73BF910BD10B5034A112103486B
:1043900001F0B6FB10BDC04698DB000020DC000039
:1043A0000120034B1860034B1B6883401843704780
:1043B00008100020E80F0020F0B5EFF31081012372
:1043C000194083F31088134C134AA4461268134E05
:1043D000013A9340124F134A002B17D0146803423E
:1043E0000FD03D682C60C046C046C046C046C0469F
:1043F000C046C046C0460C4C1568246825605B0862
:10440000EAE765462C6014683460F8E781F31088A9
:10441000F0BDC04608050050200000200C050050EB
:10442000F40F0020FC0F0020F00F002030B585B005
:1044300001AD0C220649280007F0A4FD0024285DE8
:1044400001210134FFF7CEF80C2CF8D105B030BDB6
:1044500009DD0000F7B56A463B4B01AE13800A2325
:1044600093703A4B33801C23B370FFF79BF8384BA3
:10447000384DC0182B68984201D200232B602C685D
:10448000002C41D1375D01213800FFF7ABF8013432
:104490000021380003F0C8FF032CF3D100240127CA
:1044A0006B461E5D39003000FFF79CF8013439007F
:1044B000300003F0B9FF032CF2D1C8200138C04608
:1044C000C046C046C046C046C046C046C046C046BC
:1044D000C046C046C046F1D16B4600211878FFF7B0
:1044E00081F86B4600215878FFF77CF86B46002175
:1044F0009878FFF777F8FFF755F8FA2300241B01A7
:10450000C01828602000FEBDFFF74CF82B6800247F
:104510009842F7D3032003F017FE0600042003F0AF
:1045200013FE36180A2003F00FFE0B4B9B1B181AC4
:104530000A4BA04206DB18600023094A2B60136077
:104540000124DFE71C60F7E7030400001A1B0000EA
:104550001027000000100020E3030000E80F0020F7
:10456000081000200022054B10B51A60044B1B6890
:10457000934201D002F040FE002010BD0410002044
:10458000F41A002010B5041E10DA00240A4BA4000F
:10459000E25801239340094A09491360094A11600E
:1045A000094A0A4911600A4A136010BDFFF718F85A
:1045B000A042EADDEAE7C046C8EA0000FC0F00209E
:1045C00008050050F40F0020F00F00200C050050EB
:1045D00018050050F0B53B4B85B01B680C00002B54
:1045E00003D101204042FFF7CDFF246801222700BC
:1045F000174028D0FF236012184033496714661013
:1046000040431F401E4005F095FB050438002E492D
:10461000784305F08FFB0002054330002A497043C0
:1046200005F088FB294B28431B68202B06D164002A
:10463000A40E274BA400E35800021843FFF7BCFE6A
:10464000002005B0F0BD042CFAD90F2321680B40DF
:10465000092BF5D1636803925B100193019B9F4284
:10466000EEDABB00E3189E68039B1E4228D0FF23AE
:104670007012184072101A401349751440431D40BF
:10468000009205F057FB030428000F49684302938A
:1046900005F050FB029D0002054300980A49404383
:1046A00005F048FB094B28431B68202B06D17600F8
:1046B000B60E074BB600F55800022843FFF77CFE04
:1046C0000137CBE7FC0F0020590600002000002036
:1046D000F0DE00000200086810B5C3070FD54010D7
:1046E0001823012A03DD4A68042A00D10833054A49
:1046F0001360FEF79BFFFFF745FF002010BD012070
:104700004042EDE72000002010B50124044002D013
:104710004410200010BD042810D90F230268134054
:10472000042B07D1FFF702FA21000A2208F098F8BB
:104730000400EEE7032B01D10430F5E70D20FCF770
:104740005DFFE6E70868F8B5C3071AD5FFF7DCFF99
:104750000300203B5E2B25D80520434301221D1872
:104760000020114E9D4219D005211024F75C3C42D7
:1047700000D080180139520064100029F7D10133AC
:10478000F0E704280ED90F2203681A40042A09D141
:104790001B099BB2002B05D00379DAE70123400007
:1047A0001843F8BD0120FCE715DD000070B508686E
:1047B0000D00FFF7A9FF04006868FFF7A5FF621E60
:1047C0000100042A14D8451E042D11D805236B437B
:1047D0009B18012215009D402B00064805682B43BD
:1047E0000360054B1B68002B02D0200002F005FD82
:1047F000002070BD04100020F41A002070B5086875
:104800000D00FFF781FF04006868FFF77DFF621E5F
:104810000100042A13D8451E042D10D805236B432C
:104820009B1801229A400748036893430360064B94
:104830001B68002B03D00022200002F0DEFC0020C9
:1048400070BDC04604100020F41A0020F0B5050029
:1048500089B008680C00FFF757FF0690022D36DD7F
:104860006068FFF751FF0190A068FFF74DFF04005B
:104870000127231D661E0793731C0293079B9E420C
:1048800035D0052373430593019B019D05330493A4
:10489000049BAB421ED0042E16D86B1E042B13D8DB
:1048A0000122059B2349013B5B199A409446224A09
:1048B0000B681068069A3A4003920DD062461A437C
:1048C0000A60012200280DD17F000135E0E70124B4
:1048D0000194CDE7029ECFE7624693430B60002828
:1048E000F2D0039A0299280002F087FCECE7019BC2
:1048F0001E1D042E1AD8012C18D1002505273B00B7
:1049000021006B439B1999400B000A4A013511683D
:104910009943094B11601B68002B05D0019B0022B5
:10492000581D290002F069FC052DE8D1002009B0CE
:10493000F0BDC04604100020F41A0020086810B52D
:10494000C30703D5FFF7E0FE054B1860054B1B6856
:10495000002B03D0024B186802F050FC002010BD61
:1049600004100020F41A00207FB5A04C2368002B0F
:104970000AD19F4A1268002A06D19E4B1B68002B61
:1049800001D0FFF767FD7FBD9B4D2A68002A26D125
:10499000984A1268002A1BD0FFF75CFD0028F2D06D
:1049A000FFF744FD924B24681A681C60002A16D059
:1049B000002C14D101AD0C229049280007F0E2FA36
:1049C000285D00210134FEF70DFE0C2CF8D1DAE74A
:1049D000874A1268002AE5D1002BE3D0E0E70021E6
:1049E0001A2003F021FD00211B2003F01DFD0021F2
:1049F0001C2003F019FD2E68012E5CD0022E00D180
:104A0000A2E0002E50D101363100794C03202368FA
:104A1000994303F009FD0420216801404B425941AC
:104A200003F002FD102123680A2019404B4259412E
:104A300003F0FAFC80212368090119404B425941D7
:104A4000062003F0F1FC80212368090219404B4243
:104A50005941072003F0E8FC8021236849021940EE
:104A60004B425941092003F0DFFC80212368890271
:104A700019404B425941192003F0D6FC802123688C
:104A8000C90219404B425941182003F0CDFC802344
:104A900021681B0319404B425941172003F0C4FC05
:104AA00031001A2003F0C0FC2B680321581C05F0CC
:104AB00027FA296067E702214D4C17202368194027
:104AC0004B42594103F0B0FC0821236818201940DB
:104AD0004B42594103F0A8FC80212368C9001940CA
:104AE0004B425941042003F09FFC80212368490177
:104AF00019404B4259410A2003F096FC802123685B
:104B0000C90119404B425941032003F08DFC80211B
:104B10002368890319404B425941092003F084FC62
:104B2000802321681B0419404B425941192003F08E
:104B30007BFC3100062003F077FC3100072003F0F6
:104B400073FC31001B20ADE72021294C172023687E
:104B500019404B42594103F067FC4021236818205B
:104B600019404B42594103F05FFC80212368192012
:104B700019404B42594103F057FC802123684900FA
:104B800019404B425941092003F04EFC8021236813
:104B9000890019404B425941072003F045FC802110
:104BA0002368890119404B425941062003F03CFC1F
:104BB00080212368490319404B4259410A2003F0E0
:104BC00033FC80212368C90319404B42594103201B
:104BD00003F02AFC802321685B0419404B425941B1
:104BE000042003F021FC01211C205BE704100020BD
:104BF000F80F002008100020EC0F002009DD000055
:104C0000012010B54042FFF7BDFC10BD10B5034AAE
:104C10000921034800F074FF10BDC046F0DF00001A
:104C200038E000008023F0B502255B051A690A4CC4
:104C30000A4BA1261D5103278025F600ED00BA433B
:104C4000884202D300221A51F0BD5F59002FFCD0D8
:104C500098518018F4E7C0460405000000E00140C8
:104C600010B5002806D1C020B02140028902FFF70C
:104C7000D9FF10BDB02080218002C902F7E70000F3
:104C800043425841064B40421840B0239B02C01893
:104C9000036800201A0E532A01D11B02180A70471C
:104CA00000C0FEFF30B501248025054B054AED000C
:104CB0009C505C59002CFCD001600021995030BD03
:104CC00000E001400405000043425841074B4042C8
:104CD0001840B0239B02C018A62310B50902DB05BB
:104CE000090A1943FFF7DEFF10BDC04600C0FEFFF2
:104CF000F0B5012480260D4B0D4DF6005C510029C6
:104D000002DC00225A51F0BD577814783F02274345
:104D1000947824042743D478043224063C439F59D2
:104D2000002FFCD010C00139E9E7C04600E0014087
:104D30000405000070B505004B680A009C1C2100AA
:104D4000A400FFF7D5FF281970BD0000134B1B68A6
:104D5000002B0CD08022B023D2029B0200280BD162
:104D60001A1D5B681B0E522B00D110007047B02239
:104D7000C02392025B02F1E782420DD903681B0E49
:104D8000522B09D1436802339B00C018824203D9D9
:104D900003681B0E522BE9D00020E7E70C1100201E
:104DA000F0B50020B7B00024FFF7D0FF27000500C2
:104DB0002600002D2ED1284D2868FFF761FF320014
:104DC0003B0001900094254904A807F03BFC04A88F
:104DD00001F0CEF8224B64201C682B68A0215A42B7
:104DE0005341204A5B421340B02292029B18E41ABE
:104DF0006043490204F09EFFA02252020300009289
:104E00001949220004A807F01DFC04A801F0B0F81D
:104E100037B0F0BDFF226B6829689C460233FF184B
:104E20000B12013613409C4200DA1C00FF200A14CA
:104E3000024003926246014001920091039A0B499D
:104E400004A807F0FFFB04A801F092F82800FFF780
:104E50007DFF0500ADE7C0460C11002042E10000D7
:104E60001011002000C0FEFFECE000002EE1000069
:104E700070B50020FFF704FF04000120FFF700FFDA
:104E8000844200DA04000A4B1D686A42554128003A
:104E90001D60FFF7E5FEA0226B4252021340054A57
:104EA00028009B18044A611C1360FFF70DFF70BDBA
:104EB0000C1100200480010010110020F8B5002022
:104EC000FFF7DEFE07000120FFF7DAFE3E00204D6F
:104ED0000643204C0DD18021C020C9024002FFF7BB
:104EE000A1FE01213000FFF7EFFE1B4B2E60236077
:104EF0001DE0874209DD0023B0212B60164B89029B
:104F0000236023680020012517E0012380212B6006
:104F1000124BC9022360F4E7120E522A08D000286F
:104F200000D023600E4801F023F8FFF7A1FFF8BD81
:104F300028005A68023292009B188B4205D21A68E8
:104F4000561CE9D10028F2D0D1E72160EFE7C04636
:104F50000C110020101100200480010004C0020088
:104F600007E1000070B50020FFF7F0FEFF26050006
:104F7000002801D1280070BD03681C143440FFF7DD
:104F8000E5FEDA2CF4D10500F2E700008022F0B54E
:104F90005200A1B00021674807F010F880220021DC
:104FA0005200654807F00AF8644BFF271B681A0097
:104FB000049353425A4110000592FFF751FE049C9E
:104FC0000020631E9C415E4B64421C405D4BE41814
:104FD000FFF7C8FF0600002E2DD10498FFF750FE02
:104FE000411C0598FFF770FE059A574D534B2C60F6
:104FF0001A60FEF725FD514B64201B68A0215A4220
:1050000053414F4A5B421340B0222C6892029B18D6
:10501000E41A6043490204F08DFEA022520203000C
:1050200000924A49220007A807F00CFB07A800F0ED
:105030009FFF21B0F0BD3268131412123A403B407A
:1050400003921A000A3A092A49D83A4B039A995C02
:10505000002931D110223E4806F0B0FF35002B6800
:1050600003991A123A40914209D11A143A400B2A74
:1050700027D0132A2DD00A2A01D1354B1D602800D4
:10508000FFF764FE051EEAD1314B196800290FD0E5
:105090002000FFF74FFE04002D4B5B1959680029D3
:1050A00003D02000FFF746FE040004350C2DF3D199
:1050B000204B0121039A99543000FFF747FE060068
:1050C00089E73B40022BDADC214A9B00D3185D6064
:1050D000D5E7102200211E4806F070FFCFE71A0026
:1050E000153A082AE8D8144A0399525C002AE3D1F9
:1050F0003500152B00D01500300003681A143A4013
:10510000152A0FD01D2A00D10025FFF71FFE002809
:10511000F3D1002D04D020002900FFF70BFE04007E
:10512000054BC6E7039A1B123B409A42EDD105009E
:10513000EBE7C0460C100020141100200C110020D9
:1051400000C0FEFF04C0020010110020D1E00000EA
:10515000302F002010B5FFF719FF10BDF0B585B056
:10516000039203220333DC17294D1440E4182B6803
:10517000284F5A42534180225B42D202A4103B4046
:105180009B18A21C0291244E91000091019031685D
:1051900000980A18934215D2FFF7F8FE2B685A427E
:1051A000534180225B421F40D202BF183368009AED
:1051B0009B189F4206D2194800F0DAFE002528000D
:1051C00005B0F0BD029B356819066B461A7BA42317
:1051D000DB051343FF222F00090C1943019B120426
:1051E0001B04134019432800FFF75CFD0837281DF6
:1051F00021003760FFF756FD002C04D00A9A2100E9
:105200003800FFF775FD009B083BFF183760D6E7B5
:105210000C11002000C0FEFF10110020ABE00000C8
:1052200070B59AB0FFF74AFEFF221E4CD200002153
:10523000200006F0C3FEFF25FFF794FE002600289D
:1052400014D10200C300E3580130591E8B41D2181B
:10525000FF28F7D1144901A807F0F4F901A800F0DC
:1052600087FE124800F084FE1AB070BD03681A145D
:105270002A400A2A0AD11A122A40FF2A03D0D20051
:10528000A1180B71A050FFF761FDD8E7132AFAD1DE
:105290001B122B40FF2BF6D0DB00E2181671E650F4
:1052A000F1E7C046A825002077E100008BE100006F
:1052B0000021094B094A59600131516059680029A0
:1052C000FCD000211961012393600222044B81313B
:1052D000FF315A501A607047FC1000400010004027
:1052E00000E100E00222064B0121DA670022054BB3
:1052F0005A61054A11615A69002AFCD07047C046BC
:1053000004E100E0FC1000400010004010B5044C27
:105310002378002B01D0FFF7E5FF0020207010BD9F
:1053200015120020802301205B055B6E5B00184393
:10533000704700000120024B1B685B001843704758
:10534000981200200120024B1B685B001843704735
:10535000240000200120024B1B685B0018437047AB
:105360009C12002070B504000D001600FEF724F911
:10537000802301215B055A6E267000265300617060
:10538000E1706272010A5A0A6071A171A272010C85
:105390005A0C000E5B0EA6702571E1712072E2724C
:1053A000237370BD10B5044C200007F091F9010083
:1053B0002000FEF7DBFD10BDA11200200E4B10B542
:1053C0001B680E4C5A1C0FD00D4C002B0CD00D4CF2
:1053D000012B09D00C4C022B06D0094C042B03D016
:1053E0000A4C052B00D1074C200007F071F9010091
:1053F0002000FEF7BBFD10BD280000201CE20000CD
:105400000CDA000027E2000013DA000021E20000BD
:1054100070B5214C2278002A3DD1204B01215A60E1
:105420008022D20511605A68002AFCD00022072091
:105430001B4B1C4901255A500439585008315A5009
:1054400019481A4958501A491A485A501A495A5074
:10545000A622D2009D50082218495A5004315850B3
:10546000022017495850174917485850174804390F
:105470005850182016495850C12189005A500539F2
:10548000FF395858921802435A501249124A9950FB
:10549000FFF70EFF257070BD15120020FC000040C4
:1054A000001000400C050000746962751C050000C6
:1054B00024050000200004022C0500001405000053
:1054C000340500003C050000FFFF00002110010032
:1054D00054050000161200200405000070B50E4BA4
:1054E00006001B78002B01D1FFF792FF00200B4D27
:1054F0002C7884420ED00A4B202219780323091BF2
:105500001940084B4901C918300006F03BFD012045
:10551000013C2C7070BDC04615120020A012002066
:105520001412002016120020002370B588B0984293
:1055300035DD0D6801262C0034409C422FD123001C
:10554000042D2CD90F222B681A402300092A26D1BA
:105550006A683F2A23DD6846FFF7C0FF2300002862
:105560001DD06B4619783300A14203DB6B461B5DEF
:105570005B003343A200AA1801349360202CF2D1BF
:10558000092169444A780B7812021A438B781B046C
:105590001A43CB781B061343024A136004231800F6
:1055A00008B070BD9C12002070B5454B8AB01B78C6
:1055B000002B01D1FFF72CFF02AC2000FFF78EFF7C
:1055C000002802D100200AB070BD23780B2BF9D936
:1055D0006378012BF6D1E378012BF3D1002311205E
:1055E000384E394D33602B7068442379374A4178FF
:1055F0001360027809021143827812041143C278C1
:1056000012060A4332490A60002B0ED11521694463
:105610004A780B7812021A438B781B041A43CB7812
:105620001B0613433360002318E0012B1AD1152108
:1056300069444A780B7812021A438B781B041A4388
:10564000CB781A211B06134333600E23627C694416
:10565000934200DD130000229A422CD10022042044
:10566000EA54B0E7022B03D1627B10331621EEE738
:10567000042B0DD1152108226944684606F082FCEE
:105680000098019902F00CFF06F02EFB3060CAE78B
:10569000052BC8D1152108226944684606F072FC22
:1056A0000098019902F0FCFE06F01EFB3060627D5E
:1056B0000A231E21CBE7885CA8540132CCE7C04600
:1056C0001512002098120020A112002028000020AE
:1056D0009C12002010B5134B04001B78002B01D145
:1056E000FFF796FEFFF7FEFD00200F4A0F49104B13
:1056F000545058600130106058680028FCD00020D9
:1057000018610130906018690028FCD0094B0A48E4
:105710001B785B011B185350FFF7E4FDFFF7C8FD32
:1057200010BDC04615120020001000400405000006
:10573000FC100040141200201612002010B588B092
:1057400000281DDD0A68012113000B4018D1042A2E
:1057500016D90F2014682040092811D150683F281D
:105760000EDD9800101880680024084201D0401017
:10577000C4B26846C4540133202BF2D1FFF7AAFF0C
:10578000002008B010BD000010B5002813DD0C6823
:10579000E30710D56410532C0DD8084B1B78002B51
:1057A00001D1FFF735FEFFF79DFDA123044ADB0081
:1057B000D450FFF77DFD002010BDC046151200201B
:1057C0000010004010B500280EDD0C68E3070BD573
:1057D0006410FF2C08D8054B1B78002B01D1FFF774
:1057E00017FE034A034BD450002010BD15120020B1
:1057F000001000402405000013B5002814DD0C68DB
:10580000E30711D5094B64100093094B0193072C52
:105810000AD8084B1B78002B01D1FFF7F9FD6B4626
:10582000054A1957054BD150002016BDE2ECF0F4A3
:10583000F8FC000415120020001000400C050000C8
:1058400070B588B0002820DD0124086804401CD110
:1058500004281AD90F2302681340042B15D1FEF730
:1058600065F9060006F034FF0500122800D912255C
:105870002A0002210D326846FFF774FD6B465D7306
:10588000A54205DC6846FFF725FF002008B070BD83
:105890002300325D6B449A730134F1E7F0B50D00DB
:1058A0008BB0012832DD08680122040014402DD19C
:1058B00004282BD90F2301680B40042B26D16B68D9
:1058C000134223D0FEF732F96E680700731001937C
:1058D00006F0FEFE05000E2800D90E252A00012143
:1058E000113202A8FFF73EFD6A46127902AB5A73E5
:1058F00002AA73129373019B76141B0ED673137452
:105900005574A54205DC02A8FFF7E4FE00200BB0A9
:10591000F0BD3A5D02A963189A740134F1E730B51D
:1059200089B0002814DD0C68E30711D51022684601
:105930000021FFF717FD6B466A4665105D736846E8
:1059400063122D0E64149373D4731574FFF7C2FEA3
:10595000002009B030BD0000174B184A59680029D3
:1059600003D00021596001319160196900291FD0CD
:10597000002018618023DB00D3581149012B18D176
:10598000A923DB00D3585B420B600E490B78032B35
:1059900001D801330B7003200B490B78013303400E
:1059A0000B700A495B015B1809495350012393604E
:1059B00070470860FAE7C046FC1000400010004045
:1059C00024000020A0120020141200201612002033
:1059D0000405000010B5034A1021034800F090F8B8
:1059E00010BDC0469CE1000093E10000044A054957
:1059F0001368C85401339B059B0D13607047C04664
:105A0000D0160020D012002070B5114C114A236826
:105A1000834202DC0023236016E0155C411C2E004B
:105A2000FA3E012E05D899420FDA555C013D1F2D33
:105A300001D90800ECE70100151A565C6E540131DB
:105A40008B42FADC181A206070BD1570FAE7C04668
:105A5000DC1A0020DC16002010B5FDF7A3FD064B74
:105A60001A68824201D900221A601B68C31A0348CF
:105A700098428041404210BDCC120020204E0000D0
:105A800010B5094C094A23681268934200D110BD31
:105A9000074AD05CFDF7CCFF0028F8D0236801331B
:105AA0009B059B0D2360ECE7D4160020D016002048
:105AB000D012002010B50400064B074A1B6812687C
:105AC0009B1ADB439B059B0DA34200DB10BDFFF738
:105AD000D7FFF1E7D0160020D416002070B5FFF7ED
:105AE00041FAFF250400002801D1200070BD0368A1
:105AF0001B142B401D2B00D10400FFF727F9F2E700
:105B000070B5074E33680B2B08DC0C255D43054C44
:105B10000133285164196160A260336070BDC046D2
:105B2000D8160020402F002010B5FBF7A5FBFFF78B
:105B30006DF8FBF7C9FBFDF70FFFFEF7C7FBFEF79C
:105B400023FCFFF747FF01F045F801F02BFB01F0C4
:105B500057FB01F0A1FD10BD962210B512010021E6
:105B6000034806F02BFA0022024B1A6010BDC04613
:105B7000481C0020D805002070B514007F22174B68
:105B8000C000C0580D00836813401C2B01D00020BA
:105B900070BDC368190011400429F8D101690A4099
:105BA000192AF4D11B0A01339B000C30C018FDF7F1
:105BB000BDFF037806000120002BE9D0300006F07D
:105BC00087FD0023A042E2D1A34201DB0120DFE7F1
:105BD000F15CEA5C9142DAD10133F5E7A8250020B7
:105BE000064B074A1B6812689B1ADB439B059B0DFB
:105BF0000122834200DC002210007047D0160020F2
:105C0000D4160020F8B505000C0016001F1E0ED19A
:105C10000320FFF7E5FF002808D0FA20FFF7E6FE93
:105C2000E8B2FFF7E3FEE0B2FFF7E0FEF8BD501D7B
:105C3000FFF7D6FF0028F9D0FB20FFF7D7FEE8B228
:105C4000FFF7D4FEE0B2FFF7D1FEF0B2FFF7CEFED1
:105C50003012C0B2FFF7CAFE3C00E31B9E42E5DDF6
:105C60002078FFF7C3FE0134F7E7000070B5002489
:105C7000F0250B4B1B68A34202DCFFF76DFF70BDE4
:105C80002B006343074A9B181A78002A05D05978DD
:105C9000002311201A00FFF7B5FF0134E9E7C046E1
:105CA000D8050020481C0020F8B507000024F02586
:105CB0002B0063430C4A01349E18B74211D031784F
:105CC00000290BD00133D15C002311201A00FFF70B
:105CD00099FF2A000021300006F070F90A2CE7D164
:105CE000F8BD024B1C60F9E7481C0020D8050020D5
:105CF000F0B5150001222F007A4C1740A544019001
:105D00000291002F11D005AB1A706A105A70120E52
:105D10001A710522691299706D140299DD70FFF7EE
:105D200071FFCF239B009D44F0BD042D2AD90F2481
:105D300028680440042C32D1022304AA28001371DD
:105D4000FDF7F4FE050006F0C3FCC82302009B002B
:105D5000984200DD1A007C1C97420DD1984206D96A
:105D6000614804AB03226149C01806F00BF9220018
:105D700005AB02990198D2E72700611E695C05AC6A
:105D8000E155E8E7042D00D0A7E0032304AA043D71
:105D900013716B425D4105AB55710222E9E7092C95
:105DA0007ED1042205AB1A706A68511000916946D1
:105DB000521209789A70009A59701F2A01DD202228
:105DC00000926A46127806ACDA70009BBB4202DC95
:105DD00005ABE21ACDE70126BB00EB189868064038
:105DE00006D1042837D90F210368194002290CD1A4
:105DF000012323704310637042121B0E4014A270E3
:105E0000E070237105340137DFE7042921D1022333
:105E10002370FDF78BFE039006F05AFCA31C0C28A0
:105E200009D86070864201D19C19ECE7039A925D13
:105E30009A550136F6E70C226270039A925D9A55E4
:105E40000136092EF9D12E23E372237363730E34C6
:105E5000D9E7012907D1032304382370434258416D
:105E600060700234CFE7092909D104232370436805
:105E70005A1062705B12A370E6700434C3E7032902
:105E80000BD1052323700068020992B2430F9200E0
:105E90000B40D31A63701B12EDE726700134B2E792
:105EA000032C00D03DE7052205AB01091A7089B229
:105EB000420F890022408A1A11125A709970642A7E
:105EC00000DD64220421DA70081F824201DC043202
:105ED0004FE7685C58540131F6E7002D00D020E709
:105EE00053E7C046C4FCFFFF2203000078D6000041
:105EF00070B502000024F0210D4E080060438019A7
:105F00004578954203D001340A2CF6D170BDF022B9
:105F1000002106F053F8074A1368013BA34200D161
:105F20001460002329001A001120FFF76BFEEDE733
:105F3000481C0020D805002010B5B2B002236A46E4
:105F40000400137006F0C4FBC72800D9C720002343
:105F5000984207DC421C6B46FE211420FFF752FEDC
:105F600032B010BD694601335A1EA25CCA54EFE735
:105F700030B5B3B002236A460500137006F0A8FBE3
:105F80000400C72800D9C72400239C420BDC200052
:105F90003230FFF78FFD621C6B46FF211420FFF7A4
:105FA00031FE33B030BD694601335A1EAA5CCA5473
:105FB000EBE70000F0B5BDB005900C00012803DC54
:105FC0001B20FBF71BFB55E02C4B08680393C30712
:105FD00009D4042807D90F2302681340042B02D1E7
:105FE000FDF7A4FD0390254B60680493C30709D413
:105FF000042807D90F2302681340042B02D1FDF7B0
:1060000095FD049000261E4B1B680893089BB34225
:106010000BDC049B1B4A0093C821039B0AA806F0D3
:10602000DFFA0AA8FFF7A4FFCAE70C257543164B51
:106030000399ED18286806F041FB071E05D16B682F
:10604000AD680993099B9F4201DB0136DEE72868B2
:106050000499079506F032FB0835069000280BD10D
:1060600021000598079B08315B6802389847074B69
:10607000069A1A603DB0F0BD0137E3E723DB00006C
:10608000D8160020F8E20000402F0020E40F002086
:10609000F7B5234B06001B68F02100930023009AFC
:1060A0009A4211DC0024F0231A0062430192019904
:1060B0001C4A55182F78002F12D001340A2CF3D126
:1060C0001948FFF755FF29E00A005A43154882187E
:1060D0005078B04202D11278002A1FD10133DEE796
:1060E000F0223900280005F069FF02230D4A0199CA
:1060F000EB6053540D4AF1008A58009B6E70AE70ED
:10610000AA602F616F61A34202DC054B01341C6061
:10611000002331001A001020FFF774FDF7BDC046C0
:10612000D8050020481C002041E70000A8250020D9
:1061300010B5FFF79BFDFF24084AE3005B429B1864
:10614000074AD35C043B012B03D8E043C0B2FFF7FE
:106150009FFF013C002CEFD110BDC046FC070000A2
:10616000A8250020F8B505000E00FDF7FFFEFF246E
:106170000D4B18600D4AE3005B429B180C4AD35C40
:10618000062B01D0032B0BD1E743FFB232002900CD
:106190003800FFF7F1FC002802D03800FFF778FF45
:1061A000013C002CE6D1F8BD08000020FC070000EF
:1061B000A825002070B50500FF24084AE3005B42D3
:1061C0009B18074AD35CAB4203D1E043C0B2FFF750
:1061D0005FFF013C002CF0D170BDC046FC07000001
:1061E000A8250020F7B5FDF7DDF9574B1A68824264
:1061F00001D900221A601A685449821A8A420DD9BC
:10620000FF2253491860D3005248CB1A1B181B7841
:10621000073B022B0CD9013A002AF4D1F7BD072025
:10622000FFF7C8FF4C4B27E00820FFF7C3FF38E01B
:10623000FDF7C2F9071E00D101270020FDF7BAFAC9
:1062400001900020FDF7CAFA019B0090434C444D99
:10625000002B12D02368002B6ED12B682760002BF7
:106260006ED0404B01261B78002BD8D10920FFF7B8
:10627000A1FF394B1E703B4B1E70009B002B12D0B0
:106280002B68002B0FD123682F60002B1ED0324BC0
:1062900001261B78002BC7D10920FFF78BFF2E4B5F
:1062A0001E70304B1E702368002B0FD02A4E3278A0
:1062B000002A0BD19F4200D227602368FB1A312BA2
:1062C00004D90720FFF776FF012333702B68002BDA
:1062D0000FD0244E3278002A0BD1BB4200D92F6058
:1062E0002B68FF1A312F04D90820FFF763FF012321
:1062F00033702368002B0CD0019B002B09D1164E64
:106300003378002B02D10720FFF754FF00232360CE
:1063100033702B68002B00D180E7009B002B00D04E
:106320007CE7104C2378002B02D10820FFF742FFB6
:1063300000232B60237071E7009A002AA0D1B5E7F3
:10634000009B002B9FD1AEE7C81200200F27000052
:10635000A8250020FC070000BC120020B812002075
:10636000C0120020C412002037B500240500FFF73A
:106370007DFC01A80194FDF70BFA21002000FEF737
:10638000F1F8FEF7F1FAFDF73DFAFDF7C1FAFDF776
:10639000DBFAFEF735FCFDF733F9A54204D0FDF733
:1063A00071FB0248FFF7E4FD37BDC04632E700004D
:1063B000002310B501001A001120FFF723FC10BDC7
:1063C00007B56B46197069465A7013128B70131417
:1063D000120ECB700A716B46010005221320FFF7E5
:1063E00011FC07BD10B50A0001001220FFF780FC68
:1063F00010BD70B505000C00FDF7ECF8002809D0C1
:1064000020003230FFF756FB2B00220000211B201A
:10641000FFF7F8FB70BD10B50C000300110014204D
:106420002200FFF7EFFB10BD012370B5FF24084ADF
:1064300041185B42884201D3D84370BD06781D0ADB
:10644000234073409B009B5801306B40F2E7C046ED
:1064500014E3000013B50400FE2813D80A4BC20051
:10646000D05800280ED0436808309900FFF7DCFFB1
:1064700001900920FFF71EFB01AB04222100172029
:10648000FFF7C0FB13BDC046A8250020F7B501905B
:10649000FFF724FB01250400FF276D42002C01D1EA
:1064A0002800FEBD266833143B40152B0DD121007A
:1064B0000198083106F002F9002801D135123D405B
:1064C0002000FEF743FC0400E8E71D2BF8D101256E
:1064D0006D42F5E7F0B580279FB0FFF7D1FAB54CD4
:1064E000B54D2068FF00391A4019FDF787FA236877
:1064F0000600C3182360002B0ED11FB0F0BD20682A
:10650000391A2818FDF77AFA236806001B18236049
:10651000FDF748F8A94B1860002EF0DC2B78FA2B19
:1065200000D00EE12368022B07DCFFF795FA002864
:10653000E3D00120FFF768FADFE76B78AC78981EAC
:10654000182800D9F2E003F061FB0D2024282B3439
:10655000F13E707A7E94CDDEF1F1F1F1F1F1F1F1DD
:10656000F1F1EC00FF2C0ED02000FFF7C1FC00225F
:10657000934BE100CA505B181A712100009213007E
:106580001320FEF7EBFD0320D4E72000FFF780FD8A
:10659000F9E72000FFF7ACFCF5E7FFF7C9FDF2E7EC
:1065A000FFF764FB0020FFF7DFFE8648FFF7E0FC03
:1065B000E9E7632CE7D8844BA200D25821001520CC
:1065C000FFF796FBDFE7FFF789FAFF270400002CAF
:1065D000D9D025682B143B40152B04D02000FEF7A2
:1065E000B5FB0400F3E72000083006F071F8060060
:1065F0000530FFF75FFAFB20FFF7F8F92D121D2099
:10660000FFF7F4F9E8B2FFF7F1F9F0B2FFF7EEF9AE
:106610003012C0B2FFF7EAF925002B1B9E42DDDDE8
:10662000287AFFF7E3F90135F7E700211D200091F3
:106630000B000A00FEF792FDFDF724FAA3E7200005
:10664000FFF708FF9FE7FCF7C7FF05AC5F4A64212F
:1066500000905F4B200005F0C3FF02232000237051
:1066600006F036F82300020000211620FFF7CAFAD0
:1066700089E70026524AF3009B181C68002C28D09A
:106680001B790393636808349F00B81D0293FFF7DA
:1066900011FAFB20FFF7AAF901207D1CFFF7A6F9EC
:1066A000F0B2FFF7A3F9E8B22D12FFF79FF9E8B2B5
:1066B000FFF79CF90398FFF799F9E719A7420CD85F
:1066C000FFF7DEF905230298584301F08DFCFFF730
:1066D000D7F90136FF2ECDD155E72078FFF786F99F
:1066E0000134EBE70024FFF7C1FA220021000094F7
:1066F0002300DA20FEF732FDFF222100D2003048CD
:1067000005F05CFC98E7012C02D1FEF749FB3AE763
:10671000022C02D1FEF71EFD35E70120FFF724FE13
:1067200031E7002321001A001A209FE71A00C83A17
:10673000052A00D927E7002218001100FAF7D0FD3A
:1067400021E7FB2B00D0F4E62268042A00DCECE60B
:106750002E79E8781F4B360206439E4200DDE8E6BC
:10676000331D9A4200DCE0E6EB5CFE2B00D0E0E655
:106770006878AC78771E1B2800D17DE02ED80728DA
:1067800063D0082838D001282DD1FF2C10D020004C
:10679000FFF7AEFB6D79104AB31E009221002A006C
:1067A0000A20FEF7DBFC064BE400E0501B191D71CC
:1067B000701DBFE6DC1A0020DC160020CC12002081
:1067C000A825002014E70000A02D00202BE70000E2
:1067D00026E70000F6030000E21600201D285DD029
:1067E0004FD31E2871D00300C83B052BE0D8404A88
:1067F0003900FAF775FDDBE7632CD9D86A79022AEC
:1068000013D0032A1BD0012AD2D1E979AB7909022E
:1068100019432B7AA4001B0419436B7A1B060B4304
:106820005B001343334AA350C2E7002FC0DDB11E03
:106830003148FDF79BFB2F4BA400E050B8E7AB7944
:10684000A4005A1E93419B00ECE7632FB0DC05AD1A
:106850003A002749280005F095FB00232800EB5556
:10686000FFF714FE0028A3DB224B8000C258210052
:106870001520FFF73DFA9BE739001D48FFF772FC32
:1068800096E7FF2C94D06A79022A91D81A490B20F6
:1068900000912100B31EFEF761FC89E7632F00DD44
:1068A0006327002305A9BB420ADBFB430022DB1759
:1068B0003B40CB181A70152000917B1C2100EAE7A1
:1068C000EA185279CA540133EDE7012C00D06FE782
:1068D000002F00DC6CE76B79002B03D01C00322BFF
:1068E00000DD322464235C43044B1C6060E7C04637
:1068F000E1160020A02D0020E21600200400002058
:106900000122094B1A60094A1368002BFCD00322AC
:10691000074B1B68D8171040C01801238010063899
:10692000400018437047C04600C0004000C100400E
:1069300008C500400120704710B5064C200000F04B
:10694000BFFF0549200000F0EFFF0122034B1A6052
:1069500010BDC046181B0020801A0600E01A002057
:106960001FB500210E20FCF73DFE01210F20FCF792
:1069700039FE01210D20FCF735FE1C4C200000F0F3
:10698000FDFE1B4B1B4A1B6812681B49D2B28B428F
:106990000BD880239B04019301AB1A710199029AD1
:1069A0000023200000F006FF1FBD14498B4202D8CF
:1069B0008023DB04EFE712498B4202D880231B05BA
:1069C000E9E710498B4202D880235B05E3E70E49D3
:1069D0008B4202D880239B05DDE70C498B4202D80D
:1069E0008023DB05D7E780231B06D4E7F81A0020B5
:1069F000300000202C00002048E8010090D0030067
:106A000020A1070040420F0080841E0000093D00C5
:106A100010B5002815DD01240B68234211D0234155
:106A20000C4A13600C4AA04209D04B68234206D09E
:106A30002341022B09D0032B09D0A34203D0022308
:106A40001360002010BD0023FAE70323F8E7146069
:106A5000F7E7C046300000202C000020F8B50125E3
:106A60000C682C4203D10D20FAF7C8FDF8BD641064
:106A70002DD4FCF7B5FDA04229DB00212000FCF756
:106A8000B1FDFA222900D200200001F0DFFA00282F
:106A90001DD0002500270726FA22012192002000A0
:106AA00001F0D4FA002812D0282802DD0123B340D7
:106AB0001F43013EF0D20E4EAF550135052DE9D1F1
:106AC000012206210920FDF7D3F9002801D1002079
:106AD000CCE70B23012443600023F25C99005200B1
:106AE0004118224301338A60052BF6D1BEE7C04628
:106AF000E41A0020F0B50E0085B000282BDD01233C
:106B00000A68134027D1042A25D917680F22174095
:106B1000032F20D1802101AA104D13718904029AFC
:106B200028000393019100F045FE366833681C0984
:106B30005B0F3B403700A4B2A400E41ABB1B9C428D
:106B400006DD3979280000F03BFE0137F870F5E7E3
:106B5000280000F034FE002005B0F0BDF81A002037
:106B600010B504680D20E30703D56410FF2C03D98A
:106B70001720FAF743FD10BDFFF7F2FEE1B2044C17
:106B8000200000F01DFE200000F019FE0020F2E7BA
:106B9000F81A002070B5FFF7E3FE064D002128002B
:106BA00000F00EFE0400280000F009FE0120640041
:106BB000204370BDF81A002010B5002001F0C4FA7F
:106BC000800810BD10B5FFF7F7FF43000120184300
:106BD00010BD000010B5034A0D210348FEF790FFD9
:106BE00010BDC04658E70000C0E700000D4B70B56F
:106BF0001B6804000E001500002B01D1FFF79CFE5E
:106C0000E1B2094C200000F026FFF1B2200000F0B4
:106C100023FEE9B2200000F01FFE200000F086FFF6
:106C200070BDC046E01A0020181B002010B50124DA
:106C30000368234205D04168214202D08268224283
:106C400003D10D20FAF7DAFC10BD5810802801D9C5
:106C50001520F7E74910FF2901D91620F2E7521055
:106C6000FF2A01D91720EDE7FFF7C0FF0020EBE76F
:106C7000F7B501221400904226DD0D682A4223D088
:106C80002D4B15411B684C68002B01D1FFF754FEBA
:106C90002A4EE9B2300000F0DEFE27000122174044
:106CA00014D01441FF2C02D91720FAF7A7FCE1B247
:106CB000300000F0D1FD300000F038FF0024A04289
:106CC00002D02320FAF79AFC2000FEBD042CF2D952
:106CD0000F2523681D40092D1CD1636801925B10AC
:106CE0000093009BBB42E6DDBB00E3189D68019B5F
:106CF0001D420BD06D10FF2D02D91720FAF77EFC34
:106D0000E9B2300000F0A8FD0137EAE71720FAF7F2
:106D100075FCF9E7032DCED127001A0992B25B0F5B
:106D200092001D40551B3B1B9D42C4DD397930004C
:106D300000F092FD0137F6E7E01A0020181B002052
:106D4000154B70B51B6805000E00002B01D1FFF735
:106D5000F3FD124CEDB22900200000F07CFEF1B2F0
:106D6000200000F079FD0021200000F07FFE0028C7
:106D700001D0404270BD72B601222900200000F00F
:106D800065FE62B6200000F058FD0028F2D0200019
:106D900000F058FDEEE7C046E01A0020181B002066
:106DA00010B501240368234202D04168214203D177
:106DB0000D20FAF723FC10BD5810802801D91520AA
:106DC000F7E74910FF2901D91620F2E7FFF7B8FFCE
:106DD00040002043EFE7000070B50D211D20FFF7B4
:106DE000AFFF184C5A280CD101222A2122703D38BD
:106DF000FFF7FCFE022001F0F7F80122124B1A60A7
:106E000070BD0F211920FFF79BFF332805D1022306
:106E10008F22237020211A38EAE70D211E20FFF768
:106E20008FFFC7280AD1032500222A21A9382570FF
:106E3000FFF7DCFE2A002A211E20D9E70023237059
:106E4000D8E7C04634000020EC1A002010B5002816
:106E500003DC1C20FAF7D2FB10BD01240B681C4098
:106E600001D10D20F6E75B10012B2BDD022B03D0A7
:106E70000224042B00DD0134194B1B68002B01D1C7
:106E8000FFF7AAFF174B1B785BB2022B1CD0032B1A
:106E90001ED0012B11D1032C00D1013C00222A214C
:106EA0001D20FFF7A3FE22000E211D20FFF79EFEEE
:106EB00001222A211D20FFF799FE022001F094F8FB
:106EC0000020C9E70024D7E7220123211920F2E797
:106ED000032C00D1013C22000E211E20EBE7C0460E
:106EE000EC1A002034000020204B10B51B68040071
:106EF000002B01D1FFF770FF1D4B1B785BB2022BFB
:106F00000AD0032B29D0012B2CD121001D200124D4
:106F1000FFF716FF644205E0012C13D12921192047
:106F2000FFF70EFF7F2801DD0138FF3803007F33B4
:106F300001DA7F204042C8237F21584302F0FAFE45
:106F4000604310BD032C0BD12B211920FFF7F8FE55
:106F5000043CE7E72D211920D9E721001E20D6E7C0
:106F6000052CF7D0012400206442E4E7EC1A00204D
:106F70003400002010B50120FFF7B6FF43000120C8
:106F8000184310BD10B50320FFF7AEFF43000120EA
:106F9000184310BD10B50520FFF7A6FF43000120E0
:106FA000184310BD144B70B51B68002B02D1012093
:106FB000FFF79AFF114B1B785BB2013301D1FFF74A
:106FC0000BFF0120FFF790FF04000320FFF78CFF69
:106FD00005000520FFF788FF6D43644340436419B3
:106FE000201804F0B7FE01F08BFB04F07DFE430097
:106FF0000120184370BDC046EC1A00203400002068
:10700000F8B501231C0098422BDD0F683B4228D0C5
:107010004E6835001D4024D1042E22D90F2231683C
:107020000A40092A1DD173685C10202C00DD202441
:10703000144B1B68002B01D1FFF77EFC72B67F104A
:10704000F9B2114F2200380000F000FD62B6A542EF
:1070500014DA380000F0F1FB002804D101246D009F
:107060002C432000F8BD380000F0ECFB0122AB00FF
:107070004000F31810439860AD18E8E7640001255C
:10708000EEE7C046E01A0020181B002010B5054CA2
:107090002368002B02D01B20FAF7B0FA00202060F2
:1070A00010BDC046F01A002010B5002803DC1C20DB
:1070B000FAF7A4FA10BD0B68DA0706D4042B04D93A
:1070C0000F221B681340032B01D02420F0E7034B51
:1070D00025201B68002BEBD01B20E9E7F01A0020CD
:1070E00010B5002803DC1C20FAF788FA10BD0B68E5
:1070F000DB0701D40D20F7E71B20FAF77FFA002009
:10710000F4E710B50400802803DD2620FAF776FAAC
:1071100010BD002CFCDD1B20FAF770FA012000F0F6
:1071200063FFF6E710B5002805DC1C20FAF766FAC5
:107130000400200010BD144B1B68002B01D125203A
:10714000F4E701240868044006D01B20FAF756FA39
:10715000012000F049FFF8E70428EAD90F2102686E
:107160001140042906D1FCF7E1FC05F0B1FAFFF764
:10717000C8FFDEE70329DCD1100980B2520F80007E
:107180000A40801AF3E7C046F01A0020044B10B5FD
:107190001B682520002B00D01B20FAF72FFA10BD0A
:1071A000F01A002010B5034A05210348FEF7A8FC99
:1071B00010BDC0464CE8000074E800000020704795
:1071C0000120704700207047002070470020704762
:1071D0000120704700207047002070470020704752
:1071E0000020704700207047002070470020704743
:1071F00000207047002070477047704770470000BC
:1072000010B5034A0F210348FEF77AFC10BDC046B3
:1072100090E8000008E900000378013B1F2B00D92B
:1072200070470130F8E710B5FFF7F6FF0378002B41
:107230000BD00130222B11D10378002B03D0421C3C
:10724000222B03D11000FFF7E7FF10BD5C2B03D109
:107250004378002B00D0821C1000EDE73A2BF2D0CF
:107260002C2BF0D07B2B0BD1FFF7D6FF0378002B14
:10727000E9D07D2B01D10130E5E7FFF7D4FFF5E739
:1072800020225B2B14D1FFF7C7FF0378002BDAD045
:107290005D2BF0D0FFF7C7FFF7E7202BD3DD2C2BBA
:1072A000D3D0190091435D29CFD0222BCDD001300E
:1072B0000378002BF1D1C6E7002210B5904216D01A
:1072C000FFF7AAFF03780422222B10D0023A7B2B6F
:1072D0000DD0013A5B2B0AD019003039023209294E
:1072E00005D92D2B05D14178303909290AD810004C
:1072F00010BD0522742BFAD00132662BF7D0013273
:107300006E2BF4D0581E83415A42F0E770B5FFF758
:1073100083FF037801222D2B01D18018023A00232C
:107320000A2502E06B430130CB1801783039CCB22A
:10733000092CF7D95A43100070BDF8B50C001500A0
:10734000FFF76AFF0378222B02D000232370F8BDD9
:107350000D236A1E210008250C260A279C460130B1
:107360000378222B02D100230B70F0E7002BFAD018
:10737000441C5C2B0BD14378841C622B0ED0662BF3
:107380000ED06E2B0ED0722B0ED0742B0ED0002A86
:10739000E9DD0B70013A01312000E1E72B00F6E74F
:1073A0003300F4E73B00F2E76346F0E70923EEE73A
:1073B00010B50400FFF737FFA04203D90378013B63
:1073C0001F2B00D910BD0138F6E710B5002815D0E5
:1073D0000378002B13D0FFF71FFF20210378020052
:1073E0008B4300205D2B09D01000FFF71CFF0378B2
:1073F0002C3B5A425341C018FFF70EFF10BD180036
:10740000FCE70300002070B50C0081420EDD1A7805
:107410005B2A0BD1581CFFF7FFFE0125AC4205D0BB
:10742000FFF7D3FF002801D00135F7E770BD70B535
:107430000C001500002901D000230B70002820D07B
:107440000378002B1ED0FFF7E7FE037806002C2BF5
:1074500003D10130FFF7E0FE0600337800207D2BDA
:107460000FD0844204D02A0021003000FFF765FFCE
:107470003000FFF7D8FE03783A2B02D10130FFF736
:10748000CBFE70BD1800FCE7F0B50D0004009DB008
:107490002E78002E35D02E21280005F001F9071E88
:1074A00014D0431B0193303E092E14D82800FFF757
:1074B0002DFF01002000FFF7A4FF0400002C20D0C6
:1074C000002F1ED0019B0133ED18E1E7280005F0E5
:1074D000FFF80190E7E723787B2B11D1601C642231
:1074E00003A9FFF7A4FF041E0BD0019A290003A8EB
:1074F00005F0F5F80028E1D02000FFF794FEEEE754
:10750000002420001DB0F0BD70B5050000200C0067
:1075100081421DDD2800FFF7CFFE0300681C012B10
:1075200014D00020022B13D10022681C1100FFF799
:107530007EFF012C0CD0FFF748FF00221100FFF75F
:1075400076FF013CF5E7FFF740FF013C012CFAD143
:1075500070BDF8B5050000200C0016001F00814228
:107560000DDD2800FFF7A8FE03000020022B06D146
:10757000681C3A003100FFF75AFF012C00D1F8BD1A
:10758000FFF723FF3A003100FFF751FF013CF4E71A
:1075900010B50024A04218D0FFF73EFE03787B2BE5
:1075A0000AD1013000221100FFF741FF00280CD062
:1075B000FFF739FE0134F5E75B2B06D10130FFF709
:1075C00004FF002801D00134F9E7200010BDF8B510
:1075D000002816DD0D68EB0713D56D10013D012461
:1075E000FDF7C0FC0026FF27644200280CD1002EC6
:1075F00021D0300005F06CF801003000FCF7B6FC3B
:10760000F8BD01256D42EAE703681A143A40152ACD
:107610000BD11B123B409C4200DA1C009D4201D161
:1076200006000836FDF792FBDFE71D2AFAD1012498
:1076300000266442F6E70120013464002043DFE7BE
:1076400010B508680C00FCF771FAFEF71FFF002860
:1076500003DB6268024B8000C250002010BDC046B0
:10766000A02D002010B50868FCF760FAFEF70EFFA9
:107670000123002802DB024B8000C358180010BD14
:10768000A02D002010B50868FCF750FAFEF7FEFEAA
:10769000C043C00F800010BD10B5034A0421034849
:1076A000FEF72EFA10BDC046A4E900009EE90000D6
:1076B00010B5FCF75DF9FCF70BFAFEF735FA044854
:1076C000FEF756FCFDF7ACFDFEF732FD10BDC046DF
:1076D000F3E9000010B5FBF7D9FD10BD70B500252A
:1076E00004AC24780573A94205D10A4B0A4A252126
:1076F0000A4804F0D9FB01600949920052589B00E6
:1077000002715B58A4008371635885604371022342
:10771000C37170BD0BEA00006AEA000019EA0000BC
:10772000C8EA0000037B002B04D143738373036119
:1077300001330373704700001FB50191A02100249D
:107740000068C900D2B24450012A10D0A24209D028
:10775000032A0AD0074A8350074B019AC2500123DB
:1077600043501FBD02221343F4E70422FBE7062225
:10777000F9E7C046540500002405000010B50400D8
:10778000FFF7D0FFA1222368A179D2009950617937
:10779000064A20009950217904329950044B196807
:1077A0005A689B68FFF7C8FF10BDC0460C05000073
:1077B0000C1B00201FB5FFF7BFFF05B000BD7047D1
:1077C0000368074A99501A00FC32D1680029FCD09E
:1077D000A321C90058580023C0B2D3607047C046E7
:1077E0001C05000007B58022074BD2051A60002255
:1077F0009A6002321A710F230C3200930349023B44
:107800000348FFF76BFF07BD0C1B00200030004052
:10781000F81A0020F8B505000E0017000024BC423D
:1078200008D02B68315D1B6828009847002801D0DC
:107830000134F4E72000F8BD704710B51C3000F0AB
:10784000AFF910BD10B51C3000F09CF910BD10B59B
:107850001C3000F0ABF910BD70B5437E0D00002B5D
:1078600001D1002070BD6430040000F0A8F90028A8
:10787000F7D12000290000F076F90120F2E700009E
:10788000F7B50193FA23002504009B0083600B4B9E
:107890004560083303601C300F00160000F058F9F3
:1078A0002000643000F054F96B461B79276166753F
:1078B0006576A5762000A375FEBDC046A8EA000047
:1078C000012330B5A024C375837D13499B005A580A
:1078D000437DC132114DFF32E40592009B005B589D
:1078E0001551CC22C133FF339B001D5104690C4B51
:1078F0005204E25005220469243BE250837D04696E
:107900009B005A58A123DB00E250437D02699B0093
:107910005958044BD15030BDC8EA00000C06000095
:10792000240500000C050000A022002310B5046906
:10793000D200A3500A4CA1420FD90A4C8C425B41A1
:1079400009495B420B40CD21C9045B180469074912
:10795000635005210369995010BDCC235B04F5E702
:10796000A086010090D00300000098FD24050000CF
:10797000F7B5040000200D000193824265D0160087
:10798000402A00D9402627001C37380000F0F6F8BE
:10799000B1232269DB00D5508022012321699200A6
:1079A0008B50A27E002A03D12269136222691360E0
:1079B0000025731EAB4207D1019B002B04D080220F
:1079C0000221236992009950012223691A622369D6
:1079D000FC33DA68002A02D19A6A002AF9D09A6A3E
:1079E000002A0BD1DA60A3232269DB00D1583800CA
:1079F000C9B2013500F0B7F8B542DAD3019B22696C
:107A0000002B0FD11300FC339B6A002B0AD10133EA
:107A1000A376D3612369FC33DA6C002AFCD0002200
:107A2000DA640AE000230121A37651611A00236978
:107A3000FC3399680029FCD09A602369FC339A6A68
:107A4000002A01D000229A62E8B2FEBD10B50123DF
:107A5000FFF78EFF10BD0300AC3310B504001970A2
:107A6000643000F08BF80123637610BD0023020020
:107A700070B5AC3243760D001178B1220400006974
:107A8000D20081508022216992008B5022690133FB
:107A900013622269936026006436300000F080F89B
:107AA000002812D0300000F06DF81E4B2269D05033
:107AB0002369FC331A6A002A02D19A6A002AF9D093
:107AC0009A6A002A01D11A62E5E723690122002D92
:107AD0000DD11900FC31896A002908D1DA612369C6
:107AE000FC33DA6C002AFCD00022DA6407E05A6129
:107AF0002369FC339A68002AFCD000229A60002097
:107B00002369FC339A6A82420BD098622169064A43
:107B10008B588B501800022B03D0181F431E98411E
:107B2000033070BD1C050000C404000010B5012125
:107B3000FFF79CFF10BD000010B51323142202496B
:107B40000248FFF79DFE10BD00400040181B0020BA
:107B500010B540220021040004F030FA0023200078
:107B60002364636410BD10B53F24026C531C234092
:107B7000446C9C4201D08154036410BD0023036413
:107B800043647047436C026C934206D03F21C25C51
:107B900001330B4043641000704701204042FBE773
:107BA000036C406C181A00D540307047436C026C6F
:107BB000934201D0C05C704701204042FBE73F2266
:107BC000036C406C01331340181A43425841C0B251
:107BD0007047000003210A4802680A43026009480E
:107BE00002680A4302600849084A094B9B1A03DDF0
:107BF000043BC858D050FBDC00F012F8F8F784FAC8
:107C0000240500405405004018F00000000000204A
:107C100070020020FEE7FEE7FEE7FEE7FEE7FEE774
:107C2000014B024A1A607047380000200024F4001B
:107C30000120704710B503681322DB69984710BD17
:107C400070470000054B0269D1500369FC331A6A82
:107C5000002AFCD0002201201A6270471C05000097
:107C6000030010B55C331A781F231A401E3B19001D
:107C70009140114AD167C222042104699200A150A7
:107C8000026953600269D360A02300220169DB000E
:107C9000CA5001230169094A5B428B500169084AB5
:107CA0008B5001690C3A8B50016908328B501430AB
:107CB000FFF764FF10BDC04604E100E00C050000C2
:107CC0001405000010B51430FFF76AFF10BD10B5A1
:107CD0001430FFF76BFF10BD10B51430FFF752FFE3
:107CE00010BD0000030070B55E331A780469724B52
:107CF000E25003005D331A780469704BE2500300D0
:107D000061331C7802696E4B012C00D09EE00500A7
:107D10005F352E78A225ED005651020060321578AD
:107D2000A1220669D200B5500269D4509623DB0027
:107D3000994200D88CE096231B01994200D88AE032
:107D400096235B01994200D888E096239B019942D3
:107D500000D885E0E1239B01994200D882E0962378
:107D6000DB01994200D880E0E123DB01994200D891
:107D70007DE096231B02994200D87AE0E1231B02A2
:107D8000994200D877E096235B02994200D874E0CC
:107D9000E1235B02994200D871E0E1239B02994202
:107DA00000D86EE0474B994200D86CE0E123DB023B
:107DB000994200D86AE0E122002312038A425B4123
:107DC000414A5B421340802252059B1801693F4A99
:107DD0008B50A02304220169DB00CA5000210369F3
:107DE000FC33D9600369FC331962012301690B601C
:107DF00001698B60C1210469890062501F215C30D8
:107E000002780A4093406231314AFF3153500021D9
:107E1000415600293CDA0F230B40083B2D4C9B08B0
:107E20009B001B1903242140A140FC348C40DD69D8
:107E3000A5432C00C0258D4029002143D9611F2373
:107E4000017819401E3B8B40136070BD00246CE725
:107E50009E23DB02BAE79D231B03B7E71E4BB5E762
:107E60001E4BB3E7EC239B03B0E71D4BAEE71D4B66
:107E7000ACE71D4BAAE71D4BA8E71D4BA6E71D4B22
:107E8000A4E71D4BA2E78023DB049FE71B4B9DE784
:107E90008C080F4BA400E41803230B40FF21C025DE
:107EA000DB009940AD0066598E433100C0269E40EC
:107EB00033000B436351C2E70C05000014050000BA
:107EC0006C05000090D0030000D0BEFE2405000029
:107ED00000E100E000ED00E000B0130000502700DA
:107EE00000A04E0000F0750000509D0000F0EB0077
:107EF00000903A0100E0D70100B0AF0300705F07C7
:107F0000F7B5009308AB1B7800250193FA23040012
:107F10009B0083600E4B45600833036014300F00F4
:107F20001600FFF715FE23005C3327611E70009BCF
:107F3000084A9B00995823005D331970019B20006B
:107F40009B009A5823005E33DD701A70FEBDC04658
:107F50004CEB0000C8EA0000036910B51A00FC32BF
:107F6000D2680400002A0AD0A322D2009958143003
:107F7000C9B2FFF7F8FD00222369FC33DA6010BDB7
:107F800010B50248FFF7E8FF10BDC046D01B002027
:107F9000162307B5022200930249013B0248FFF76E
:107FA000AFFF07BD00200040D01B002010B5002807
:107FB00001D004F0BFFA10BD0849094A094B10B5B9
:107FC0001B688858FA22190A1B06184392000023DE
:107FD00001F0E8FF4904C00B084310BD0010014048
:107FE00004050000341C002070B5041E09D0FFF702
:107FF000E3FF050000F014F8FFF7DEFF401BA0428E
:10800000F8D370BD0022044B9A60044A1368013310
:10801000DBB213607047C046FC100140341C0020E6
:108020007047704710B500F05FF8FFF7FAFF0120C6
:10803000FFF7DAFFFFF73CFBFFF74CFB024B002B8F
:10804000FAD000E000BFF7E700000000F8B54C1ED2
:10805000A1410125104B114F8000C3584C42386894
:108060000F499D40160001F0DBFD0A21704301F02D
:10807000D7FD2C400300220029000A4800F016F822
:10808000FA21094C89004443386801F0C9FD010018
:10809000200001F0C5FDF8BDC8EA0000380000204E
:1080A00040420F00100500501027000030B5046852
:1080B0000C40944206D1013B002BF8D112E0013B69
:1080C000002B0FD004680C409442F8D100240568BE
:1080D0000D40954204D101349C42F8D1002002E0C9
:1080E000201C00E0181C30BDC420114B80001A5821
:1080F00010491140C02212020A431A50C0218022A6
:10810000490092025A501A608023A3220021DB0505
:10811000D20099500122F9309A60074BFF30195074
:10812000C120023180001950403019501A60704748
:1081300000E100E0FF00FFFF00100140014B18606C
:108140007047C04684000020F7B5002320285AD885
:10815000384B8000C258042A5BD007D8022A54D07A
:1081600055D80423012A09D000234CE0062A54D014
:1081700051D31A2A53D002231B2AF5D12E4A116853
:1081800008294ED909294FD00A240226A02001250A
:108190002A4AC00015502A482A4D07681C20BF00F3
:1081A00007402948019700685759009027481B024B
:1081B00007401F43C02300989B020340FF205751F4
:1081C0005759000207401F43019B1F43009B580162
:1081D0006023184007433E43565101251C4B156050
:1081E00058680028FCD000205860A1230125DB003E
:1081F000D3585560A025ED0050511BB2A14202D0CA
:1082000015D2611ACB401800FEBD0823B6E7102333
:10821000B4E72023B2E74023B0E78023AEE7012391
:10822000ACE708240026B1E70C000126AEE7091BE5
:108230008B40E8E7C8EA00008000002000700040A2
:108240003C0000200405000040000020FF00FFFF6C
:10825000FC700040F0B520285BD8364B8000C25837
:10826000354B1E68002E30D1C227344BBF00D85981
:10827000334C03250440C02000022043D851C024C1
:1082800080206400800018512E4F18602E4B803CD7
:10829000D859FF3CA043D8510437D859A8432043AC
:1082A000D8510837D8590C35A8438446072065466D
:1082B0002843D851A820C0001E50C120802680002D
:1082C00076021E501C601C4B1C60142500202B00E5
:1082D0001E4C2E0046433659771C1BD14343E250B7
:1082E000A0230325C132FF329200DB05D550184B85
:1082F0001A68082A14D114234343E3189A681248D1
:108300005132FF32920059601150DA68C1239B004C
:10831000C250F0BD9642E1D001300328D9D1F8E730
:10832000082A02D9083AD140E5E708239A1A914071
:10833000E1E7C046C8EA0000381C002000E100E088
:10834000FF00FFFF040500000090004044000020F3
:10835000840000202149F0B54A6C2148002A14D03D
:10836000A025A12600230124ED05F600C258571CC4
:1083700006D0C7187F68002F02D027009740AF5162
:1083800014333C2BF2D100234B64A0230121DB05E5
:1083900000260F009C4614234B43C3181A1F126873
:1083A000104C0E4D920014195219526C002A10D024
:1083B0001A00143A1268551C09D0103B1B68FF2B99
:1083C00005D03B00934065461A00074BEA50FC3449
:1083D000666401310429DED1F0BDC046FC90004046
:1083E00044000020009000400C05000000B520284B
:1083F00010D80C4A8000835803290BD8A02208000B
:10840000C133FF33D2059B0001F000FC02090507D0
:108410000021D15000BD0C21FBE70421F9E7032125
:10842000F7E7C046C8EA000020280AD8074B8000BA
:10843000C25801239340A022D205002902D1044949
:1084400053507047A121C900FAE7C046C8EA0000AE
:108450000C05000003000020202B0AD8A021A22236
:10846000C905D2008858034A9B009B58D840012375
:1084700018407047C8EA0000F7B506000D000C0070
:108480008B180193019B671B9C4207D033682178AE
:108490001B683000984701340028F3D13800FEBD36
:1084A000F0B5C64600B5CB0F9846404A4B005B0D71
:1084B0009A1882B00D000400132A2FDC002A49DB31
:1084C0003B4F17413E000E40064323D07F08390042
:1084D00029400C430AD03749BD438C4663445C4273
:1084E0005C418023DB021341E4071D434146CE007B
:1084F00031492B008E19220034687568200029004C
:1085000001F0F6FE009001910098019922002B00E5
:1085100003F086F802B004BC9046F0BD332A08DDB3
:108520008023DB009A42F5D102000B0001F0E0FE4F
:10853000F0E7224A9446012263445242DA40024262
:10854000E8D052080242D1D094438022D2051A4189
:108550001443CBE74B005B080343DBD00B031B0B3F
:108560001C436342234380244D0C24031B0B2340F4
:108570006D042B4319004346DA000F4B9B181C680F
:108580005D6802000B002000290001F0B1FE0090A0
:1085900001910098019922002B0003F041F8424616
:1085A0004B005B08D60733431900B3E701FCFFFF1C
:1085B000FFFF0F00EEFBFFFF80EB0000EDFBFFFF76
:1085C000F8B5274A4B005B0D9A180C000700132AD8
:1085D00010DC002A36DB234B13410B423AD08024B7
:1085E00024031441002064189C4306002500300039
:1085F0002900F8BD332A0EDD80230600DB000D00C4
:108600009A42F4D102000B003800210001F070FE04
:1086100006000D00EBE7144D0600AC46012563444F
:108620006D42DD40AC4663460D000342DFD033238C
:108630009A1A323B93401818874200D94C1C634663
:108640009843D2E7C90FCC070020531CCDD1074B6C
:108650001C43CAE706000D000028C0D1C7E7C0468A
:1086600001FCFFFFFFFF0F00EDFBFFFF0000F03FED
:1086700030B5214A4B0087B05B0893421EDD1F4A8C
:10868000934205DD02000B0002F0CAFF07B030BDC7
:1086900002AA00F095F803231840049A059B0128CC
:1086A00013D002281DD0002814D00298039900F09E
:1086B0006FFB80231B069C466144E7E700230022F2
:1086C0000093002301F0DEF8E0E70298039900F040
:1086D0005FFBDBE7012402980399009401F0D2F8D4
:1086E000D4E7012402980399009401F0CBF8802389
:1086F0001B069C466144C9E7FB21E93FFFFFEF7F72
:10870000F0B54746CE4680B58DB004000D0000F0B0
:1087100067FA294B06001B780F005BB298460133BD
:1087200010D022002B002000290003F0C1FA81465E
:10873000002807D1002200232000290001F00AFCB4
:10874000002806D1300039000DB00CBC9046994687
:10875000F0BD01230293194B0694079503934B46F2
:108760000A93434604940595002B15D0002300225C
:108770001900100002F0D8F8434608900991022B26
:108780000ED103F0AFFB212303600A9B0193002B62
:108790000CD1089E099FD5E7002300240893099473
:1087A00002A801F0C1F90028EFD1EAE703F09AFB33
:1087B0000A9B01930360ECE78800002090EB000027
:1087C000F0B54E464546DE465746E0B5E14B4C0017
:1087D0008FB09046894664089C4200DC87E0DE4BFF
:1087E0009C4222DCDD4A002900DC92E0DC4B02F0F6
:1087F00017FFDB4B06000F009C4200D17EE1D94AF7
:10880000D94B02F00DFF02000B00414630000A6018
:108810004B60390002F004FFD34BD24A02F000FF54
:10882000434601259860D9606BE0D04B9C4200DC48
:108830008FE0CF4B9C4200DD55E1CE4A2315924696
:108840009A4451460905631A19001D00040003F0FB
:108850004BFA03F07FFA02000B0020002900089277
:10886000099302F0DDFE0022C34B02F067FC0F000B
:10887000060003F039FA03F06DFA04000D0002005F
:108880000B00300039000A940B9502F0C9FE00225B
:10889000B94B02F053FC002200230C900D9101F023
:1088A00053FB002800D192E1002300222000290080
:1088B00001F04AFB434243410133B04A4146019231
:1088C000022208A80092524600F07CFB4B460500AD
:1088D000002B16DA802243461206944642465B6815
:1088E000454263445360D3686344D36009E00B009E
:1088F000020041460A604B600022002300258A6086
:10890000CB6028000FB03CBC90469946A246AB46CF
:10891000F0BD934B01F0ECFC914B06000F009C4224
:1089200000D13DE18F4A904B01F0E2FC02000B00C8
:10893000414630000A604B60390002F071FE894AFE
:10894000894B01F0D5FC012543466D429860D96002
:10895000D7E701F049F88A4A8A4B06000F0002F077
:10896000EDFB0022884B01F0C3FC03F0BDF90500CC
:1089700003F0F0F9794A7A4B0490059102F0DEFB9E
:1089800002000B003000390002F04AFE754A060072
:108990000F0004980599744B02F0D0FB02900391EC
:1089A0001F2D00DCC7E0029A039B3000390002F063
:1089B00037FE83468A4653465B0024155B0DE31A57
:1089C000102B6CDD04980599D322674B520502F0F9
:1089D000B5FB02000B00300039000292039302F055
:1089E0001FFE0A00010013000691079202003900E1
:1089F000300002F015FE029A039B02F011FE060001
:108A00000F0004980599614A614B02F097FB320010
:108A10003B0002F005FE069E079F0B000200390096
:108A200030000292039302F0FBFD4B005B0D834686
:108A30008A46E41A312C32DD04980599B822544B49
:108A4000920502F07BFB03000C00020002930394EA
:108A50000B000698079902F0E3FD02000B000600E8
:108A60000F000698079902F0DBFD029A039B02F0C3
:108A7000D7FD484A0290039104980599464B02F0AD
:108A80005DFB029A039B02F0CBFD02000B0030005D
:108A900039000292039302F0C3FD83468A465A4688
:108AA0005346414630000A604B60390002F0B8FD81
:108AB000029A039B02F0B4FD44460B000200A26040
:108AC000E3604B46002B00DB1BE75B462360802303
:108AD0001B065344636080231B069C466144A060D0
:108AE000E1606D420DE70B00020002F099FD434684
:108AF00000259860D9601860596002E7D3221A4BAC
:108B0000520502F08DFD214A214B0D00040002F0B8
:108B100087FD02000B00414620000A604B602900DF
:108B200002F07EFD1A4B194A02F07AFD43460125F8
:108B30009860D960E5E602000B003000390002F0D1
:108B40006FFD6B1E154A9B009B5883468A46A342C5
:108B5000A5D130E7FB21E93F7BD90240000040541A
:108B6000FB21F93F3163621A61B4D03DFB213941E9
:108B7000FFFFEF7FEAFBFFFF0000704118EC0000F1
:108B800083C8C96D305FE43F0000E03F7370032E7F
:108B90008A19A33BC14920259A837B3998EB0000B1
:108BA000D3220C4B520501F0A3FB0B4A0B4B0400E4
:108BB0000D0001F09DFB02000B00414620000A6001
:108BC0004B60290002F02CFD034A044BB9E6032355
:108BD00073E6C04661B4D03D7370032E8A19A33B7F
:108BE000F8B54746CE46674B80B50A000F0019001E
:108BF00005003940994200D19BE004000100002F9C
:108C000069DD3F1500D1B4E05F4B12039C46802321
:108C1000120B5B0313435B00CA0F67449B184A00A7
:108C2000F80703D5D20F5B009B188A0079108C4699
:108C3000002180201624894680030D189D4202DC05
:108C400029185B1B8144D50F5B00013C5B19520066
:108C50004008002CF1D100208046802020250027EC
:108C6000000609E08B425CD0D40F5B00013DE318A5
:108C700052004008002D16D0C4198B42F2DD27188F
:108C80000E00002C49DB5B1AA242894149425B1A63
:108C9000121BD40F5B00013D80443100E3185200E9
:108CA0004008002DE8D113434ED143465B083749B5
:108CB0004A468846494652104244C90702D5802197
:108CC00009060B4361460F05BD18180029000CBCAE
:108CD00090469946F8BD7B005B0803433900002BA2
:108CE000F5D0002F3CD1E30A153A6405002BFAD0E9
:108CF0008020400303423FD1002700E00F005B00CB
:108D0000791C0342FAD0250020208D40401A29000A
:108D1000D71B2200C2401A4376E7FE43F60F8E1996
:108D2000B1E79442A0D82718002CF6DB1E000023E0
:108D3000AEE702003B002800390002F0FFF92A00EC
:108D40003B0001F0D5FAC2E74346013303D0434666
:108D500001335B08ABE7012398460023C144A6E733
:108D60003B00020002F05CFC02000B0001F0DCFDA5
:108D7000ADE713000022BBE70127210020207F423E
:108D8000C6E7C0460000F07F01FCFFFF0000E03FA7
:108D9000F0B54746CE4680B587B000920193754B3B
:108DA0004F00814688467F089F4263DC02F09CFFAB
:108DB000002800D1D4E04A4643464846414602F0E6
:108DC000BDF904000D006C4A6C4B02F0B7F96C4A17
:108DD0006C4B01F08DFA22002B0002F0AFF96A4AC9
:108DE0006A4B02F01DFC22002B0002F0A7F9684A32
:108DF000684B01F07DFA22002B0002F09FF9664AD1
:108E0000664B02F00DFC22002B0002F097F9644A39
:108E1000644B01F06DFA22002B0002F08FF90290F2
:108E200003910022604B2000290002F087F9029A8A
:108E3000039B06000F002000290002F07FF9009A32
:108E4000019B04000D004846414602F077F90200FC
:108E50000B002000290002F0E3FB02000B003000B1
:108E6000390002F0DDFB02000B0000204F4902F048
:108E7000D7FB70E002000B0002F060F904000D0067
:108E80003D4A3E4B02F05AF93D4A3E4B01F030FA62
:108E900022002B0002F052F93B4A3C4B02F0C0FB8F
:108EA00022002B0002F04AF9394A3A4B01F020FA2D
:108EB00022002B0002F042F9374A384B02F0B0FB97
:108EC00022002B0002F03AF9354A364B01F010FA35
:108ED0002B00220002F032F9354B029003919F42A1
:108EE0009FDD344B00229F423DDC334900207B183C
:108EF0002E4916001F0002F093FB049005910022FA
:108F0000294B2000290002F019F932003B0002F041
:108F100087FB029A039B06000F002000290002F045
:108F20000DF9009A019B04000D004846414602F0ED
:108F300005F902000B002000290002F071FB02007D
:108F40000B003000390002F06BFB02000B000498AC
:108F5000059902F065FB07B00CBC90469946F0BD40
:108F600000201249F7E7154B002604920593144F91
:108F7000C5E7C046FFFF3F3ED43888BEE9FAA8BD2A
:108F8000C4B1B4BD9EEE213EAD529C804F7E923E58
:108F90009015CB19A001FA3E7751C1166CC1563F0E
:108FA0004C5555555555A53F0000E03F0000F03F9A
:108FB0003233D33F0000E93F0000E0FF0000E73F0D
:108FC0000000D23FF0B5DE464E4645465746E0B576
:108FD000DC4CA5440D9114001900A49A0993DA4BB6
:108FE0009200D6584D1E03901821E01E0696029559
:108FF00000F0A0FEC3430100DB1719404B1C9A0090
:109000009B1ADB001B190B9105934C1B771918D485
:10901000A59BA5009C463F1922AE6544013707E099
:10902000286802F097FE013403C60435BC4208D01C
:10903000002CF5DA00200021013403C60435BC42BF
:10904000F6D1069B002B01DA00F0FDFB069B03998D
:109050000133DB009A46099BDA0094460092002215
:10906000914672AA0492B94A6144934688469AABE3
:1090700063449B44029B002B00DABCE15D46002662
:109080000027039C4D442A686B6803CC02F056F815
:1090900002000B003000390001F02AF9083D0600FB
:1090A0000F004445EFD1049B4B441E605F600823D2
:1090B0009C46E144D145DDD10EA8042184464942B5
:1090C00061448C46069A93009C44614684460A910A
:1090D0000399083B63448C460C93009B00926344C5
:1090E0009B46009A0498D10003008C466344089183
:1090F0001E685F68002A33DD954980468C466244CD
:10910000D300984470AB9A460EAB99460022914B1F
:109110003000390002F012F802F0E6FD02F01AFE0B
:1091200000228D4B04000D0002F008F802000B0035
:109130003000390002F074FA02F0D6FD4B4601C34C
:109140009946434620001A685B68290001F0D0F870
:1091500008235B429C46E04406000F00D045D5D171
:10916000059B30001A003900984600F0DFFCFF2311
:1091700000229B0504000D0001F0E0FF00F038FC28
:109180000022764B01F0DAFF02000B0020002900DC
:1091900002F046FA0D00040002F0A6FD814602F03E
:1091A000D9FD02000B002000290002F039FA060068
:1091B00040460F00002800DCEEE0009B18215A1EFC
:1091C00092000EAB9B58091A1D000D41A9448D4019
:1091D0005D1B0EAB9D5017231B1A1D41002D2DDD6D
:1091E00001239C46009BE144002B00DC1CE20E9C0A
:1091F0000123002C00D0B5E0009A012A09D0990083
:109200000EAA54580133002C00D0ACE0009A9A42C8
:10921000F5D1059B002B0EDD012B00D1A8E1022B1F
:1092200009D1009B0EA95A1E92000EAB9B580793C2
:109230009B029B0A8B50022D00D1C1E0002300222B
:109240003000390000F080FE009B002800D194E23D
:10925000069A591E8A4210DC414A0A9894460EAA80
:109260006344944600229B0063441C68043B2243F1
:109270008342FAD1002A00D0C0E0069B0EAA013B2F
:109280009B00D358002B00D0B3E001220C9B043B81
:10929000596801320029FAD0009B9C4662441100B3
:1092A00007921A0001338B4246DC0B9863468046D6
:1092B000A59C4344A046099C9B00A1464A4498446F
:1092C000D30022AA9146049A99449446089BA59AF1
:1092D00063448446614494469A468B0063440093F9
:1092E0004346586802F036FD4B4618605960029BB1
:1092F000002B24DB4D46039C0026002701E0286854
:1093000069680CCC01F01AFF02000B003000390034
:1093100000F0EEFF083D06000F005C45EFD153461C
:109320009E60DF6004239C460433E0449C46009B1F
:10933000E144E2449845D3D1079B0093D1E600264F
:109340000027ECE794FDFFFF60ED000018FEFFFF33
:10935000FFFFFF1F0000703E000070410000204032
:10936000FFFFFF3F002180225204141B0EAA54501D
:10937000009999420EDD0EA884469B000EAA890032
:10938000D25861446344CF4800E01A68821A04C38B
:109390008B42FAD101243CE7059B002B06D1009BB0
:1093A0000EAA013B9B00D558ED1517E70022C64BCE
:1093B000300000F0EDFD002800D024E100253DE75D
:1093C00032003B000020C14902F02AF906000F00DC
:1093D000002C00D132E7059A0020BC4900F0A6FB22
:1093E00002000B003000390002F01AF906000F00ED
:1093F00024E7012250E70026002754E64B46059A51
:10940000079388468B000EA9CB58183A0895059209
:10941000002B0DD18C464146AD4B43449B00634429
:10942000043B58680139183A0028F9D0884605925B
:10943000059A0020A54900F079FB434604000D0081
:10944000002B00DA05E29E000EAB9C464346DB0093
:1094500066449C46059370AB9946049F6744009709
:10946000306802F077FC22002B0001F067FE00223A
:1094700038607960974B2000290001F05FFE083FBB
:1094800004000D00043EB945EAD14AAB03939B4664
:1094900000239A46069B4246994643460132029271
:1094A00004934B46002B00DAAAE080208A4B009DF3
:1094B0009846C005894900260027002408E00823B3
:1094C0009C460835E044544511DC43461868596809
:1094D0002A686B6801F032FE02000B003000390090
:1094E00000F006FF013406000F00A145E7DA5B46F5
:1094F000C0C39B4601239C46009BE244083B00936B
:10950000029B9A45CDD1049B9846A49B022B00DD7B
:109510008EE0002B37DC1FD1059B00271D00039B2D
:1095200000249C461E006544083E2A686B6838008B
:10953000210000F0DDFE083D07000C00AE42F4D132
:10954000089B002B03D080231B069C4664443A00F2
:1095500023000D990A604B600720079B18409B234E
:109560009B009D443CBC90469946A246AB46F0BD4C
:10957000009B0EA95A1E92000EAB9B5807935B02EC
:109580005B0A8B5057E64346002B00DA70E100205F
:109590000021DB004AAAD61848AF32687368083E3B
:1095A00000F0A6FEB742F8D1089B002B00D025E1C1
:1095B0000B0002004A984B990D9C2260636002F0F8
:1095C0002FF8434607000C00002B13DD01254CAE9D
:1095D000B14638002E0021004C4601360CCC00F07C
:1095E00087FEA146B045F7DA089B07000C00002B68
:1095F00000D015E13A0023000D998A60CB60ABE7FB
:109600000026002773E701239C46009BE1440225C6
:10961000002B00DDEBE532003B0000202B4901F080
:10962000FFFF06000F0009E60024F2E54AAB0393B2
:10963000A49B032B00D08FE74346002B00DC14E1F2
:10964000039ADB009B46130091465B441E685F68EB
:10965000234B43440293DB00994448AB9A464B4664
:109660005C681B681800210032003B0000900191EB
:1096700000F03EFE04000D0002000B00009801996E
:1096800001F0CEFF3B00320000F032FE4B46986006
:10969000D9601C605D6008235B429C46E144260063
:1096A0002F00CA45DBD14346012B00DCE3E0039ADF
:1096B00013005B441E685F68029BDB0099464A44C6
:1096C000904610E0FFFFFF000000E03F0000F03F89
:1096D000FFFFFF3F0000703E20ED0000FB21F93F3F
:1096E000FFFFFF1F984643465C681B681800210077
:1096F00032003B000090019100F0FAFD04000D00E3
:1097000002000B000098019901F08AFF32003B0033
:1097100000F0EEFD4346039A9860D9601C605D60DE
:10972000083B26002F009A42DCD14D469446002685
:1097300000244746083565442A686B6830002100DC
:1097400000F0D6FD083D06000C00AF42F4D1039BAB
:109750004A9F5D689968D868089B002B65D0802275
:10976000120694460D9B6544604464441F605D602E
:109770009960D8601E615C61EEE69A464B4607939D
:10978000059B30005A423900089500F0CFF90022BD
:109790003A4B06000F0000F0FBFB002824D0384BAA
:1097A00000223000390001F0C9FC02F09DFA524657
:1097B0000400950002F0CEFA0022304B01F0BEFC0E
:1097C00002000B003000390001F02AFF02F08CFA91
:1097D0000EAA50510122059B52441833904605931E
:1097E00093000EAAD45023E65346300039009C0063
:1097F00002F07AFA0EAB1851D04619E680230D9A82
:109800001B06CB18106053600B0002004A984B995E
:1098100001F006FF434607000C00002B00DDD5E6F3
:1098200080231B069C466444E4E62B003A000D9D11
:109830002A606B600A000300AA60EB60320023001C
:109840002A616B6188E6099BDB00009372AB04938D
:1098500032E4A49B022B00DDE8E6002B00DD92E65B
:1098600000D079E6002700246AE6002600246EE78F
:109870000020002198E60026340068E700007041CF
:109880000000703EF0B5CE46474680B587B00092E6
:109890000193474A4B00814688465B08934207DCA8
:1098A0004146484602F020FA4146031E484666D02B
:1098B0004A4643464846414601F040FC04000D003C
:1098C00002000B004846414601F038FC394A3A4B49
:1098D00006000F002000290001F030FC374A384B09
:1098E00001F09EFE22002B0001F028FC354A364B89
:1098F00000F0FEFC22002B0001F020FC334A344B28
:1099000001F08EFE22002B0001F018FC314B324A90
:1099100000F0EEFC0E9B02900391002B34D00098D7
:10992000019900222D4B01F009FC029A039B04903F
:1099300005913000390001F001FC02000B00049891
:10994000059901F06DFE22002B0001F0F7FB009A53
:10995000019B01F065FE224A04000D00214B3000FE
:10996000390001F0EBFB02000B002000290000F0A1
:10997000BFFC02000B004846414601F051FE07B013
:109980000CBC90469946F0BD02000B002000290057
:1099900001F0D4FB124A134B01F042FE32003B00AF
:1099A00001F0CCFB4A46434600F0A2FCE7E7C04684
:1099B000FFFF3F3E7CD5CF5A3AD9E53DEB9C2B8A41
:1099C000E6E55A3E7DFEB157E31DC73ED561C1199C
:1099D000A0012A3F1111813FA6F810110000E03FBD
:1099E000495555555555C53F49004B081900704715
:1099F000474AF0B54F4691464B005B0D99444646A9
:109A0000D6464A46C0B505000C000E008846070041
:109A1000132A27DC002A4BDB3E4B13419A460B00EE
:109A200052461340034318D03B4A3C4B28002100C8
:109A300000F05EFC0022002300F0A0FA002847D0CE
:109A4000002C04DA80234A465B03134198444646BF
:109A5000534600279E43380031001CBC904699466F
:109A6000A246F0BD332A08DD8023DB009945F4D1FE
:109A700002000B0000F03CFCEFE7294A944601226B
:109A800063445242DA4092460242E6D0224A234BD5
:109A90002800210000F02CFC0022002300F06EFAC8
:109AA000002815D0002C1EDB534646469F430FE08E
:109AB000194A1A4B2800210000F01AFC002200234A
:109AC00000F05CFA002803D0002C04DB00270026FD
:109AD00038003100C1E76400640825430027002DE9
:109AE000F6D0104EF4E74B46142B0BD03422D21A8A
:109AF000012393405D19BD4208D201239C462F00EB
:109B0000E044D1E7133B9C46E044CDE72F00CBE790
:109B100001FCFFFFFFFF0F009C7500883CE4377ECF
:109B2000EDFBFFFF0000F0BF002070474B0070B559
:109B30005B0D14000A00002B1AD14B005B08034395
:109B400015D0234B002201F0F9FA224B9C422DDB69
:109B50000A004B005B0D363B1F4DE318AB422ADC7D
:109B6000002B0DDD1D4C1B0522401A43110070BD5A
:109B70001B4DAB42F0D102000B0000F0B9FBF6E741
:109B80001D00353519DA174B02009C4209DD0B0028
:109B90001548164900F032F8134A144B01F0CEFA7A
:109BA000E5E70B001248134900F028F8104A114B62
:109BB00001F0C4FADBE70200E9E7084C3633224043
:109BC0001B051343190000220B4B01F0B7FACEE737
:109BD00000005043B03CFFFFFE070000FFFF0F8076
:109BE000FF07000050C300009C7500883CE4377EEE
:109BF00059F3F8C21F6EA5010000903C30B54A0031
:109C0000DB0FDB0752081A43110030BD02B4714666
:109C100049084900095C49008E4402BC7047C046AF
:109C2000002243088B4274D303098B425FD3030A9B
:109C30008B4244D3030B8B4228D3030C8B420DD3AE
:109C4000FF22090212BA030C8B4202D3121209023C
:109C500065D0030B8B4219D300E0090AC30B8B427A
:109C600001D3CB03C01A5241830B8B4201D38B0328
:109C7000C01A5241430B8B4201D34B03C01A5241CD
:109C8000030B8B4201D30B03C01A5241C30A8B4210
:109C900001D3CB02C01A5241830A8B4201D38B02FB
:109CA000C01A5241430A8B4201D34B02C01A52419F
:109CB000030A8B4201D30B02C01A5241CDD2C30911
:109CC0008B4201D3CB01C01A524183098B4201D38D
:109CD0008B01C01A524143098B4201D34B01C01A78
:109CE000524103098B4201D30B01C01A5241C308F0
:109CF0008B4201D3CB00C01A524183088B4201D35F
:109D00008B00C01A524143088B4201D34B00C01A4A
:109D10005241411A00D20146524110467047FFE7B6
:109D200001B5002000F0F0F802BDC0460029F7D0D0
:109D300076E7704703460B437FD4002243088B42EB
:109D400074D303098B425FD3030A8B4244D3030BC2
:109D50008B4228D3030C8B420DD3FF22090212BA87
:109D6000030C8B4202D31212090265D0030B8B4203
:109D700019D300E0090AC30B8B4201D3CB03C01AED
:109D80005241830B8B4201D38B03C01A5241430BC8
:109D90008B4201D34B03C01A5241030B8B4201D3B8
:109DA0000B03C01A5241C30A8B4201D3CB02C01A23
:109DB0005241830A8B4201D38B02C01A5241430A9B
:109DC0008B4201D34B02C01A5241030A8B4201D38A
:109DD0000B02C01A5241CDD2C3098B4201D3CB0131
:109DE000C01A524183098B4201D38B01C01A5241E0
:109DF00043098B4201D34B01C01A524103098B42E4
:109E000001D30B01C01A5241C3088B4201D3CB00CE
:109E1000C01A524183088B4201D38B00C01A5241B1
:109E200043088B4201D34B00C01A5241411A00D261
:109E300001465241104670475DE0CA0F00D04942CA
:109E4000031000D34042534000229C4603098B423A
:109E50002DD3030A8B4212D3FC22890112BA030AC2
:109E60008B420CD3890192118B4208D38901921144
:109E70008B4204D389013AD0921100E08909C309C9
:109E80008B4201D3CB01C01A524183098B4201D3CB
:109E90008B01C01A524143098B4201D34B01C01AB6
:109EA000524103098B4201D30B01C01A5241C3082E
:109EB0008B4201D3CB00C01A524183088B4201D39D
:109EC0008B00C01A5241D9D243088B4201D34B00B8
:109ED000C01A5241411A00D20146634652415B10FA
:109EE000104601D34042002B00D5494270476346DB
:109EF0005B1000D3404201B5002000F005F802BD20
:109F00000029F8D016E770477047C046D0400B1CB8
:109F10001141203A03D49C461341184363465242F0
:109F2000934018437047C0468446101C62468C46D6
:109F3000191C634600E0C0461FB501F097F80028E1
:109F400001D40021C8421FBD10B500F0EFFF404210
:109F5000013010BD10B501F089F8002801DB0020A8
:109F600010BD012010BDC04610B501F07FF80028DB
:109F700001DD002010BD012010BDC04610B501F06C
:109F800011F8002801DC002010BD012010BDC046E2
:109F900010B501F007F8002801DA002010BD0120FB
:109FA00010BDC046F0B5CE46474615042D0C2E0018
:109FB00080B50704140C3F0C9946030C7E435D43A7
:109FC000674363437F19340CE4199C46A54203D9C7
:109FD00080235B029846C4444B4643435143250CBF
:109FE00036046544360C2404A4195B195918200062
:109FF0000CBC90469946F0BDF0B54E4657464546D6
:10A00000DE46E0B543025B0A450083B00F1C99466B
:10A010002D0EC60F002D57D0FF2D24D08020DB0041
:10A02000C0041843002381469A469B467F3D7C022C
:10A030007A00FB0F640A120E984623D0FF2A4BD0F9
:10A04000E30080240020E4047F3A1C43AD186B1C1D
:10A0500047460193534677403A000F2B48D87D4935
:10A060009B00CB589F46002B00D085E008339A46D2
:10A07000063B9B467C027A00FB0FFF25640A120E0A
:10A080009846DBD1002C00D090E0524601231A43C1
:10A0900092460120DBE74C4658461700022824D0A0
:10A0A000032800D1CFE00022002301284DD158021F
:10A0B000D205400AFF071043384303B03CBC90462A
:10A0C0009946A246AB46F0BD002B5BD104239A46CD
:10A0D000033B00259B46AAE7FF35002C60D1524682
:10A0E00002231A4392460220B1E7FF220023DEE753
:10A0F0004B461B0C9C464B462604360C1804614606
:10A100003300220C6446000C43434E4350435443F7
:10A1100080191A0C1218964203D9802149028C46E4
:10A1200064441B041B0C1004C01883015E1EB34161
:10A13000800E1843130C1B199B0103431C002301C1
:10A1400079D5012362081C401443019A7F32002A0A
:10A150004DDD630704D00F232340042B00D00434CB
:10A16000230103D53C4B019A1C408032FE2ABCDC03
:10A17000A3015B0AD2B29AE70C239A46093BFF255A
:10A180009B4654E7180001F071FE4A46431F7625AE
:10A190009A4000236D4291462D1A9A469B4646E707
:10A1A000524603231A439246032050E7200001F051
:10A1B0005DFE431F2D1A9C40763D002047E780231B
:10A1C0000027DB03FF2272E7424666E74C46320077
:10A1D000584662E780234A46DB031A4222D01C42DB
:10A1E00020D123435B025B0A4746FF225FE701233E
:10A1F0009A1A1B2A21DC23000199D3409E318C40FE
:10A200001A0023005C1EA34113435A0704D00F22F7
:10A210001A40042A00D004335A0111D49B015B0A6E
:10A22000002244E780234A46DB0313435B025B0AB8
:10A230003700FF223BE7019587E70022002336E73E
:10A240000122002333E78023DB0323435B025B0A05
:10A25000FF222CE770ED0000FFFFFFF770B500282C
:10A260003DD0C317C5185D40C40F280001F0FEFDA6
:10A270009E22121A962A07DCD2B2082833DD08384B
:10A2800085406802400A23E0992A0BDD0523290056
:10A290001B1AD94003001B339D402B005D1EAB41B0
:10A2A00019430D00052801DD431F9D402B000F4978
:10A2B0000B406E0709D00F263540042D05D004331E
:10A2C0005D0102D59F220B40121A9B01580AD2B29F
:10A2D0004002D205400AE4071043204370BD002429
:10A2E00000220020F4E76802400AF1E7FFFFFFFBCD
:10A2F000F0B54F464646D6460C000903C0B5490A9C
:10A30000470F5E0039431F03DB0F9C4665007B0A45
:10A31000570F1F436D0DE40F760DA146C000B846E0
:10A32000D200AB1B64457BD0002B5FDD002E00D03C
:10A33000A4E03E00164300D112E15E1E002E00D0C4
:10A340009EE1871A4346B84280410125C91A40421E
:10A35000091A0B0200D431E149024E0A002E00D145
:10A360006EE1300001F082FD0300083B1F2B00DD91
:10A3700061E120223900D21A9E40D1409F400E4315
:10A380009D4200DD51E15D1B6B1C1F2B00DD7CE15C
:10A390002021C91A3D0030008F408840DD40791EE1
:10A3A0008F41310007222843D940002507433A4016
:10A3B000002A09D00F233B40042B05D03B1DBB4294
:10A3C000BF417F42C9191F000B0200D426E26A1C5C
:10A3D000C64B55056D0D9A4200D106E1C44AFF08EF
:10A3E0000A40530752023B43120B8EE0002B00D071
:10A3F000B8E06B1C5B055B0D012B00DC30E1871ABC
:10A400004346B842B641CB1A76429E1B330200D572
:10A410004CE13B003343A1D100220024002570E031
:10A42000002B00DCE5E0002E00D183E0AF4EB5420A
:10A4300060D0802636043743B846382B00DC3EE136
:10A44000434613431F007A1E97413F1887428041BD
:10A45000404209180B0200D4B0E0A44B01359D42E4
:10A4600000D1C3E0A24A7B080A4001210F401F43EC
:10A470005108D30707221F433A4099E79B4EB54244
:10A4800038D0802636043743B846382B00DDDCE070
:10A490001F2B00DC30E11E004746203EF740BC4643
:10A4A000202B04D04026F31A46469E403243170024
:10A4B00063467A1E97411F43CCE0002B00D104E293
:10A4C0004346134300D159E14B07C008184380238A
:10A4D000C9081B03194208D04546ED081D4204D1A6
:10A4E0004346D008590708432900420FC9007F4D51
:10A4F0001143C0004B07CA087C49C00803438D4282
:10A5000068D012036D05120B6D0D002112031800A7
:10A51000130B0A0D12051A43764B2D0513402B43DE
:10A520005B00E4075B08234319001CBC9046994676
:10A53000A246F0BD3E00164312D05E1E002E00D093
:10A5400000E18718874280414144404209180125B3
:10A550000B0233D5022585E76446330041461000DF
:10A560001D00C7E7002D00D0DAE00C000443F3D053
:10A570005C1C00D19FE15D4CA64200D12FE1DB4382
:10A58000382B00DD66E11F2B00DD83E12024050070
:10A59000E41A0F00DD40D940A0404346A7405B1AB3
:10A5A000441EA04198462F433843171ABA4292419D
:10A5B00043465242991A64463500CAE607223A4099
:10A5C000002A00D0F6E64B07CA084849FF083B437B
:10A5D0008D4296D11900114300D19EE180210903DB
:10A5E0000A431203120B414D8FE71500002200238E
:10A5F0008BE7002B00D0C7E06B1C5F057F0D012FA0
:10A6000000DCF1E0394DAB4200D1B9E085180A0019
:10A61000854289414244494251180722CF076D08BB
:10A620002F4349083A401D00C2E607223049ED1A7F
:10A6300031403A40BCE63E002838864000279FE67D
:10A64000380001F013FC20308EE6434613431F0010
:10A650007A1E9741C71BB84280414042091A78E6EA
:10A660000E003B0006431343002D61D1002E00D0A5
:10A67000F4E0002B00D11BE164463900100039E7FB
:10A680001A4FBB427AD03300FFE630001F3DE8404E
:10A69000202B03D04021CB1A9E4037437B1E9F4185
:10A6A000072207433A400021002589E7171A43464D
:10A6B000BA42B641591A76428E1B64464EE61F2BAB
:10A6C00000DDADE020264746F61AB740B946170030
:10A6D000B246DF404E463E4337005646B240561E15
:10A6E000B24117434246DA408918AEE6FF07000040
:10A6F000FFFF7FFFFFFF0F8020264746F61AB74077
:10A70000B9461700B246DF404E463E433700564634
:10A71000B240561EB24117434246DA40891A99E7C1
:10A720007F4CA6425BD0802424045B42214327E770
:10A73000002E0CD1002B00D1CBE064463900100074
:10A74000774DD7E6764FBB4218D0330075E6002B25
:10A7500014D04B07C00818438023C9081B031942B3
:10A7600007D0FC081C4204D17907D0080843E14611
:10A7700021004C46420FC9001143C000684DB9E6A4
:10A780001D0000220023C0E6002D5BD10D00054313
:10A7900000D1E2E65D1C00D1B0E0614DAE421FD0B9
:10A7A000DB43382B71DC1F2B00DD96E020250F00EA
:10A7B000ED1AAF40B9460700AA46DF404D463D437B
:10A7C0002F005546A840D940451EA841884407435C
:10A7D000BF18974292415142414435003AE66446DF
:10A7E00035004146100085E60B000343002D00D0E4
:10A7F00063E6002BF5D04346134300D17AE6871871
:10A800008742804107224144404209183A400B02E6
:10A8100000D4D5E6434B01351940C9E5380069E657
:10A820001E004746203EF740BC46202B04D0402661
:10A83000F31A46469E403243170063467A1E9741FC
:10A840001F4302E6364DAE42CAD080252D045B423E
:10A850002943A6E70843411E8841A6E6002B00D104
:10A8600048E6871A4346B842B641CB1A76429E1B49
:10A8700033024BD5171A4346BA429241591A5242F3
:10A88000891A072264463A4092E501430F00791E77
:10A890008F419DE71C000F00203CE740202B03D098
:10A8A0004024E31A99400843411E884138437CE61E
:10A8B0000022002425E6171A4346BA429241591A4B
:10A8C0005242891A6446350043E541461000144D52
:10A8D00010E680220024120380E61D000F00203DB8
:10A8E000EF40BC46202B03D04025EB1A994008438B
:10A8F00007006346781E87411F4369E78718974220
:10A900009B4141445B42C9183500A3E53B003343FA
:10A91000CED0072231003A4052E600231A00F4E577
:10A92000FF070000FFFF7FFFF0B55746DE464E46AB
:10A930004546E0B5834607000E03480085B09246C1
:10A940001C00360B400DCD0F002800D19DE0954B2B
:10A95000984239D08023F6001B041E43924A7B0F95
:10A960003343994694460300634400930023002632
:10A97000FF00029323031B0B98466300E40F52462B
:10A980005B0D019400D1B3E086498B4200D19EE07B
:10A990004246D100802212040A435146490F114316
:10A9A0008B46814952468C4600996344CB1A00215C
:10A9B000D20000932B0063409A460F2E00D905E188
:10A9C0007A4BB6009B599F465B463343994600D06D
:10A9D000B8E002230826002700900293CAE7CB467E
:10A9E0003A0002990195019B9A46022927D0032932
:10A9F00000D180E2012944D06D49009B8C4663441C
:10AA00001C00002C38DD530700D013E2D2085B464F
:10AA1000DB0109D55946674B19408B468021C90097
:10AA20008C46009B63441C00634B9C4207DC5B46E6
:10AA300064055F075B0217431B0B620D02E00023F6
:10AA40000027584A00211B031C0B0B0D1B05234339
:10AA500014055A4A380013401C4353466400DB0770
:10AA600064081C43210005B03CBC90469946A246B0
:10AA7000AB46F0BD0122524201231B1B382B00DCE8
:10AA8000ADE1002200230027DCE75B463343994613
:10AA90005ED0002E00D18AE1300001F0E7F903001A
:10AAA0000B3B1C2B00DD7BE11D22D31A5A46010013
:10AAB000DA4008398E4013005F46334399468F4091
:10AAC0003F4B00261B1A00930023029352E7414696
:10AAD00053460B433B499B468C46009B6344009383
:10AAE0005B46002B3BD1022300221E43022161E77B
:10AAF000434613439B4637D04346002B00D162E1C7
:10AB0000404601F0B3F903000B3B1C2B00DD53E181
:10AB100002004146083A914088461D21CB1A514611
:10AB2000D9400B0041460B439B46534693401A00C5
:10AB3000009B25499C46604403008C466344009377
:10AB4000002137E70323B14600900C26029311E75A
:10AB50000023009301330426002702930AE703230E
:10AB6000C3461E43032125E701331E430022012172
:10AB700020E700239A46802300271B03094A61E748
:10AB8000802349461B03194200D1E2E0594619428D
:10AB900000D0DEE00B431B0317001B0BA246014A4B
:10ABA00050E7C046FF07000001FCFFFFB0ED0000CA
:10ABB000FF030000FFFFFFFEFE070000FFFF0F8006
:10ABC0000DFCFFFF01F8FFFFF3030000D94500D99A
:10ABD000CBE000D1C6E03C0048460027009B013B8B
:10ABE00000935B46160E1B021E4313029846330465
:10ABF0001B0C9946310C0191FFF798F84A464243E5
:10AC00000B04210C050019438A4207D98919013D1B
:10AC10008E4203D88A4201D9851E8919881A019962
:10AC2000FFF784F809048C464A46210464464243EF
:10AC3000090C030021438A4204D98919013B8E4241
:10AC400000D8F1E02D041D43AB464346891A424625
:10AC5000280C12041D0C5B46140C22001B041B0C58
:10AC60005A4303946B434443029568431B19150CE4
:10AC7000EB189C4203D980246402A44660441C0C57
:10AC800015041B042D0C20185D19814277D373D055
:10AC90000C1AA24A7D1BAF42BF419446009B7F42E3
:10ACA0006344E01B1C00864200D1DBE00199FFF702
:10ACB0003DF84A4642430B04290C070019438A42D7
:10ACC00007D98919013F8E4203D88A4201D9871ECC
:10ACD0008919881A0199FFF729F809044A46894613
:10ACE00029044D464243090C030029438A4207D9EF
:10ACF0008919013B8E4203D88A4201D9831E8919E2
:10AD00003F04891A3A00039F1A43380013041B0CAE
:10AD1000584381460298150C6F43434345434846C8
:10AD2000000C8446DB1963449F4203D98020400213
:10AD30008446654448461F0C00041B04000C7D1922
:10AD40001818A94200D284E000D17FE001231A4301
:10AD500057E680234A461B0313431B031B0BAA46DB
:10AD60006F4A6FE6BA4200D935E74B46DC07580810
:10AD70007B081C43FF0734E70024AF4289D24744D5
:10AD80004745A4415B466442A4196418013BA642AE
:10AD90001ED2A0426DD800D1B6E0241A9B4678E7B7
:10ADA00003005A46283B9A400027914688E65846B9
:10ADB00001F05CF8203072E603005246283B9A40CE
:10ADC00093460022B4E6504601F050F820309AE64F
:10ADD000A642E2D1B845DCD9341A9B4659E71F2B6D
:10ADE00065DC504C0099A4465C46614408008C40E8
:10ADF00011008240D940501E82410C4314435A46F0
:10AE0000DA401300620709D00F222240042A05D03D
:10AE10002200141D9442894149425B181A0262D5EE
:10AE20000122002300270DE68A4200D80AE7831E8C
:10AE3000891907E70F231340042B00D1E6E5171DFE
:10AE40009742924153429B44FA08E0E5002800D122
:10AE5000D7E57118531EB14227D3A94215D358D054
:10AE60001A0073E7002B00DC04E6012300229B4458
:10AE7000CDE502234744474589415B429C46494210
:10AE800089190C19E344241A03E743465F00474538
:10AE90009B41B8465B429E19023A8919A94200D0EB
:10AEA00054E7404500D051E7ABE51A00F6E71F2113
:10AEB0005F4649420C1BE740202B07D01A49009BF4
:10AEC0008C46634418005B4683401A43501E8241FF
:10AED0003A4307270023174009D00F2100231140D0
:10AEE0001400042995D122005F075B021B0BD208D6
:10AEF00017430022A6E5802359461B030B431B037F
:10AF000017001B0B064A9DE5BD42B2D89B460024A4
:10AF1000BFE68045B9D31A00C3E7C046FF0300006F
:10AF2000FF0700001E0400003E040000F0B54F467D
:10AF30004646D6468446C0B58046194E18030F03D0
:10AF40004D00000B5C0082463F0B6D0DC90F914612
:10AF5000640DDB0F0120B5420AD0B44203D0A542F4
:10AF600001D157450CD01CBC90469946A246F0BD75
:10AF700066463E43F7D1AC42F5D154461443F2D174
:10AF80000120C845EFD1994207D0002DEBD163468F
:10AF90001F433800471EB841E5E70020E3E7C046FD
:10AFA000FF070000F0B54F464646D6464D00C0B5F7
:10AFB0000E03C90F8A462C491F035C008046360BDE
:10AFC0006D0D91463F0B640DDB0F8D421ED08C4200
:10AFD00016D0002D1ED130438446002C01D13A43B7
:10AFE00023D06246002A1AD09A4529D05146022021
:10AFF0000139084001381CBC90469946A246F0BD74
:10B0000039001143E5D002204042F4E73043FAD141
:10B01000AC420FD0002C0FD13A43E7D00CE0012214
:10B02000013B934318000130E5E763460020002B05
:10B03000E1D0DBE73A43E6D19A45D7D1A542D5DC4A
:10B04000A54205DBBE42D1D808D00020BE42D2D2F4
:10B0500050460123013898430130CCE7C845C5D894
:10B060000020C845F4D3C6E7FF070000F0B54F46FF
:10B070004646D6464D00C0B50E03C90F8A462E4936
:10B080001F035C008046360B6D0D91463F0B640D2F
:10B09000DB0F8D4218D08C4211D0002D18D13043D7
:10B0A0008446002C1ED13A431CD163460020002B5D
:10B0B00030D0514602200139084001382AE03900D9
:10B0C0001143EAD0022025E03043FBD1AC4226D028
:10B0D000002C26D13A4324D15146022001390840A0
:10B0E000013817E06246002A0FD09A45E1D1A54207
:10B0F00005DBBE42DDD819D00020BE420AD2504640
:10B10000012301389843013004E00122013B9343BD
:10B11000180001301CBC90469946A246F0BD3A4347
:10B12000D0D19A45C5D1A542C3DCE0E7C845C0D817
:10B130000020C845E3D3EDE7FF070000F0B5574610
:10B14000DE464E464546E0B5834606000F034800FE
:10B1500087B092461D003F0B400DCC0F002800D158
:10B160006FE0DE4B984238D08023FF001B041F4362
:10B17000730F3B430193DA4B0027994600239B460C
:10B18000F60081442B0369001B0B52469846490D7B
:10B19000ED0F002900D185E0D04B994200D173E03A
:10B1A0004346DA0080231B0413435246CC48520F17
:10B1B00084461343524600206144D2008944210052
:10B1C000694000918C46012149448A460F2F00D9DD
:10B1D00090E0C449BF00CF59BF465B463B43019353
:10B1E00000D06AE102230827002681469B46C9E772
:10B1F00032005846019B61460091022800D175E05B
:10B20000032800D1FEE1012800D02CE10023002713
:10B21000002600253F032A0D3F0BB34812053A4391
:10B2200002401B051343009A5B00D1075B080B43E8
:10B230003000190007B03CBC90469946A246AB4688
:10B24000F0BD5B463B43019300D12FE1002F00D1BD
:10B25000A5E1380000F00AFE03000B3B1C2B00DDCB
:10B2600096E11D22D31A5A460100DA405E4608399B
:10B270008F4013008E403B4301939C4B00271B1AC9
:10B28000994600239B467DE7414653460B4393492D
:10B290008C46E144002B00D01AE102220220174321
:10B2A00000228CE7134300D10DE14346002B00D16F
:10B2B00081E1404600F0DAFD02000B3A1C2A00DD75
:10B2C00072E10100434608398B4098461D239A1AC3
:10B2D0005346D3401A004346134352468A404946D8
:10B2E000081A824989468144002068E77B4B002781
:10B2F00000268EE7140C1204120C1100370C3604D1
:10B30000350C794328008C462E0060436044834608
:10B3100056432100300C8046584679434044029100
:10B32000844506D98846802149028C46E04441463E
:10B3300002913604010C360C00048B4681191E0C58
:10B340001B041B0C0391190079438C46280075439C
:10B350006544A8465843050C45447743A94203D9A0
:10B36000802149028C466744290C8C463900000430
:10B37000000C2D042D186144AB44059159460491ED
:10B3800001990F043F0C080C390051434243904689
:10B3900002008C46090C8B4662437C4344445C4467
:10B3A000A04503D98021490288464244210C8846A1
:10B3B00061460904090C8C463900594343437043E4
:10B3C0007E430F0CF6182404BE19644442448C4694
:10B3D000B34203D980235B0298464044029B6146F6
:10B3E0009846049B370443449B46AB45AD416B42B2
:10B3F0000D0405992D0C8C467F196744FD18A8464D
:10B400005D462D19A542A44193466442A446C34417
:10B41000DC448F42BF4198459B4193459241A445EE
:10B42000A4415B427F421F43360C52426442BF1923
:10B430002243BF18624638184302D20D03991343C2
:10B440006A020A43501E82416146ED0D2A434E02B4
:10B450003243D90100D4B3E0012650083240024300
:10B46000DE0732435B08224C5444002C62DD510756
:10B4700009D00F201040042805D0101D90429241A1
:10B4800052429B180200D90104D580241948E400D7
:10B49000034054441848844200DD27E75E075B02FE
:10B4A000D2081F0B630516435B0DB2E600239946D5
:10B4B0000133042700269B4664E603230197814657
:10B4C0000C279B465EE6012201201743002276E608
:10B4D000032303201F43434671E6C046FF070000D5
:10B4E00001FCFFFFF0ED0000FFFF0F800DFCFFFFF0
:10B4F000FF030000FFFFFFFEFE0700000023802780
:10B5000000933F030026434B83E6019B3200A44691
:10B51000584670E6AC466EE6802701993F033942F3
:10B520002DD03B422BD11F433F033F0B009516000C
:10B53000384B6EE601252D1B382D00DD66E61F2DEC
:10B5400040DC35481C005044160082408440EE40E8
:10B55000501E824134431443EB40620709D00F224E
:10B560002240042A05D02200141D9442804140420A
:10B570001B181A023ED501230027002649E6802722
:10B58000019B3F031F433F033F0B0094214B40E6C9
:10B5900003005A46283B9A40002601926DE6584621
:10B5A00000F064FC203057E603005246283B9A40E6
:10B5B0001300002293E6504600F058FC20307BE652
:10B5C000CA4650E71F201E004042041BE640202DC3
:10B5D00003D0124C5444A3401A43501E82413243BC
:10B5E00007260027164009D00F2000231040140022
:10B5F0000428B9D122005E075B021F0BD208164354
:10B60000002306E680273F031F433F033F0B16003E
:10B61000004BFEE5FF0700001E0400003E04000092
:10B62000F8B557464E464546DE460C000903E0B5E0
:10B63000490A460F5F0031431E03DB0F760A9B4623
:10B64000530F3343C84E6500C000E40FD2006D0DA8
:10B65000A24681467F0D9C469046B74200D1B9E094
:10B660005B46012673409B46EE1BA34500D183E059
:10B67000002E63DD002F00D0B1E06346134300D1FC
:10B6800023E1731E002B00D0BAE1861A6346B04254
:10B6900080410125C91A4042091A0B0200D447E132
:10B6A00049024B0A98464346002B00D189E14046A7
:10B6B00000F0DCFB0300083B1F2B00DD7CE12022B7
:10B6C0003000D21A4146D040994002009E400A43C1
:10B6D0009D4200DD6AE15D1B6B1C1F2B00DD94E1C8
:10B6E000202110003500C91A8E40DA408840DD4024
:10B6F000711E8E4111000722284300250643324067
:10B70000002A09D00F233340042B05D0331DB34248
:10B71000B641764289191E000B0200D43DE26A1C34
:10B72000914B55056D0D9A4200D119E18F4AF608EB
:10B730000A40570752023743120B9BE0002E00D0FD
:10B74000C5E06E1C7605760D012E00DC48E16746EB
:10B75000861ACB1BB042BF417F42B8461F0043460A
:10B76000FF1A3B00B8461B0200D55FE137439AD170
:10B7700000220024002579E0002E00DCFAE0002FF2
:10B7800000D18DE0784B9D4267D0802367461B0433
:10B790001F43BC46382E00DC52E1634613435A1E59
:10B7A00093411E1886428041404209180B0200D482
:10B7B000BEE06D4B01359D4200D1D2E06B4A73086B
:10B7C0000A4001210E401E435108D30707221E43A1
:10B7D000324095E71E00164300D045E740E7624B34
:10B7E0009D423AD0802367461B041F43BC46382E37
:10B7F00000DDEBE01F2E00DC3AE133006746203B22
:10B80000DF403B00202E05D04027BF1B6646BE40D0
:10B81000324390464646721E96413343DAE0002B8F
:10B8200000D114E26346134300D168E180234E0740
:10B83000C008C9081B030643194208D06046C00867
:10B84000184204D163460100D2085E071643F30094
:10B850009946C900720F444D11434B46DE08424BD6
:10B860004F073743CA089D4200D16EE012036D05B1
:10B87000120B6D0D00211203130B0A0D12051A4352
:10B880003B4B2D0513402B435B00E4075B08234330
:10B89000380019003CBC90469946A246AB46F8BD1C
:10B8A0006346134311D0731E002B00D007E18618A6
:10B8B0008642804161444042091801250B0237D578
:10B8C00002257BE73E00614691463500C5E75C46B0
:10B8D000002D00D0E1E00B000343F3D0731C00D136
:10B8E000ACE1214B9F4200D13AE1F343382B00DD1C
:10B8F0006FE11F2B00DD8CE120250E00ED1AAE401C
:10B90000B0460600AA46DE40454635432E00554661
:10B91000D940A8406346451EA8415B1A9C46304367
:10B92000161AB242924163465242991A3D00B4E659
:10B9300007223240002A00D0E4E60B4BF6084F07FE
:10B940003743CA089D4200D090E73B00134300D123
:10B95000A6E180231B031A431203120B024D89E751
:10B9600015000022002785E7FF070000FFFF7FFF8B
:10B97000FFFF0F80002E00D0C7E06B1C5E05760D28
:10B98000012E00DCF0E0C84DAB4200D1B9E08518D3
:10B990000A00854289416244494251180722CE0774
:10B9A0006D082E43490832401D00A9E6BF49ED1A33
:10B9B000114007223240A3E6320028388240002698
:10B9C00086E6300000F052FA203073E663461343F7
:10B9D0005A1E9341C61AB04280414042091A5CE6A1
:10B9E0000E00674606431743002D5ED1002E00D09F
:10B9F000F3E0002F00D11EE15C46614691462CE742
:10BA0000A94FBE427BD01E00F1E610001F3DE8406A
:10BA1000202B03D04021CB1A9A401643731E9E411F
:10BA20000722064332400021002583E7161A6346A9
:10BA3000B2428041591A40420B1A98465C4632E69F
:10BA40001F2E00DDABE02027BB1B9A4663465746FE
:10BA5000BB40994613004F46F3401F433B005746F7
:10BA6000BA40571EBA4113436246F240891898E61D
:10BA70002027BB1B9A4663465746BB409946130096
:10BA80004F46F3401F433B005746BA40571EBA414A
:10BA900013436246F240891A9CE7834B9F425FD072
:10BAA00080252D047342294320E7002E0CD1002F5E
:10BAB00000D1D0E05C46614691467B4DCDE67A4FA1
:10BAC000BE421CD01E0065E6002F18D0C0084E07ED
:10BAD00006438020C9080003014208D06346DC0801
:10BAE000044204D12100DA46D2085E071643F3006F
:10BAF000994601245346C900720F11431C406A4DF8
:10BB0000ABE61D0000220027B4E6002D59D10B0042
:10BB1000034300D1D6E6731C00D1B2E0624B9F42D2
:10BB20001ED0F343382B6FDC1F2B00DD97E0202560
:10BB30000E00ED1AAE40B0460600AA46DE4045466D
:10BB400035432E005546A840D940451EA8418C4497
:10BB50000643B61896429241514261443D0025E6A3
:10BB60003D006146914678E60B000343002D00D06E
:10BB700055E6002BF5D06346134300D16DE68618D9
:10BB80008642804161444042091800220B0200D4E1
:10BB9000D0E6464B01351940B2E5B1465DE63300CB
:10BBA0006746203BDF403B00202E05D04027BF1BCF
:10BBB0006646BE40324390464646721E9641334327
:10BBC000EFE5394B9F42CBD080252D0473422943AA
:10BBD000A8E70843411E8841A2E6002F00D13CE6B9
:10BBE0006346861ACF1AB0429B415B42FB1A9846C5
:10BBF0001B024ED5161A6346B2429241591A52425E
:10BC0000891A5C4600227BE501430E00711E8E41BD
:10BC10009FE71D000E00203DEE40B046202B04D0D3
:10BC20004025EB1A99400843814648464346411E49
:10BC30008841184374E60022002417E6161A63466A
:10BC4000B2429241591A5242891A3D0025E5614695
:10BC50009146154D01E680220024120379E61D006D
:10BC60000E00203DEE40B046202B04D04025EB1ABC
:10BC70009940084381464E464346711E8E411E43FD
:10BC800067E7861896429B4161445B42C9183D00B4
:10BC90008CE547463743CED007224146324049E63D
:10BCA00000273A00E6E5C046FF070000FFFF7FFFE0
:10BCB00070B50C4E0D031C0349005B002D0B490DA4
:10BCC000240B5B0DB14208D0064900208B4203D102
:10BCD00014432000441EA04170BD05430120002DE7
:10BCE000FAD1F1E7FF07000030B5144D0A034B000D
:10BCF000120B5B0DC90F0024AB4211DD104CA342A7
:10BD000010DC8024640322430E4CE41A1F2C0CDD4B
:10BD10000D48C31ADA4013005C42002900D11C0010
:10BD2000200030BD094BCC18FAE7094DE040AC4685
:10BD300063449A4013000343EEE7C046FE0300004D
:10BD40001D0400003304000013040000FFFFFF7F08
:10BD5000EDFBFFFF70B500282DD0C317C5185D405F
:10BD6000C40F280000F082F8154B1B1A5B055B0D11
:10BD70000A2815DD0B38854000222D032D0B0021EC
:10BD800010002D030A0D2D0B12052A430D4D1B0526
:10BD90002A4013435B00E4075B082343190070BD8E
:10BDA00002002900153291400A000B21081AC540F3
:10BDB0002D032D0BE3E70024002300250022DEE7FE
:10BDC0001E040000FFFF0F804100090E4B1C70B5E0
:10BDD000DBB24602750AC40F012B14DDE0239B0081
:10BDE0006D07360BCB1800210A0D280012051C4DDB
:10BDF00032435B052A405B0813435B00E4075B08A2
:10BE00002343190070BD002914D1002D1ED0280035
:10BE100000F02CF80A281CDC0B232A001B1ADA403D
:10BE2000030015339D400F4B12031B1A5B05160BC5
:10BE30005B0DD8E7002D06D0320B802636036D0748
:10BE40001643094BCFE7084B0026CCE7002300261A
:10BE5000C9E703002A000B3B9A400025E3E7C046F0
:10BE6000FFFF0F8089030000FF0700001C21012352
:10BE70001B04984201D3000C10391B0A984201D3CD
:10BE8000000A08391B09984201D30009043902A2AB
:10BE9000105C40187047C046040302020101010112
:10BEA000000000000000000030B51C00094B050038
:10BEB0001B6885B0D868084B002A01D1074B1A00CF
:10BEC0000292019300912B002200054900F026F810
:10BED00000F0A6FD8C00002030EE000023DB000007
:10BEE0003DEE0000014B18687047C0468C000020F2
:10BEF000084B10B50400002B02D0002100E000BF69
:10BF0000054B1868836A002B00D09847200001F089
:10BF10005DFBC046000000006CEE00000EB403B5EF
:10BF2000010003AB044804CB0068019300F076F8ED
:10BF300002B008BC03B018478C00002070B5002682
:10BF40000C4D0D4C641BA410A64209D1002601F033
:10BF50003FFB0A4D0A4C641BA410A64205D170BDDC
:10BF6000B300EB5898470136EEE7B300EB5898471B
:10BF70000136F2E75C0200205C0200205C02002037
:10BF80006C020020002310B59A4200D110BDCC5C99
:10BF9000C4540133F8E710B5884202D98B1898428F
:10BFA00003D3002307E08B5C8354013AFBD210BD1E
:10BFB000CC5CC45401339A42FAD1F8E7030012185A
:10BFC000934200D1704719700133F9E7936810B5B7
:10BFD000013B9360002B04DA9469A34207DB0A2932
:10BFE00005D01368581C10601970080010BD00F0CF
:10BFF0004BFC0100F9E7F8B506000F001400D51856
:10C00000AC4201D1002007E021783A003000FFF770
:10C01000DDFF0134431CF3D1F8BD0000F0B59FB043
:10C0200002900F0016000593002805D08369049341
:10C03000002B01D100F0F4FD7B4B9F425BD1029BB2
:10C040005F68BB891B0762D53B69002B5FD000236B
:10C0500006AC6361203363761033A37635002B780A
:10C06000002B01D0252B5CD1AB1B04930CD03200EC
:10C0700039000298FFF7BFFF431C00D1C4E062699A
:10C08000049B9446634463612B78002B00D1BBE092
:10C09000012200235242626002A9543252186E1CDF
:10C0A0002360E360A3601370A365317805225F48C5
:10C0B00000F0D4FE751C002835D12268D30604D5C3
:10C0C000532302A95B1820211970130704D55323A9
:10C0D00002A95B182B21197033782A2B2CD035003C
:10C0E00000210A20E3682A786E1C303A092A64D9B4
:10C0F00000292ED026E04E4B9F4202D1029B9F6822
:10C100009FE74C4B9F429CD1029BDF6899E7390027
:10C11000029800F00FFC002899D0012040421FB087
:10C12000F0BD01359BE7414B2268C01A01238340D3
:10C13000134323602E00B8E7059B191D1B6805916A
:10C14000002B01DB099304E05B42E360022313430D
:10C1500023602B782E2B0AD16B782A2B35D1059BA7
:10C1600002351A1D1B680592002B2BDB0793324EFC
:10C1700029780322300000F071FE002806D0402309
:10C18000801B8340226801351343236029780622EF
:10C190002A486E1C217600F061FE00283AD0284B18
:10C1A000002B25D10722059B0733934308330593C2
:10C1B0006369039A9B18636150E7434301219B180D
:10C1C000350090E701235B42D0E700230A201A00E4
:10C1D0000135636029786E1C3039092903D9002B99
:10C1E000C5D00792C3E74243012352183500F1E757
:10C1F00005AB00933A00134B2100029800E000BF0A
:10C200000390039B0133D3D1BB895B0600D584E740
:10C210000B9884E705AB00933A000A4B2100029883
:10C2200000F080F8ECE7C046C4EE000070EE0000BD
:10C23000E4EE0000A4EE000076EE00007AEE0000CE
:10C2400000000000F7BF0000F7B5150001938A68F1
:10C250000B6900900C00934200DA130022002B605F
:10C2600043321278002A01D001332B6023689B06E9
:10C2700002D52B6802332B60062723681F4027D086
:10C28000230043331B785A1E93412268920630D410
:10C290002200019943320098089EB047431C25D0E4
:10C2A000062320682A68E16803400025042B03D197
:10C2B0008D1AEB43DB171D40A3682269934201DD11
:10C2C0009B1AED180027BD4220D1002010E0013755
:10C2D000E3682A689B1ABB42D2DD2200012319328F
:10C2E00001990098089EB047431CF0D101204042BC
:10C2F000FEBD3020E1184331087021005A1C453141
:10C300000978A218433202331170C1E722000123D9
:10C310001A3201990098089EB047431CE6D00137B5
:10C32000D1E70000F0B589B004920A0043320593CA
:10C33000039002920A7E0C000E9B6E2A00D186E0CA
:10C340001FD8632A33D008D8002A00D18CE0582A9D
:10C350004DD0250042352A7030E0642A01D0692A88
:10C36000F7D1196825680A1D280629D508681A60BA
:10C37000002803DA2D23029A404213706B4E0A27DD
:10C380004FE0732A74D008D86F2A1FD0702AE0D1EA
:10C39000202209680A43226003E0752A16D0782A11
:10C3A000D7D12200782145321170614E22E025005C
:10C3B0001A684235111D196013682B70012365E05E
:10C3C00008681A606906D3D500B2D1E719682568F4
:10C3D000081D186008682E0605D5544E08276F2AD8
:10C3E0001BD00A2719E06D06F7D580B2F5E7453175
:10C3F0004E4E0A7018682268011D00681960150603
:10C4000021D5D30702D520231A4322601027002804
:10C4100003D1202322689A43226023000022433361
:10C420001A706368A360002B58DB042221689143D3
:10C430002160002854D1029D002B5AD0250033786A
:10C4400042352B7055E05506DBD580B2D9E71A6826
:10C450000D68101D4969186013682E0601D5196012
:10C4600002E06D06FBD519800023029D23614FE099
:10C470001A68111D1960156800216268280000F013
:10C48000EDFC002801D0401B60606368236100233D
:10C49000029A13703CE023692A0004990398059DD1
:10C4A000A847431C3ED023689B0715D4079BE06830
:10C4B000984239DA180037E0220001231932049932
:10C4C0000398059EB047431C2CD00135E368079ABA
:10C4D0009B1AAB42F0DCE9E70025F7E70028ADD076
:10C4E000029D3900FDF722FC735C013D2B70002892
:10C4F000F7D1082F09D12368DB0706D563682269C5
:10C50000934202DC3023013D2B70029B5B1B2361B5
:10C51000059B07AA00932100049B0398FFF794FE54
:10C52000431CB8D10120404209B0F0BD81EE0000AB
:10C5300092EE00000D4B70B51C680500A36B002B3C
:10C540000FD1182000F06EFC094BA0630360094B6B
:10C5500001224360084B83600B2383810023026127
:10C5600043610022A36B1D615A6170BD8C000020E5
:10C570000E33CDAB34126DE6ECDE0500124B10B578
:10C580001C68A36B002B0FD1182000F04BFC0F4B45
:10C59000A06303600E4B012243600E4B83600B23AC
:10C5A0008381002302614361A46B0B4A20696169A6
:10C5B0000A4BFDF7F7FC0122002380185941206146
:10C5C00061614800400810BD8C0000200E33CDABE7
:10C5D00034126DE6ECDE05002D7F954C2DF451589C
:10C5E0000CB430B5164B9DB00C1E1D6808DA8B23B9
:10C5F00001202B6040421DB030BC08BC02B018477F
:10C60000822302A99B008B810023029008619C4237
:10C6100000D0631E8B604B6101235B42CB81209A6B
:10C6200021AB2800019300F055FD431C01DA8B2358
:10C630002B60002CDFD00023029A1370DBE7C0468A
:10C640008C0000200EB400B50B499CB01DAB0290CD
:10C650000690079104910948094904CB05910068A7
:10C6600002A9019300F036FD0023029A13701CB05A
:10C6700008BC03B01847C046FFFFFF7F8C000020B6
:10C680000802FFFF020010B51378541C002B05D1DF
:10C69000CC5CD4540133002CFAD110BD2200F3E756
:10C6A000C9B20378002B04D08B4200D1704701300F
:10C6B000F7E74B42594149420840F7E702780B78C7
:10C6C000002A03D0013001319A42F7D0D01A7047C6
:10C6D0000023C25C0133002AFBD1581E704700239F
:10C6E00030B59A420AD0013AC45CCD5CAC4204D168
:10C6F000934202D00133002CF6D1631B180030BDE9
:10C7000030B50500002A00D130BD0C78013A6B1C11
:10C710002C700131002C05D19A189A42F4D01C706B
:10C720000133FAE71D00EDE710B50378002B0FD1B8
:10C730000B785A4253415B42184010BD0023CA5C3B
:10C74000002AFAD0C45C944201D10133F7E70130EA
:10C750000378002BF2D11800EFE70000F0B51F00BE
:10C760000E0087B00590019102920C98347800F089
:10C77000EAFA082200194378751C134036D12D2C93
:10C7800036D1B51C74780126002F62D0102F09D144
:10C79000302C07D120222B789343582B54D11027CB
:10C7A0006C7802352D4B3900F31818000393FDF710
:10C7B000BDFA049101210023494202008C46180071
:10C7C0002100303909291AD80C00A74223DD591C51
:10C7D00009D06346824206D302D10499A14202DB0A
:10C7E0000123784320182C780135E9E72E00BCE7B7
:10C7F0002B2C01D01E00C7E7B51C7478FAE7210086
:10C800004139192901D8373CDFE72100613919295D
:10C8100001D8573CD9E75A1C08D1059A2333136035
:10C82000029B0398002B09D107B0F0BD002E00D069
:10C830004042029A002AF7D0002B01D06B1E0193D0
:10C84000029B019A1A60EFE73024002FAAD1082733
:10C85000A8E7302C9ED00A27A4E7C046FFFFFF7F41
:10C8600037B51300064A05001068046A002C00D191
:10C87000044C0A0000942900FFF770FF3EBDC0463B
:10C880008C000020F0000020F8B505000E00140018
:10C89000002804D08369002B01D100F0C1F9224B9C
:10C8A0009C422DD16C68A369A360A3891B0731D575
:10C8B0002369002B2ED023682269F7B2981A636986
:10C8C000F6B2834205DC2100280000F03BF9002885
:10C8D00026D1A3680130013BA36023685A1C226063
:10C8E0001F706369834204D0A389DB071AD50A2E1F
:10C8F00018D12100280000F025F9002812D00FE0FF
:10C900000A4B9C4201D1AC68CDE7094B9C42CAD18D
:10C91000EC68C8E72100280000F00CF80028CAD015
:10C92000012676423000F8BDC4EE0000E4EE0000BF
:10C93000A4EE0000364B70B51D6806000C00002DFB
:10C9400005D0AB69002B02D1280000F069F9314B0A
:10C950009C420FD16C680C23E25E93B219072DD470
:10C96000D90611D409230120336037331343A3813F
:10C97000404270BD284B9C4201D1AC68EBE7274B8D
:10C980009C42E8D1EC68E6E75B0713D5616B0029B0
:10C9900008D023004433994202D0300000F06AFAF4
:10C9A000002363632422A3899343A381002363604C
:10C9B000236923600823A2891343A3812369002BE1
:10C9C0000BD1A0218022A389890092000B409342C1
:10C9D00003D02100300000F0E1F90123A2891340C7
:10C9E00011D00023A36063695B42A3610020236927
:10C9F0008342BED10C23E25E1306BAD54023134313
:10CA0000A3810138B5E7920700D46369A360EDE71D
:10CA10008C000020C4EE0000E4EE0000A4EE000054
:10CA200010B5062000F090FC012000F0CFFD0000C2
:10CA3000F7B58A8905000C00130760D44B68002BFA
:10CA400004DC0B6C002B01DC0020FEBDE76A002F2C
:10CA5000FAD000232E682B6080235B01216A1A40E4
:10CA600034D0606DA3895B0706D56368C01A636B19
:10CA7000002B01D0236CC01A0200216A0023280079
:10CA8000E76AB847A189431C06D12B681D2B30D813
:10CA90002B4ADA40D3072CD5002363602369236037
:10CAA000CB0405D5431C02D12B68002B00D1606557
:10CAB000616B2E600029C7D023004433994202D015
:10CAC000280000F0D7F900206063BEE701232800AA
:10CAD000B847431CC6D12B68002BC3D01D2B01D0F7
:10CAE000162B01D12E60AFE74023A2891343A38107
:10CAF000ABE740230B430120A3814042A5E70F6928
:10CB0000002FA1D00B680F60DB1B0193002392075D
:10CB100000D14B69A360019B002B00DC94E7019BD3
:10CB20003A00216A2800A66AB047002803DC4023A7
:10CB3000A2891343DFE7019B3F181B1A0193EAE721
:10CB4000010040200B6970B505000C00002B01D1DD
:10CB5000002070BD002804D08369002B01D100F0B3
:10CB60005FF80B4B9C4209D16C680C22A35E002B32
:10CB7000EED021002800FFF75BFFEAE7054B9C425F
:10CB800001D1AC68F1E7044B9C42EED1EC68ECE7D4
:10CB9000C4EE0000E4EE0000A4EE0000002310B597
:10CBA000040003604360836081814366C281036146
:10CBB00043618361190008225C30FFF7FFF9054BE0
:10CBC00024626362044BA362044BE362044B23635D
:10CBD00010BDC04689D30000B1D30000E9D30000E6
:10CBE00015D4000010B5024900F08CF810BDC04605
:10CBF00045CB000070B568254A1E55430E0029003C
:10CC0000743100F081F9041E08D000212A0001606F
:10CC100046600C30A0606832FFF7D0F9200070BD8C
:10CC2000836913B50400002B28D18364C3640365B2
:10CC3000134B144A1B6882620193984201D101236D
:10CC40008361200000F020F86060200000F01CF8F4
:10CC5000A060200000F018F80022E0600421606865
:10CC6000FFF79CFF01220921A068FFF797FF02222E
:10CC70001221E068FFF792FF0123A36113BDC046B4
:10CC80006CEE0000E5CB0000F8B51C4B07001E68F9
:10CC9000B369002B02D13000FFF7C2FF4836B468F9
:10CCA0007368013B04D53368002B07D03668F6E77C
:10CCB0000C22A55E002D0DD06834F2E70421380067
:10CCC000FFF798FF30600028F0D10C2304003B6090
:10CCD0002000F8BD20000A4B656625606560A560F0
:10CCE000E36025616561A561082229005C30FFF7DA
:10CCF00065F96563A563A564E564E9E76CEE00008A
:10CD00000100FFFFF7B50400070000260191483439
:10CD1000002C01D13000FEBD6368A5680093009B24
:10CD2000013B009301D52468F2E7AB89012B08D9B8
:10CD30000E22AB5E013304D029003800019B9847D6
:10CD400006436835EBE7EC300068704770B50E00BD
:10CD50001D000E23C95E96B01400002907DA0023D7
:10CD60002B60B3891B0611D48023DB000FE06A46D9
:10CD700000F088FB0028F2DBF022019B1202134036
:10CD8000054A9B185A4253412B60EDE7402300208F
:10CD9000236016B070BDC04600E0FFFFF7B5022665
:10CDA0008B8905000C00334206D0230047332360F3
:10CDB000236101236361F7BD01AB6A46FFF7C6FF3C
:10CDC00000990700280000F09FF8002808D10C22E5
:10CDD000A35E9A05EFD4032293431E43A681E4E7A2
:10CDE0000F4BAB628023A28920601343A381009B79
:10CDF00020616361019B002B0DD00E23E15E2800B2
:10CE000000F052FB002806D00322A38993431A00A6
:10CE100001231343A381A0893843A081CBE7C046F7
:10CE2000E5CB000010B5034B0100186800F06CF86A
:10CE300010BDC0468C00002082B0002900D101A99D
:10CE4000101E06D0002B06D013780B601078431EFE
:10CE5000984102B0704702204042FAE7C9B28218F6
:10CE6000904201D10020704703788B42FBD0013003
:10CE7000F6E7000070B50500002910D00C1F2368EC
:10CE8000002B00DAE418280000F034FB1D4A136878
:10CE9000002B05D163601460280000F02CFB70BDEE
:10CEA000A34209D9216860188342F3D118685B68EE
:10CEB00041182160EEE713005A68002A01D0A2420F
:10CEC000F9D919685818A0420BD1206809185818C8
:10CED00019608242E0D110685268411819605A60A6
:10CEE000DAE7A04202D90C232B60D5E7216860184D
:10CEF000824203D1106852684118216062605C6010
:10CF0000CAE7C0463C1C0020032370B5CD1C9D43DE
:10CF1000083506000C2D1ED20C25A9421DD8300064
:10CF200000F0E8FA254A14682100002919D1244CA0
:10CF30002368002B03D1300000F0CAF920602900DB
:10CF4000300000F0C5F9431C2BD10C2330003360B6
:10CF500000F0D1FA03E0002DDFDA0C23336000206B
:10CF600070BD0B685B1B19D40B2B03D90B60CC185D
:10CF7000256003E04B688C420DD11360300000F057
:10CF8000BAFA200007220B30231D9043C31AE7D0C2
:10CF90005A42E250E4E763600C00EFE70C00496896
:10CFA000C3E70323C41C9C43A042E1D0211A3000F4
:10CFB00000F08EF9431CDBD1C7E7C0463C1C0020C3
:10CFC000401C0020F8B507000D001600002905D10F
:10CFD0001100FFF799FF04002000F8BD002A03D1DB
:10CFE000FFF748FF3400F7E700F086FA2C00B04264
:10CFF000F2D231003800FFF787FF041EECD0290081
:10D000003200FEF7BFFF29003800FFF733FFE3E7E8
:10D01000F0B58E6885B007000C00039201939E4224
:10D020003CD890238A89DB001A4234D00325096951
:10D0300023685B1A0293636902985D43EB0F5D19E5
:10D04000019B6D1001331B18AB4200D91D00530525
:10D0500032D529003800FFF757FF061E09D10C23EF
:10D060003B6040230120A28940421343A38105B0C5
:10D07000F0BD029A2169FEF785FFA389144A1A4080
:10D0800080231343A381029B2661F6182660656105
:10D09000019EED1AA560019B9E4200D9019E3200BF
:10D0A00003992068FEF777FFA36800209B1BA3600D
:10D0B00023689E192660DAE72A003800FFF782FF0E
:10D0C000061EE0D121693800FFF7D4FEC7E7C0464D
:10D0D0007FFBFFFFF0B59FB0029005938B890F0097
:10D0E00016001B0611D50B69002B0ED14021FFF74E
:10D0F0000BFF38603861002805D10C23029A0138F3
:10D1000013601FB0F0BD40237B61002306AC636158
:10D11000203363761033A37635002B78002B01D0B3
:10D12000252B46D1AB1B04930CD03200390002985A
:10D13000FFF76EFF431C00D1AEE06269049B94468A
:10D14000634463612B78002B00D1A5E0012200230A
:10D150005242626002A9543252186E1C2360E3608E
:10D16000A3601370A365317805225448FFF776FE5B
:10D17000751C00281FD12268D30604D5532302A9A9
:10D180005B1820211970130704D5532302A95B18DB
:10D190002B21197033782A2B16D0350000210A2054
:10D1A000E3682A786E1C303A092A4ED9002918D033
:10D1B00010E00135B1E7414B2268C01A01238340DA
:10D1C000134323602E00CEE7059B191D1B680591B4
:10D1D000002B01DB099304E05B42E360022313436D
:10D1E00023602B782E2B0AD16B782A2B35D1059B07
:10D1F00002351A1D1B680592002B2BDB0793304E5E
:10D20000297803223000FFF729FE002806D04023AA
:10D21000801B83402268013513432360297806224E
:10D2200028486E1C2176FFF719FE00283CD0264BBB
:10D23000002B25D10722059B073393430833059321
:10D240006369039A9B18636166E7434301219B1856
:10D250003500A6E701235B42D0E700230A201A002D
:10D260000135636029786E1C3039092903D9002BF8
:10D27000C5D00792C3E74243012352183500F1E7B6
:10D2800005AB00933A00114B2100029800E000BF6B
:10D290000390039B0133D3D1BB890B985B0600D469
:10D2A0002FE7012040422CE705AB00933A00074BE3
:10D2B00021000298FFF736F8EAE7C04670EE00005A
:10D2C00076EE00007AEE00000000000011D00000B1
:10D2D000002370B5064C05000800236000F060F9DB
:10D2E000431C03D12368002B00D02B6070BDC046C7
:10D2F000D02F002070B504000D001F2904D916237B
:10D3000003600120404270BD436C002B04D08A00B2
:10D310009B181A68002A08D1200000F031F82A0072
:10D320000100200000F01AF8EDE70020012AEAD001
:10D33000511C03D1162301302360E4E700242800A8
:10D340001C6090472000DEE710B5034B0100186811
:10D35000FFF7D0FF10BDC0468C000020002370B541
:10D36000064C050008001100236000F001F9431C81
:10D3700003D12368002B00D02B6070BDD02F00207C
:10D3800010B500F0E5F810BD70B50C000E25495F32
:10D3900000F0BAF8002803DB636D1B18636570BDED
:10D3A000A389024A1340A381F9E7C046FFEFFFFFBC
:10D3B000F8B51F008B8905000C001600DB0505D5AC
:10D3C0000E23C95E0022022300F080F8A389054ADB
:10D3D00028001340A38132000E23E15E3B0000F0E1
:10D3E0002BF8F8BDFFEFFFFF70B50C000E25495F6D
:10D3F00000F06CF8A389421C03D1054A1340A381B5
:10D4000070BD802252011343A3816065F8E7C046D6
:10D41000FFEFFFFF10B50E23C95E00F021F810BD2D
:10D420000B1E04D0FF2A04D98A2303608B3B18000B
:10D4300070470A700123FAE770B505000800110073
:10D440000022064C22601A0000F0B8F8431C03D1F9
:10D450002368002B00D02B6070BDC046D02F002069
:10D46000002370B5064C05000800236000F060F84A
:10D47000431C03D12368002B00D02B6070BDC04635
:10D48000D02F0020002370B5064C050008001100C5
:10D49000236000F055F8431C03D12368002B00D013
:10D4A0002B6070BDD02F0020002370B5064C050006
:10D4B0000800236000F054F8431C03D12368002BBC
:10D4C00000D02B6070BDC046D02F002070B5050085
:10D4D000080011000022064C22601A0000F050F8EB
:10D4E000431C03D12368002B00D02B6070BDC046C5
:10D4F000D02F0020704770470B1F1B68181F002B90
:10D5000001DA0B58C018704770B50500080011000B
:10D510000022064C22601A0000F03AF8431C03D1A6
:10D520002368002B00D02B6070BDC046D02F002098
:10D5300058220120014B40421A607047D02F002032
:10D5400058220120014B40421A607047D02F002022
:10D5500058220120014B40421A607047D02F002012
:10D560005822024B00201A607047C046D02F00207E
:10D5700058220120014B40421A607047D02F0020F2
:10D5800058220120014B40421A607047D02F0020E2
:10D5900058220120014B40421A607047D02F0020D2
:10D5A000044A1368002B00D1034B181810601800B0
:10D5B0007047C046441C0020D82F0020582201206C
:10D5C000014B40421A607047D02F0020FEE7C04652
:10D5D000F8B5C046F8BC08BC9E467047F8B5C046D2
:10D5E000F8BC08BC9E46704764617461000000008E
:10D5F0007CD60000EF01000085D60000E3020000A9
:10D600008DD600009D0A000094D60000AD0B0000EE
:10D6100099D60000090500009FD600008906000089
:10D62000AAD6000053030000AFD60000050E00008C
:10D63000BBD600001F020000C5D60000690900002B
:10D64000D3D60000310A0000E0D600001508000023
:10D65000ECD600004906000072616E646F6D0061D7
:10D660006C6C006C6173740066616C73650074723D
:10D67000756500252E3135732E2E2E006D616B657C
:10D680004C697374006164644C6173740064656C0C
:10D69000657465006A6F696E0073706C697400630D
:10D6A0006F707946726F6D546F0066696E64006AC0
:10D6B0006F696E537472696E677300756E69636F1C
:10D6C0006465417400756E69636F64655374726953
:10D6D0006E67006E65774279746541727261790098
:10D6E0006173427974654172726179006672656531
:10D6F0004D656D6F727900005DD7000091120000DA
:10D7000062D70000AF1200008DD60000B3120000F7
:10D7100068D700009512000072D70000B712000011
:10D720007BD70000BB12000085D70000BF120000AD
:10D7300090D70000C31200009CD70000991200008F
:10D74000A5D70000A7120000AFD700009D1200006F
:10D75000BAD70000AB12000066696C65006F706597
:10D760006E00636C6F736500656E644F6646696C2E
:10D770006500726561644C696E6500726561644242
:10D780007974657300617070656E644C696E6500D4
:10D79000617070656E6442797465730066696C656A
:10D7A00053697A650073746172744C697374006EA6
:10D7B000657874496E4C6973740073797374656D20
:10D7C000496E666F000000007C1600008C16000099
:10D7D000A6160000221700005A1700008E1700003E
:10D7E000C6170000EC170000301800007218000087
:10D7F000C81800000C1900006E190000B8190000CC
:10D80000DE190000161A00005C1A0000821A0000DF
:10D81000B01A0000DE1A0000B6310000961B0000AE
:10D82000681C0000DE1C00004E1D00009A1D000058
:10D83000BA1D0000DC1D0000341F0000781F00002E
:10D84000F01F00001E200000502000008220000079
:10D85000022100006A210000C621000024220000ED
:10D86000962200000823000064230000BE2300006D
:10D87000F4230000442400008A240000D224000085
:10D88000262500007A250000B82500002426000087
:10D890005A260000A2260000EA26000032270000D7
:10D8A0006C270000B427000004280000662900004F
:10D8B000B01A0000161A00006C2800007C16000048
:10D8C000A2280000CE280000042900003029000012
:10D8D0007C1600007C1600007C1600007C16000000
:10D8E000E2290000242A00006A2A0000BA2A000067
:10D8F000E62A00005E2B0000B02B0000142C000074
:10D900007C1600007C160000382C0000682C0000FB
:10D91000982C0000CE2C0000F82C00002E2D0000CA
:10D92000582D0000802D0000A82D0000D82D0000EB
:10D93000082E0000322E00005C2E00008C2E00000D
:10D94000B62E00007C1600007C1600007C1600003D
:10D950007C1600007C160000E62E0000122F00004E
:10D960003E2F00006A2F0000962F0000CC2F0000F1
:10D970000C3000004230000078300000A43000007D
:10D98000D0300000063100007C1600007C1600003C
:10D990007C1600007C1600007C1600007C1600003F
:10D9A0007C1600007C1600007C1600007C1600002F
:10D9B0007C1600007C16000032310000323100007D
:10D9C0000C320000423200005B2564206974656DF2
:10D9D000206C6973745D0028256420627974657316
:10D9E0002900286F626A65637420747970653A2033
:10D9F00025642900537461636B20756E64657266DB
:10DA00006C6F7700626F6F6C65616E006E756D6232
:10DA1000657200737472696E67006C69737400627A
:10DA2000797465206172726179000000070000005E
:10DA3000030000008EDA00006533000096DA000073
:10DA4000153400009FDA000087350000A8DA0000D6
:10DA500069330000B1DA00008B350000B9DA00004C
:10DA600075350000C2DA0000A53400000000000097
:10DA7000010000000200000003000000040000009C
:10DA80000A0000006D6963726F3A62697400686130
:10DA900073546F6E6500706C6179546F6E650068C9
:10DAA0006173536572766F00736574536572766F38
:10DAB00000646163496E69740064616357726974DC
:10DAC0006500737175617265576176650047432023
:10DAD000746F6F6B2025642075736563733B2066DC
:10DAE00072656520256420776F726473003C496E0F
:10DAF00074656765723E003C4C6973743E003C4F30
:10DB0000626A6563743E003C427974654172726179
:10DB1000793E000D0A564D2050616E69633A20250A
:10DB2000730D0A006D6973630000000061DB000083
:10DB3000794200006ADB0000094200006EDB000051
:10DB40005D41000076DB00000341000080DB000047
:10DB5000994000008CDB00009B3F00006E756C6CF0
:10DB600000686578546F496E740073696E006A735B
:10DB70006F6E476574006A736F6E436F756E7400E5
:10DB80006A736F6E56616C75654174006A736F6E6F
:10DB90004B6579417400000024DC0000E542000080
:10DBA0002CDC0000E942000036DC000007430000E6
:10DBB0003FDC0000114300004ADC00001B43000072
:10DBC00056DC00002543000064DC00002F43000009
:10DBD0006CDC00003943000072DC000043430000AD
:10DBE00087DC00004D4300009CDC00005743000030
:10DBF000A8DC000061430000B8DC00006B430000BB
:10DC0000C4DC000075430000D1DC00007F4300004D
:10DC1000E0DC0000F3420000F3DC0000FD42000005
:10DC20006E65740068617357694669007374617248
:10DC300074576946690073746F7057694669007755
:10DC4000696669537461747573006D7949504164F4
:10DC500064726573730073746172745353494473CF
:10DC600063616E0067657453534944006D794D419B
:10DC700043006874747053657276657247657452B8
:10DC800065717565737400726573706F6E64546F3F
:10DC9000487474705265717565737400687474703B
:10DCA000436F6E6E65637400687474704973436F7C
:10DCB0006E6E656374656400687474705265717526
:10DCC0006573740068747470526573706F6E7365F9
:10DCD00000776562536F636B65745374617274008F
:10DCE000776562536F636B65744C617374457665D9
:10DCF0006E7400776562536F636B657453656E6411
:10DD0000546F436C69656E74001A1B1C030406078C
:10DD1000090A171819000000000008080800080A7E
:10DD20004A4000000A5FEA5FEA0ED92ED36E19322C
:10DD30004489330C924C924D080800000004880876
:10DD400008040804848488000A448A4000048EC4BD
:10DD500080000000048800000EC0000000000800E1
:10DD600001224488100C9252524C048C84848E1CE4
:10DD7000824C901E1EC244924C06CA525FE21FF0B3
:10DD80001EC13E02448ED12E1FE24488100ED12EB9
:10DD9000D12E0ED12EC48800080008000004800493
:10DDA000880244880482000EC00EC00804824488A1
:10DDB0000ED126C0040ED135B36C0C925ED2521C2B
:10DDC000925C925C0ED010100E1C9252525C1ED0CF
:10DDD0001C901E1ED01C90100ED013712E12525E7D
:10DDE000D2521C8808081C1FE242524C125498144C
:10DDF00092101010101E113B75B131113935B371ED
:10DE00000C9252524C1C925C90100C92524C861CFC
:10DE1000925C92510ED00C825C1FE4848484125276
:10DE200052524C1131312A44113135BB7112524CCE
:10DE30009252112A4484841EC488101E0EC80808F9
:10DE40000E10080482410EC242424E048A40000075
:10DE5000000000001F0804800000000ED2524F1086
:10DE6000101C925C000ED0100E02424ED24E0C924C
:10DE70005C900E06C81C88080ED24EC24C10101CB6
:10DE800092520800080808024002424C10149814EC
:10DE9000920808080806001B75B131001C92525206
:10DEA000000C92524C001C925C90000ED24EC200AC
:10DEB0000ED010100006C8049808080EC8070012FB
:10DEC00052524F0011312A4400113135BB00124C1F
:10DED0008C9200112A4498001EC4881E06C48C84AB
:10DEE00086080808080818080C881800000C8360C9
:10DEF000000000000100000002000000030000001C
:10DF000004000000050000000600000007000000FB
:10DF100008000000090000000A0000000B000000DB
:10DF20000C0000000D0000000E0000000F000000BB
:10DF30001000000012000000140000001600000095
:10DF4000180000001A0000001C0000001E00000065
:10DF5000200000002300000026000000290000002F
:10DF60002C0000002F0000003200000036000000EE
:10DF70003A0000003E0000004200000046000000A1
:10DF80004B00000050000000550000005A00000047
:10DF900061000000680000006F00000076000000D3
:10DFA0007D000000840000008B0000009200000053
:10DFB00099000000A0000000A7000000AE000000D3
:10DFC000B5000000BC000000C3000000CA00000053
:10DFD000D1000000D8000000DF000000E6000000D3
:10DFE000ED000000F4000000FB000000FF00000056
:10DFF00040E00000A14300004BE000003D4900006C
:10E0000055E000006545000062E00000AD470000FB
:10E0100069E00000FD47000072E000004D4800008C
:10E020007EE00000454700008FE00000D54500007D
:10E030009CE00000D5460000646973706C61790053
:10E040006C696768744C6576656C006D62446973D1
:10E05000706C6179006D62446973706C61794F66B0
:10E0600066006D62506C6F74006D62556E706C6FFF
:10E0700074006D62447261775368617065006D620F
:10E080005368617065466F724C6574746572006E9A
:10E09000656F506978656C53656E64006E656F508E
:10E0A0006978656C53657450696E004E6F742065B5
:10E0B0006E6F75676820726F6F6D206576656E2074
:10E0C000616674657220636F6D70616374696F6EF1
:10E0D00000436F6D70616374656420466C617368A2
:10E0E00020636F64652073746F72650A2564206213
:10E0F0007974657320757365642028256425252946
:10E10000206F6620256400426164207265636F722F
:10E110006420666F756E6420647572696E6720692D
:10E120006E697469616C697A6174696F6E002564E7
:10E130002025642025642028256420776F7264736D
:10E1400029002564207265636F7264732C20256436
:10E1500020776F7264732C206D61784944202564A8
:10E160002C20636F6D70616374696F6E20637963D7
:10E170006C657320256400526573746F726564204A
:10E1800025642073637269707473005374617274D0
:10E19000656400726164696F000000002CE2000099
:10E1A0000D53000039E20000A955000049E20000CB
:10E1B0002955000057E200003D57000062E20000D0
:10E1C0003553000072E20000BD53000086E20000FB
:10E1D000A553000095E200001F590000A1E20000D5
:10E1E0009D580000AAE2000041580000B5E200007E
:10E1F00089570000C0E20000C5570000C9E20000D6
:10E20000F9570000D2E2000045530000E1E20000AF
:10E2100025530000EAE20000555300006E6F6E6562
:10E22000006F74686572007061697200646973617F
:10E23000626C65526164696F006D657373616765D7
:10E240005265636569766564007061636B657452DD
:10E25000656365697665007061636B657453656EAF
:10E2600064007265636569766564496E74656765A7
:10E27000720072656365697665644D657373616785
:10E280006554797065007265636569766564537479
:10E2900072696E670073656E64496E746567657256
:10E2A0000073656E64506169720073656E645374C7
:10E2B00072696E67007365744368616E6E656C00A9
:10E2C00073657447726F757000736574506F77650E
:10E2D00072007369676E616C537472656E677468FF
:10E2E000006465766963654944006C6173744D65CB
:10E2F0007373616765494400556E6B6E6F776E206E
:10E300007072696D6974697665205B25733A25734F
:10E310005D00000000000000963007772C610EEED3
:10E32000BA51099919C46D078FF46A7035A563E96C
:10E33000A395649E3288DB0EA4B8DC791EE9D5E093
:10E3400088D9D2972B4CB609BD7CB17E072DB8E792
:10E35000911DBF906410B71DF220B06A4871B9F3E7
:10E36000DE41BE847DD4DA1AEBE4DD6D51B5D4F420
:10E37000C785D38356986C13C0A86B647AF962FD85
:10E38000ECC9658A4F5C0114D96C0663633D0FFAD2
:10E39000F50D088DC8206E3B5E10694CE44160D5D8
:10E3A000727167A2D1E4033C47D4044BFD850DD2C2
:10E3B0006BB50AA5FAA8B5356C98B242D6C9BBDBD5
:10E3C00040F9BCACE36CD832755CDF45CF0DD6DCD0
:10E3D000593DD1ABAC30D9263A00DE518051D7C877
:10E3E0001661D0BFB5F4B42123C4B3569995BACF02
:10E3F0000FA5BDB89EB802280888055FB2D90CC623
:10E4000024E90BB1877C6F2F114C6858AB1D61C19B
:10E410003D2D66B69041DC760671DB01BC20D298BA
:10E420002A10D5EF8985B1711FB5B606A5E4BF9F47
:10E4300033D4B8E8A2C9077834F9000F8EA809963A
:10E4400018980EE1BB0D6A7F2D3D6D08976C6491A5
:10E45000015C63E6F4516B6B62616C1CD8306585BE
:10E460004E0062F2ED95066C7BA5011BC1F408829B
:10E4700057C40FF5C6D9B06550E9B712EAB8BE8BDC
:10E480007C88B9FCDF1DDD62492DDA15F37CD38C65
:10E49000654CD4FB5861B24DCE51B53A7400BCA363
:10E4A000E230BBD441A5DF4AD795D83D6DC4D1A495
:10E4B000FBF4D6D36AE96943FCD96E34468867AD6C
:10E4C000D0B860DA732D0444E51D03335F4C0AAA0B
:10E4D000C97C0DDD3C710550AA41022710100BBE0E
:10E4E00086200CC925B56857B3856F2009D466B955
:10E4F0009FE461CE0EF9DE5E98C9D9292298D0B08A
:10E50000B4A8D7C7173DB359810DB42E3B5CBDB736
:10E51000AD6CBAC02083B8EDB6B3BF9A0CE2B603B7
:10E520009AD2B1743947D5EAAF77D29D1526DB046C
:10E530008316DC73120B63E3843B64943E6A6D0DB7
:10E54000A85A6A7A0BCF0EE49DFF099327AE000A02
:10E55000B19E077D44930FF0D2A3088768F2011E95
:10E56000FEC206695D5762F7CB67658071366C192C
:10E57000E7066B6E761BD4FEE02BD3895A7ADA104D
:10E58000CC4ADD676FDFB9F9F9EFBE8E43BEB7172E
:10E59000D58EB060E8A3D6D67E93D1A1C4C2D838B8
:10E5A00052F2DF4FF167BBD16757BCA6DD06B53F1E
:10E5B0004B36B248DA2B0DD84C1B0AAFF64A03365D
:10E5C000607A0441C3EF60DF55DF67A8EF8E6E31DC
:10E5D00079BE69468CB361CB1A8366BCA0D26F2525
:10E5E00036E2685295770CCC03470BBBB916022272
:10E5F0002F260555BE3BBAC5280BBDB2925AB42B87
:10E60000046AB35CA7FFD7C231CFD0B58B9ED92C9B
:10E610001DAEDE5BB0C2649B26F263EC9CA36A7500
:10E620000A936D02A906099C3F360EEB85670772B7
:10E6300013570005824ABF95147AB8E2AE2BB17B1E
:10E64000381BB60C9B8ED2920DBED5E5B7EFDC7CA5
:10E6500021DFDB0BD4D2D38642E2D4F1F8B3DD68FC
:10E660006E83DA1FCD16BE815B26B9F6E177B06FF7
:10E670007747B718E65A0888706A0FFFCA3B0666E4
:10E680005C0B0111FF9E658F69AE62F8D3FF6B6171
:10E6900045CF6C1678E20AA0EED20DD75483044E13
:10E6A000C2B30339612667A7F71660D04D476949A1
:10E6B000DB776E3E4A6AD1AEDC5AD6D9660BDF40B4
:10E6C000F03BD83753AEBCA9C59EBBDE7FCFB24767
:10E6D000E9FFB5301CF2BDBD8AC2BACA3093B3534C
:10E6E000A6A3B4240536D0BA9306D7CD2957DE5455
:10E6F000BF67D9232E7A66B3B84A61C4021B685D2E
:10E70000942B6F2A37BE0BB4A18E0CC31BDF055AA6
:10E710008DEF022D416C6C207461736B73207374E8
:10E720006F707065640076313230002025732025CB
:10E7300073004D656D6F727920636C6561726564FD
:10E74000004E6F2066726565207461736B20656E84
:10E750007472696573000000C8E70000A56F0000CF
:10E76000D5E7000001690000E1E70000756F0000D7
:10E77000E7E70000856F0000EDE70000956F0000FF
:10E78000F3E700004D6E000009E800003569000065
:10E7900013E80000017000001BE80000716C00002D
:10E7A00024E80000F56A000030E80000116A00006B
:10E7B00039E800005D6A000041E80000C56B000018
:10E7C00073656E736F727300616363656C6572610C
:10E7D00074696F6E0074656D7065726174757265D1
:10E7E0000074696C74580074696C74590074696CB5
:10E7F000745A00736574416363656C65726F6D650F
:10E8000074657252616E676500746F7563685265F6
:10E8100061640069326352656164006932635772F2
:10E820006974650073706945786368616E67650037
:10E8300073706953657475700072656164444854FF
:10E84000006D6963726F70686F6E65005DD7000060
:10E85000E170000062D700008D7000007BE80000CE
:10E860008D71000080E80000A970000089E80000B8
:10E870002571000073657269616C007265616400E6
:10E8800072656164496E746F007772697465000027
:10E890000CE90000BD7100001AE90000CD71000014
:10E8A00027E90000C171000030E90000D1710000CB
:10E8B0003AE90000D571000043E90000D971000079
:10E8C00048E90000DD7100004DE90000E171000041
:10E8D00059E90000E571000060E90000E9710000FD
:10E8E00069E90000ED7100006EE90000F1710000BF
:10E8F00079E90000F571000083E90000C5710000AE
:10E900008DE90000C971000074667400656E616273
:10E910006C65446973706C617900736574426163FE
:10E920006B6C696768740067657457696474680024
:10E9300067657448656967687400736574506978C1
:10E94000656C006C696E65007265637400726F754A
:10E950006E6465645265637400636972636C65001C
:10E96000747269616E676C650074657874007466B2
:10E9700074546F756368656400746674546F75636E
:10E98000685800746674546F7563685900746674CF
:10E99000546F756368507265737375726500766144
:10E9A00072730000C4E9000085760000CEE9000023
:10E9B00065760000D7E9000041760000E3E9000039
:10E9C000CF75000076617245786973747300766163
:10E9D000724E616D6564007365745661724E616D4F
:10E9E0006564007661724E616D65466F72496E6452
:10E9F00065780057656C636F6D6520746F204D6995
:10EA000063726F426C6F636B732100705F73706928
:10EA100020213D204E554C4C002F686F6D652F67AF
:10EA200069742F2E706C6174666F726D696F2F70D0
:10EA300061636B616765732F6672616D65776F7275
:10EA40006B2D61726475696E6F6E6F726469636E4F
:10EA50007266352F6C69627261726965732F5350EB
:10EA6000492F5350492E63707000535049436C61D5
:10EA700073733A3A535049436C617373284E52464C
:10EA80005F5350495F547970652A2C2075696E7404
:10EA9000385F742C2075696E74385F742C2075692A
:10EAA0006E74385F74290000000000000000000050
:10EAB00059780000157800003B7800004578000088
:10EAC0004F780000397800000300000002000000C9
:10EAD000010000000400000005000000110000001B
:10EAE0000C0000000B000000120000000A000000F3
:10EAF000060000001A0000001400000017000000CB
:10EB0000160000001500000010000000FFFFFFFFCE
:10EB1000FFFFFFFF000000001E00000019000000C2
:10EB200018000000070000000800000009000000B5
:10EB30000D0000000E0000000F0000001C0000008F
:10EB40001B0000001D00000013000000000000007A
:10EB500000000000457C000079840000C57C0000B6
:10EB6000D97C0000CF7C0000417C0000357C000097
:10EB7000E57C0000617C0000317C000000000000AA
:10EB8000000000000000304300000000000030C31F
:10EB90007371727400000000FB21F93FFB210940F2
:10EBA0007CD91240FB2119407A6A1F407CD922404F
:10EBB000BBFD2540FB2129403A462C407A6A2F4074
:10EBC0005C4731407CD932409C6B3440BBFD3540C2
:10EBD000DB8F3740FB2139401BB43A403A463C407A
:10EBE0005AD83D407A6A3F404C7E40405C474140A5
:10EBF0006C1042407CD942408CA243409C6B444004
:10EC0000AC344540BBFD4540CBC64640DB8F47405A
:10EC1000EB584840FB21494083F9A200444E6E0066
:10EC2000FC291500D1572700DD34F50062DBC00058
:10EC30003C999500419043006351FE00BBDEAB0060
:10EC4000B761C5003A6E2400D24D42004906E0008B
:10EC500009EA2E001C92D100EB1DFE0029B11C0018
:10EC6000E83EA700F535820044BB2E009CE98400F5
:10EC7000B4267000417E5F00D6913900538339007D
:10EC80009CF439008B5F840028F9BD00F81F3B001D
:10EC9000DEFF97000F980500112FEF000A5A8B0036
:10ECA0006D1F6D00CF7E360009CB2700464FB700A1
:10ECB0009E663F002DEA5F00BA277500E5EBC700AE
:10ECC0003D7BF100F739070092528A00FB6BEA00A6
:10ECD0001FB15F00085D8D00300356007BFC4600CD
:10ECE000F0AB6B0020BCCF0036F49A00E3A91D0006
:10ECF0005E619100081BE60085996500A0145F0025
:10ED00008D40680080D8FF0027734D000606310053
:10ED1000CA561500C9A873007BE260006B8CC00066
:10ED200000000040FB21F93F000000002D44743E2C
:10ED3000000000809846F83C0000006051CC783B11
:10ED400000000080831BF0390000004020257A3845
:10ED5000000000802282E336000000001DF36935C8
:10ED60000200000003000000040000000600000094
:10ED7000F0A000009AA000009AA00000C8A1000026
:10ED800096A0000096A00000BEA10000C8A100004F
:10ED900096A00000BEA1000096A00000C8A100003F
:10EDA000CCA10000CCA10000CCA10000D4A10000A7
:10EDB000CCAB00003EAA000082AA0000E6A9000039
:10EDC00082AA000072AB000082AA0000E6A900003F
:10EDD0003EAA00003EAA000072AB0000E6A90000B7
:10EDE000DEA90000DEA90000DEA9000080AB000063
:10EDF000F4B20000F6B10000F6B1000014B5000056
:10EE0000F0B10000F0B10000FCB4000014B5000047
:10EE1000F0B10000FCB40000F0B1000014B5000037
:10EE20000AB500000AB500000AB5000018B50000D8
:10EE30002C2066756E6374696F6E3A20006173737F
:10EE4000657274696F6E2022257322206661696C79
:10EE500065643A2066696C6520222573222C206C3B
:10EE6000696E65202564257325730A0090000020D3
:10EE7000232D302B2000686C4C00656667454647A3
:10EE80000030313233343536373839414243444526
:10EE90004600303132333435363738396162636495
:10EEA0006566000000000000000000000000000097
:10EEB0000000000000000000000000000000000052
:10EEC0000000000000000000000000000000000042
:10EED0000000000000000000000000000000000032
:10EEE0000000000000000000000000000000000022
:10EEF0000000000000000000000000000000000012
:10EF000000000000504F53495800002020202020CE
:10EF100020202020282828282820202020202020C9
:10EF200020202020202020202020208810101010B9
:10EF3000101010101010101010101004040404040D
:10EF40000404040404101010101010104141414139
:10EF50004141010101010101010101010101010121
:10EF60000101010101011010101010104242424233
:10EF700042420202020202020202020202020202F1
:10EF80000202020202021010101020000000000015
:10EF90000000000000000000000000000000000071
:10EFA0000000000000000000000000000000000061
:10EFB0000000000000000000000000000000000051
:10EFC0000000000000000000000000000000000041
:10EFD0000000000000000000000000000000000031
:10EFE0000000000000000000000000000000000021
:10EFF0000000000000000000000000000000000011
:10F000000000000000000000000000000000000000
:08F01000F810FF7F0100000071
:10F01800FFFFFFFFE803000001000000E803DC0534
:10F02800DC05DC05DC050000FFFFFFFFFFFFFFFF3D
:10F038001800000019FCFFFFFFFFFFFF020000009F
:10F0480040420F00FF0000000024F400020000000E
:10F0580003000000FFFFFFFF0000000001000000A8
:10F068000000020001000000FFFFFFFF0000000099
:10F07800020000000000040002000000FFFFFFFF84
:10F08800000000000300000000000800030000006A
:10F098000A000000080000000100000090000020A5
:10F0A80000000000C4EE0000E4EE0000A4EE000042
:10F0B8000000000000000000000000000000000048
:10F0C8000000000000000000000000000000000038
:10F0D8000000000000000000000000000000000028
:10F0E8000000000000000000000000000000000018
:10F0F8000000000000000000000000000000000008
:10F1080043000000000000000000000000000000B4
:10F1180000000000000000000000000000000000E7
:10F128004300000000000000000000000000000094
:10F1380000000000000000000000000000000000C7
:10F148004300000000000000000000000000000074
:10F1580000000000000000000000000000000000A7
:10F168004300000000000000000000000000000054
:10F178000000000000000000000000000000000087
:10F188004300000000000000000000000000000034
:10F198000000000000000000000000000000000067
:10F1A8004300000000000000000000000000000014
:10F1B8000000000000000000000000000000000047
:10F1C80043000000000000000000000000000000F4
:10F1D8000000000000000000000000000000000027
:10F1E80021D4000039CE0000000000000AEF000022
:10F1F8007AD6000023DB000023DB000023DB0000BD
:10F2080023DB000023DB000023DB000023DB0000FE
:10F2180023DB000023DB0000FFFFFFFFFFFFFFFFF2
:10F22800FFFFFFFFFFFF0000010041534349490072
:10F2380000000000000000000000000000000000C6
:10F24800000000000000000000004153434949004D
:10F2580000000000000000000000000000000000A6
:10F26800000000000000000000000000E9000000AD
:10F27800E5770000397B0000917F0000C1000000A5
:0400000300007BD5A9
:00000001FF
